:100000000C94E7080C9406090C9406090C949609C4
:100010000C94CC090C9406090C9406090C9406095E
:100020000C9406090C9406090C9406090C94060914
:100030000C9406090C9406090C9406090C94EC0C1B
:100040000C9406090C9406090C9406090C940609F4
:100050000C9416690C94C7600C9406090C9406095C
:100060000C9406090C949C610C9406090C94906104
:100070000C9406090C9406090C9406090C940609C4
:100080000C9449740C9406090C9406090C94060906
:100090000C94DA610C9406090C94CE610C94060958
:1000A0000C9406090C9406090C9406090C94060994
:1000B0000C9406090C9406090C9406090C94060984
:1000C0000C9406090C9406090C9406090C94060974
:1000D0000C9406090C9406090C9406090C94060964
:1000E0000C9406090C94CF680C94D9680C94C568DC
:1000F0000C9485680C940A690C94FB680C94EF6866
:100100000C94E3680C9406090C9406090C940609F7
:100110000C9406090C9406090C9406090C94060923
:10012000827DA17D207E0F7F2F7F4F7F577F047FB1
:10013000084AD73B3BCE016E84BCBFFDC12F3D6C4E
:1001400074319ABD56833DDA3D00C77F11BED9E4B4
:10015000BB4C3E916BAAAABE000000803F076342E1
:1001600036B79BD8A71A39685618AEBAAB558C1D4E
:100170003CB7CC5763BD6DEDFD753EF6177231BFD0
:10018000000000803F08000000BE922449123EABF0
:10019000AAAA2ABECDCCCC4C3E00000080BEABAAA1
:1001A000AAAA3E00000000BF000000803F0000003F
:1001B0000000084178D3BB4387D1133D190E3CC3DF
:1001C000BD4282AD2B3E68EC8276BED98FE1A93E5E
:1001D0004C80EFFFBE01C4FF7F3F00000000002500
:1001E000730A005854414C5F5452494D3D256400F8
:1001F00025730A0025730A00546573742036202580
:10020000730A005465737420352025730A00546501
:10021000737420342025730A0054657374203320CE
:1002200025730A005465737420322025730A005424
:1002300065737420312025730A006368616E3D2563
:10024000640A0074787077723D25640A0035303096
:100250006B0A003235306B0A003131356B0A0035DC
:10026000366B0A0033386B0A0025730A00765F6C20
:100270006F773D252D332E32660A0025730A0073F1
:10028000656E743D252D75206475703D252D752096
:1002900069676E6F7265643D252D752074746C5F9F
:1002A0007A65726F3D252D750A0025372E3366203D
:1002B00025372E33660025352E32662000457272B2
:1002C0006F72203020566F6C74004E6F74207375FF
:1002D00070706F727465640A004572726F722030BC
:1002E00020566F6C74004572726F72203020566F0A
:1002F0006C740025630074746C3D252D64200074BB
:10030000746C3D252D6420004E65772074746C3D1F
:10031000252D6420002563004D53353631312050A2
:100320003D252D372E326620252D372E32666D0A5B
:1003300000424D5030383520256C6420506120201B
:10034000252D372E32666D00256300545F484541E8
:10035000545F4944583D252D352E32662000545FA8
:100360004445573D252D352E3266200041483D2518
:100370002D352E32662000545F53485432583D25A7
:100380002D352E3266200052485F53485432583D76
:10039000252D352E32662000545F52483D252D34E0
:1003A0002E3166200052483D252D342E3166200026
:1003B0002563002563002563002563002563007223
:1003C00065706F72745F616C6C3D007265706F7206
:1003D000743D00256300256300256300256300202C
:1003E0004F534343414C3D256420002046757365BF
:1003F0003A2065653D253032782068663D253032EB
:1004000078206C663D25303278206C623D25303294
:1004100078004D43553D2530366C780025630074D7
:10042000785F6C656E3D252D6C752C765F6C6F77F3
:100430003D252D6C752C73687432783D252D6C75B7
:100440000A002563004F4B0A002563002563002541
:100450006300256300256300256300256300256391
:100460000064656275675F616C6C3D006465627510
:10047000673D0064656275673D0025730A00646529
:1004800065700A006E6F6E650A00707772733D00CA
:10049000696E74725F7365635F70313D252D372E11
:1004A00033660A00696E74725F70313D252D6C648D
:1004B0000A00696E74725F7365635F70303D252D4D
:1004C000372E33660A00696E74725F70303D252DD9
:1004D0006C640A00765F6D63753D252D352E32669E
:1004E0000A00745F6D63753D252D352E32660A0056
:1004F000707077723D25730A0064656275673D0010
:1005000072636D643D25730A0025730A006175747A
:100510006F0A006C6F675F6D6F64653D0075736295
:100520005F7077723D25730A0072656C61793D25B5
:10053000730A0074746C3D252D640A0052494D45C0
:100540005F616464723D252D642E252D640A006E62
:1005500065696768626F725F7461626C655F736919
:100560007A653D25640A00765F6C6F773D252D33F3
:100570002E32660A00747870773D25640A0063683D
:10058000616E3D25640A006932633D0069643D0087
:100590007478743D25730A0053797374656D205324
:1005A000756D6D6172790A006D61736B3D002C0091
:1005B000696E74657276616C3D252D750023252D5D
:1005C000642C00745F686561745F69647800745FAF
:1005D00064657700616800705F6D73353631310096
:1005E00072685F736874327800745F73687432780D
:1005F0000070610070006164340061643300616404
:100600003200616431006133006132006131007693
:100610005F696E00726800757074696D6500703195
:100620005F6C73740070315F740070310070305F04
:100630006C73740070305F7400703000765F6D63AF
:100640007500745F6D637500743100740069640037
:1006500065363400747874002D002B006175746F5A
:10066000006E6F6E6500706F7765725F736176659F
:100670005F6C656472790072656C61795F6C65644A
:100680007900636F6D7061737300616363656C0003
:100690007072657300705F707772006165730070CF
:1006A000315F6C6564790070305F6C656472006501
:1006B00076656E74006C6564006F7700706B740013
:1006C00074785F6C6564790072785F6C6564720041
:1006D0006F706572006E6F6E65002530327800763F
:1006E0005F6164343D252D382E3666002000765F2C
:1006F0006164333D252D382E3666002000765F611B
:1007000064323D252D382E3666002000765F616408
:10071000313D252D382E3666002000765F6C6967E6
:1007200068743D252D382E3666002000765F6132D4
:100730003D252D372E3366002000765F61313D2543
:100740002D372E3366002000765F696E3D252D35EE
:100750002E326600204E657665722D7573656420B5
:10076000737461636B203E20256420627974657325
:100770000A00757074696D653D252D642D6461797D
:10078000732D253032643A253032643A2530326494
:100790002D686F7572730A0074657374205B6F66E1
:1007A000667C317C327C337C347C355D202020209B
:1007B000202020202D2074657374206D6F64657374
:1007C0000A0D007478205B706B74207061796C6F17
:1007D00061645D2020202020202020202020202D4A
:1007E0002073656E6420726164696F20706B742081
:1007F0006B6579626F6172640A0D00776474205BC7
:100800006F6E7C6F66667C746573745D202020203B
:10081000202020202020202D207761746368646FC1
:10082000670A0D00765F6C6F77205B765F6C6F7781
:100830005D2020202020202020202020202020207B
:100840002D206C6F77657374207265706F727420E1
:10085000766F6C746167650A0D0075706772202091
:100860002020202020202020202020202020202088
:100870002020202020202D207265626F6F7420764A
:10088000696120626F6F746C6F616465720A0D003C
:1008900075617274205B33386B7C35366B7C31311B
:1008A000356B7C3235306B7C3530306B5D202D20E4
:1008B000736574207465726D2F7561727420737026
:1008C0006565640A0D00626F6F742020202020206F
:1008D0002020202020202020202020202020202018
:1008E00020202D207265626F6F740A0D0070777280
:1008F00073205B646565707C6E6F6E655D20202083
:100900002020202020202020202D206D63752073A2
:100910006C656570206D6F64650A0D007265737497
:1009200020656570726F6D202020202020202020FF
:1009300020202020202020202D20726573746F72CB
:100940006520656570726F6D0A0D0070707772209A
:100950005B6F6E7C6F66665D20202020202020204B
:10096000202020202020202D2070726F6772616D62
:100970006D61626C65207077720A0D007478742066
:100980005B737472696E675D202020202020202018
:1009900020202020202020202D20536574207265E7
:1009A000706F7274207465787420737472696E67E6
:1009B0000A0D0074787077205B31352D305D202072
:1009C0002020202020202020202020202020202D1A
:1009D000205458205077722E2048696768657374D8
:1009E000203020283364426D290A0D0074746C2075
:1009F0005B302D31355D202020202020202020203C
:100A000020202020202020202D2074696D652D7449
:100A10006F2D6C69766520666F72207061636B65FF
:100A200074730A0D007373202020202020202020C2
:100A300020202020202020202020202020202020B6
:100A4000202D2073797374656D2073756D6D6172DF
:100A5000790A0D00727320202020202020202020E1
:100A60002020202020202020202020202020202086
:100A70002D20726164696F2073746174730A0D00B4
:100A80007269205B236E5D205B696E745D2020209F
:100A90002020202020202020202020202D207265B2
:100AA000706F727420696E74657276616C0A0D00E5
:100AB00072636D64205B6F6E7C6F66665D202020C4
:100AC0002020202020202020202020202D20616C8C
:100AD0006C6F7720636D642066726F6D206E657435
:100AE0006F726B0A0D007265205B236E5D205B2BBD
:100AF0007C2D5D205B6D61736B7C6175746F2C6DFB
:100B000061736B5D202D206D6F7465207265706F51
:100B10007274207365742F6D6F646966790A0D00B5
:100B20006F7720202020202020202020202020201F
:100B30002020202020202020202020202D206F6E0B
:100B4000652D776972652073656E736F72730A0D18
:100B5000006C6F67205B6175746F7C6F6E7C6F6675
:100B6000665D20202020202020202020202D206DA8
:100B70006F7465732064617461206F6E20555342F9
:100B80000A0D006E65205B666C7573685D20202021
:100B90002020202020202020202020202020202D48
:100BA000206E65696768626F72207461626C650AA5
:100BB0000D0065727220202020202020202020207F
:100BC00020202020202020202020202020202D2018
:100BD0006572726F722073746174730A0D006D63B5
:100BE00075202020202020202020202020202020B0
:100BF000202020202020202020202D206D63752003
:100C0000696E666F0A0D006964205B7265736574B6
:100C10005D20202020202020202020202020202097
:100C20002020202D2069642068616E646C696E67E5
:100C30000A0D0068756D2020202020202020202013
:100C40002020202020202020202020202020202D97
:100C50002068756D69646974792073656E736F724D
:100C60000A0D0072656C6179205B6F6E7C6F666641
:100C70007C73746174735D20202020202020202D3F
:100C80002072656C6179206E6574776F726B20726B
:100C900065706F7274730A0D006465205B6D61731B
:100CA0006B5D2020202020202020202020202020BC
:100CB00020202020202D2064656275670A0D0063C6
:100CC00068616E205B31312D32365D20202020207E
:100CD00020202020202020202020202D206368613B
:100CE0006E2031312D32362028322E3430352D32DF
:100CF000343830204D687A290A0D0063616C692010
:100D00005B5B765F696E7C61317C61325D20766F02
:100D10006C747C72657365747C6E6F6E655D202D7E
:100D20002063616C6962726174650A0D00616463BD
:100D300020202020202020202020202020202020B3
:100D40002020202020202020202D2073686F772055
:100D5000765F696E2C2061312C20613220766F6CB9
:100D600074616765730A0D00752020202020202003
:100D70002020202020202020202020202020202073
:100D8000202020202D20757074696D650A0D007675
:100D90002020202020202020202020202020202053
:100DA00020202020202020202020202D2076657249
:100DB00073696F6E0A0D00682020202020202020FB
:100DC0002020202020202020202020202020202023
:100DD0002020202D2068656C700A0D0025630075A9
:100DE0006E6B6E6F776E20636D640A00484D4335FD
:100DF0003838330025730025730020257300202523
:100E0000362E32662000253032780074656D705FB2
:100E100065787465726E3D252D362E32660020256C
:100E200073002025362E3266204F6E2D426F617280
:100E30006400253032780074656D705F626F617296
:100E4000643D252D362E3266000A00503A20256C6E
:100E5000642050612020252D372E3266206D0A0037
:100E60002563002563004932433A2000452025646C
:100E70002E256420636C6F636B20256C7520637076
:100E80007520256C75206C706D20256C752069723D
:100E90007120256C7520676C656420256C75207940
:100EA0006C656420256C7520726C656420256C75FA
:100EB00020747820256C75206C697374656E20250C
:100EC0006C752073656E736F727320256C7520735B
:100ED000657269616C20256C750A00532025642EAB
:100EE000256420636C6F636B20256C7520747820FB
:100EF000256C7520727820256C75207274782025F9
:100F00006C752072727820256C75207265786D6919
:100F10007420256C752061636B747820256C7520B6
:100F20006E6F61636B747820256C752061636B72E2
:100F30007820256C752074696D65646F7574202543
:100F40006C752062616461636B727820256C75201A
:100F5000746F6F6C6F6E6720256C7520746F6F7384
:100F6000686F727420256C752062616473796E639A
:100F70006820256C752062616463726320256C753E
:100F800020636F6E74656E74696F6E64726F70202B
:100F9000256C752073656E64696E6764726F70206E
:100FA000256C75206C6C747820256C75206C6C72C7
:100FB0007820256C750A00257325730A004F6E6C26
:100FC000696E650A000A002C20636865636B2072F5
:100FD00061746520257520487A0025732025732CBF
:100FE000206368616E6E656C20257520706F776573
:100FF00072202575000A0025783A004D4143206192
:10100000646472657373200052616E646F6D204575
:101010005549363420616464726573732067656E68
:101020006572617465640A000A2A2A2A2A2A2A2A11
:10103000426F6F74696E672025732A2A2A2A2A2A2A
:101040002A0A00454550524F4D20697320636F7244
:10105000727570742C20726577726974696E67207E
:10106000776974682064656661756C74732E0A0014
:101070006C6F63616C686F73740041544D454741F8
:101080003132387266613100020000FFFE0000015B
:101090006E616E00696E660000407A10F35A00A01F
:1010A000724E18090010A5D4E80000E87648170031
:1010B00000E40B54020000CA9A3B000000E1F50571
:1010C000000080969800000040420F000000A086BB
:1010D00001000000102700000000E80300000000ED
:1010E0006400000000000A00000000000100000091
:1010F00000002C76D888DC674F0823DFC1DFAE59AB
:10110000E1B1B796E5E3E453C63AE651997696E83D
:10111000E6C28426EB898C9B62ED407C6FFCEFBCC1
:101120009C9F40F2BAA56FA5F490055A2AF75C93EC
:101130006B6CF9676DC11BFCE0E40D47FEF520E622
:10114000B500D0ED902E0300943577050080841E05
:10115000080000204E0A000000C80C333333330F60
:10116000986E12831141EF8D2114893BE65516CFFD
:10117000FEE6DB18D1844B381BF77C1D901DA4BB09
:10118000E424203284725E228100C9F124ECA1E5BE
:101190003D274E414E494E495459494E46CDCCCC3F
:1011A0003D0AD7233C17B7D13877CC2B329595E63B
:1011B000241FB14F0A000020410000C84200401C1B
:1011C0004620BCBE4CCA1B0E5AAEC59D74001124ED
:1011D0001FBECFEFD1E4DEBFCDBF19E0A0E0B2E08B
:1011E000ECE8F4E201E00BBF02C007900D92AC36D0
:1011F000B107D9F711E3ACE6B9E001C01D92A13205
:10120000B107E1F70E9426800C9444920C940000F0
:101210008AE894E09F938F930E941D8F80915402DF
:10122000909155020F900F9093FF03C084E894E0D3
:1012300002C08EE794E09F938F930E941D8F0F90C2
:101240000F900895E091251BEF71F0E0E658F44E01
:1012500080838091251B8F5F8093251B80915B2865
:10126000886080935B284EE352E061E1CA010E94EE
:10127000B65080E090E00895CF93DF93EC01809129
:1012800073099091740986FF1DC08E811F928F9300
:101290008D811F928F938C811F928F938B811F92D0
:1012A0008F938A811F928F938FE593E09F938F9303
:1012B0000E940B8F8DB79EB70C960FB6F8949EBF09
:1012C0000FBE8DBFBE018AEA99E00E94E851BE01BF
:1012D00084E092E0DF91CF910C945D5187EE93E032
:1012E0008115910511F00197F1F708958823B9F060
:1012F00052985A981DBA8091690080628093690063
:10130000EA9A53985B98EB9A809169008068809381
:101310006900809168008160809368000895109250
:1013200069005A9AEA985B9AEB9808951F920F9277
:101330000FB60F9211248F939F93AF93BF93809119
:10134000680080FF20C08091362890913728A091B6
:101350003828B09139280196A11DB11D80933628F7
:1013600090933728A0933828B09339288091730937
:101370009091740987FF07C0749882E090E0909381
:101380007F0280937E02BF91AF919F918F910F90CA
:101390000FBE0F901F9018951F920F920FB60F92CD
:1013A00011248F939F93AF93BF938091680080FF28
:1013B00020C080913A2890913B28A0913C28B09180
:1013C0003D280196A11DB11D80933A2890933B289A
:1013D000A0933C28B0933D288091730990917409A3
:1013E00090FF07C0739882E090E090937F02809313
:1013F0007E02BF91AF919F918F910F900FBE0F9082
:101400001F90189580937C0080917B00877F80934C
:101410007B0080917C00806C80937C0085E08093D1
:101420007A0080917A00806880937A0080917B00B6
:1014300087FFFCCF80917B0085FFFCCF80917A00F5
:10144000806480937A0080917A0086FDFCCF1092B0
:1014500079001092780084E090E060E070E02091E4
:101460007A00206420937A0020917A0026FDFCCF38
:101470002091780030917900620F731F01970097D7
:1014800071F710927C0080917A008F7780937A00B8
:10149000769567957695679580E090E00E947C85CB
:1014A000089580E00E94020A20917602309177022E
:1014B00040917802509179020E945C8721EE3AE7D0
:1014C00044E95EE30E941584089580E18093510110
:1014D00060E1609351018091510185FF03C06F5F0E
:1014E0006F31B9F78BE4689FB0011124882777FD2D
:1014F0008095982F0E947E8520E030E64FE954E4E5
:101500000E94158420E030E04AE754E40E94DF8422
:101510000895CF93DF93EC0188819981009799F02A
:101520008A30904121F01982188283E011C0623123
:1015300071F40E94650A6093CD237093CE2380934B
:10154000CF239093D0238AE090E19983888381E030
:10155000DF91CF91089580917B00886080937B001C
:1015600089EC80937C0085E080937A0080917A00FA
:10157000806880937A0080917B0087FFFCCF809108
:101580007B0085FFFCCF80917A00806480937A0095
:1015900080917A0086FDFCCF80917A0080648093F0
:1015A0007A0080917A0086FDFCCF6091780070917E
:1015B000790080917A008F7780937A0080E090E0C4
:1015C0000E947C8527ED33EA40E95FE30E945C8757
:1015D00026E636E648E853E40E9414840895BF9254
:1015E000CF92DF92EF92FF920F931F93CF93DF93EF
:1015F000CDB7DEB729970FB6F894DEBF0FBECDBFCB
:101600006C0110926C098FEF898706E31BE1B12C06
:101610007E0189E0E80EF11C89858823E9F1E8E084
:10162000BE16E1F1BE016F5F7F4FC7010E94515AA4
:1016300089858F3F11F08E3F19F480936C092CC07F
:10164000CE010196C114D10471F40E946A5A8093AC
:101650005828FE013196A0E5B8E281918D93EE15F0
:10166000FF05D9F71DC00E946A5AF8018083FE0168
:10167000319620E030E0A801485051098191DA010B
:10168000A20FB31F8C932F5F3F4F28303105B1F766
:10169000B394075F1F4FC0CF8B2D03C088E001C0FC
:1016A00081E029960FB6F894DEBF0FBECDBFDF9163
:1016B000CF911F910F91FF90EF90DF90CF90BF904F
:1016C000089589E49EE09F938F930E941D8F0F9051
:1016D0000F9008952F923F924F925F926F927F9258
:1016E0008F929F92AF92BF92CF92DF92EF92FF9232
:1016F0000F931F93CF93DF93EC014B01009711F4ED
:1017000027E004C08130910549F426E04AE250E028
:101710006BE270E089E290E00E943159CE010E94B4
:10172000EF0A9E012359364F5901D9018C93CD2BD5
:1017300069F096E3C92E9BE1D92ECEE2DBE1E12CE4
:10174000F12C2AEF222E2DE0322EA6C080E598E261
:101750000E949F5BBC01882777FD8095982F0E948F
:101760007E856B017C01892869F020E030E048EC3F
:1017700052E40E94DF849F938F937F936F9387E35C
:101780009EE0ACC0C0E5D8E202E31EE089911F9262
:101790008F931F930F930E941D8F0F900F900F90A8
:1017A0000F90B8E2C835DB0789F720E030E048EC5D
:1017B00052E4C701B6010E94DF849F938F937F9309
:1017C0006F9382E29EE09F938F930E941D8F0F90F4
:1017D0000F900F900F900F900F90809158288823B2
:1017E00019F08EE893E002C082E094E09F938F931B
:1017F0008EE19EE09F938F930E941D8F0F900F901C
:101800000F900F9075C000E010E0FE01E00FF11F97
:1018100080811F928F93A6E0BEE0BF93AF930E949A
:101820001D8F0F5F1F4F0F900F900F900F9008307C
:10183000110559F720E030E048EC52E4C301B20151
:101840000E94DF849F938F937F936F93AEEFBDE0F1
:10185000BF93AF930E941D8F0F900F900F900F902A
:101860000F900F90D6018C91882309F455C08EE813
:1018700093E09F938F933F922F920E941D8F0E941F
:10188000610BBFEFEB1AFB0AE9E0CE0ED11C2996E3
:101890000F900F900F900F90D5018C9190E0E8166B
:1018A000F906ECF5CE010E949F5BBC01882777FD0D
:1018B0008095982F0E947E852B013C018114910414
:1018C00009F4A1CF20E030E048EC52E40E94DF842C
:1018D0009F938F937F936F938BE09EE09F938F9363
:1018E0000E941D8F0F900F900F900F900F900F90F0
:1018F000DF91CF911F910F91FF90EF90DF90CF90EC
:10190000BF90AF909F908F907F906F905F904F901F
:101910003F902F900C94610B82E094E0AACFDF916E
:10192000CF911F910F91FF90EF90DF90CF90BF90DC
:10193000AF909F908F907F906F905F904F903F906F
:101940002F900895CF93DF9300D0CDB7DEB780916D
:1019500051288983809157288A83CE0101960E945D
:10196000AA4E0F900F90DF91CF910895CF93DF9300
:10197000EC012091502830915128409152285091EB
:101980005328609154287091552880915628909141
:101990005728AFEF0E948C8AE1F427E04AE250E03A
:1019A0006BE270E089E290E00E94315980E090E0C3
:1019B0000E94EF0AC359D64F888349E050E06AE09D
:1019C00070E080E598E20E948F90DF91CF910C94B7
:1019D000A20CDF91CF9108951F920F920FB60F9234
:1019E00011240BB60F92DF92EF92FF920F931F9389
:1019F0002F933F934F935F936F937F938F939F9317
:101A0000AF93BF93CF93DF93EF93FF9380915B28C6
:101A1000826080935B288091540286FD2B9A80918E
:101A2000540287FD2B9A80917E0290917F021816B6
:101A3000190614F4749A739A809173099091740939
:101A400085FF02C0749873988091020290910302FE
:101A500001979093030280930202892B09F039C108
:101A600080918109909182090196909382098093D7
:101A700081098091D1239091D223A091D323B09159
:101A8000D4230196A11DB11D8093D1239093D2231D
:101A9000A093D323B093D42380E190E090930302EA
:101AA000809302028091540280FD02C01D9B07C0FA
:101AB000109271091092700983B7817F09C081E08B
:101AC00090E0909371098093700983B7817F86605D
:101AD00083BF809173099091740997FF08C080912A
:101AE000700990917109892B61F0749A739805EDD2
:101AF0001AE1C2EED3E234E0E32EF12CDD24D394DC
:101B00001FC0739A7498F3CF8091810990918209D4
:101B100001960E945D88892BD1F0F801608571855E
:101B20006115710509F5F80160857185611571050B
:101B300069F5065F1F4F2596FAE10D3F1F07D1F1AA
:101B4000F801608571856115710539F3DDCF7798EE
:101B5000809173099091740992FFDFCF7498F0928D
:101B60007F02E0927E02D9CF809181099091820913
:101B700001960E945D88892BB1F61C821B82AE0102
:101B800062E186E192E00E94B650CDCF809181095A
:101B9000909182090E945D88892B59F6D8821A8318
:101BA00009831C821B82AE0162E184E392E00E9401
:101BB000B650BFCF609158027091590261157105FE
:101BC000A1F180918109909182090E945D88892B01
:101BD00061F58091362890913728A0913828B091EE
:101BE00039284091C31B5091C41B6091C51B709153
:101BF000C61B841B950BA60BB70B8093FD1A909305
:101C0000FE1AA093FF1AB093001B80913628909182
:101C10003728A0913828B09139288093C31B90931E
:101C2000C41BA093C51BB093C61B60915602709154
:101C3000570261157105A1F1809181099091820986
:101C40000E945D88892B61F580913A2890913B280C
:101C5000A0913C28B0913D284091C71B5091C81BD2
:101C60006091C91B7091CA1B841B950BA60BB70B07
:101C70008093011B9093021BA093031BB093041B42
:101C800080913A2890913B28A0913C28B0913D2822
:101C90008093C71B9093C81BA093C91BB093CA1B0A
:101CA0008091540286FD2B988091540290915502A8
:101CB00091FF0FC00E9441658A3119F0C1E0C80F41
:101CC00001C0CBE00E94FB638C2F0E9459650E94EB
:101CD000436440E050E060E080E892E00E94B6504B
:101CE000FF91EF91DF91CF91BF91AF919F918F9134
:101CF0007F916F915F914F913F912F911F910F9124
:101D0000FF90EF90DF900F900BBE0F900FBE0F90E3
:101D10001F9018958091251B9091E123891B0895B0
:101D20000E948A0E882371F0E091E123EF71F0E0C8
:101D3000E658F44E808190E02091E1232F5F2093BC
:101D4000E12308958FEF9FEF0895CF93DF93EC0188
:101D500010929E0910929D09888199810097C1F087
:101D60008E36934021F01982188283E0B6C061312B
:101D700009F0B2C0F89478940E94900E992790933D
:101D80009909809398098D3009F441C08F3F49F437
:101D90000E948A0E8111EECF8EE693E099838883AC
:101DA0009BC08231910509F458C08F37910509F025
:101DB00050C08091960990919709181619060CF554
:101DC00060911B3170911C3188E090E00E94D98EA7
:101DD00060911B3170911C3180E290E00E94D98E9D
:101DE00060911B3170911C3188E090E00E94D98E87
:101DF0008091960990919709019790939709809304
:101E000096098091960990919709CF9709F61092BB
:101E1000E1231092251B8091960990919709FC016E
:101E2000EA50FC4D108290939E0980939D09109278
:101E30009709109296098091592890915A280097F5
:101E400009F4A6CF40E050E06091AC110E94B6507A
:101E50009FCF8830910571F5ACCF60911B317091A7
:101E60001C318DE090E00E94D98E1092950910925D
:101E70009409809194099091950920919609309147
:101E80009709821793070CF0BCCFFC01EA50FC4D78
:101E9000808160911B3170911C3190E00E94D98E3D
:101EA000809194099091950901969093950980935A
:101EB0009409DFCF60911B3170911C310E94D98E43
:101EC000809196099091970920919809FC01EA5018
:101ED000FC4D2083019691CF81E0DF91CF91089551
:101EE0008091700990917109892BB1F08091540211
:101EF0009091550293FD10C00E94FB6383B7817FD0
:101F0000866083BFF89483B7816083BF7894889597
:101F100083B78E7F83BF78940895CF93DF93EC01CE
:101F200088819981009719F08D33904199F40E942E
:101F3000B8620E94700F40E050E065E88091B011F7
:101F40009091B1110E94B6508DE390E199838883FE
:101F500081E003C01982188283E0DF91CF91089558
:101F6000CF93DF9300D0CDB7DEB7892B81F05F939D
:101F70004F9387EF9DE09F938F9369837A830E94AD
:101F80001D8F0F900F900F900F907A8169817F9332
:101F90006F9384EF9DE09F938F930E941D8F0F900E
:101FA0000F900F900F900F900F90DF91CF910895A9
:101FB000FF920F931F93CF93DF930E94B86280EB41
:101FC0000E941D5C81111CC00E94815C8091CB1F0E
:101FD0009091CC1F81609093CC1F8093CB1F87E999
:101FE00093E09F938F9384EF9DE09F938F930E9444
:101FF0001D8F0F900F900F900F90C1E0D0E002C0A6
:10200000C0E0D0E0FEB08F2D8470F82E729A0E944E
:10201000B8628EE40E941D5C811116C00E94815C32
:102020008091CB1F9091CC1F82609093CC1F8093A6
:10203000CB1F8E010F5F1F4F42ED58E06FE973E039
:10204000CE010E94B00FE801F11001C072980E9409
:10205000B8628EEE0E941D5C811116C00E94815CE8
:102060008091CB1F9091CC1F84609093CC1F809364
:10207000CB1F8E010F5F1F4F42ED58E067EA73E000
:10208000CE010E94B00FE8010E94B86286EA0E9469
:102090001D5C811116C00E94815C8091CB1F9091C4
:1020A000CC1F88609093CC1F8093CB1F8E010F5F55
:1020B0001F4F42ED58E06EEA73E0CE010E94B00F70
:1020C000E8010E94B8628CE30E941D5C81111EC071
:1020D0000E94815C8091CB1F9091CC1F8061909376
:1020E000CC1F8093CB1F8E010F5F1F4F42ED58E036
:1020F00066EB73E0CE010E94B00F8CEE9DE09F93E3
:102100008F930E941D8F0F900F90E8010E94B8627C
:1021100082ED0E941D5C811116C00E94815C80913D
:10212000CB1F9091CC1F80629093CC1F8093CB1FCC
:102130008E010F5F1F4F42ED58E06EEB73E0CE0152
:102140000E94B00FE8010E94B86280E80E941D5C06
:10215000811116C00E94815C8091CB1F9091CC1F91
:1021600091609093CC1F8093CB1F8E010F5F1F4F08
:1021700042ED58E067EC73E0CE010E94B00FE80139
:102180000E94B86280ED0E941D5C811116C00E9401
:10219000815C8091CB1F9091CC1F80689093CC1F65
:1021A0008093CB1F8E010F5F1F4F42ED58E06DEC07
:1021B00073E0CE010E94B00FE8010E94B8628CEE7D
:1021C0000E941D5C811116C00E94815C8091CB1F12
:1021D0009091CC1F92609093CC1F8093CB1F8E0167
:1021E0000F5F1F4F42ED58E065ED73E0CE010E9496
:1021F000B00FE80107E010E00E94B8628CE70E948F
:102200001D5C811113C00E94815C8091CB1F909155
:10221000CC1F80649093CC1F8093CB1F42ED58E07D
:102220006CED73E0CE010E94B00F05C001501109A2
:102230000115110509F70E94815CDF91CF911F9173
:102240000F91FF900C94610BCF93DF9300D0CDB72B
:10225000DEB74A8369830E94585C6981862F0E9499
:10226000895C4A81842F0E94895C0F900F90DF91D6
:10227000CF910C94815CAF92BF92DF92EF92FF926C
:102280000F931F93CF93DF9300D01F92CDB7DEB78C
:10229000182FD22E4A835B8369830E94585C698120
:1022A000862F0E94895C812F81600E947F5C4A8119
:1022B000A42E5B81B52E00E010E0ED2CF12C81E026
:1022C000E81AF1080D1580F40E151F0519F40E9487
:1022D000A45C02C00E949A5CF50180830F5F1F4FCF
:1022E000FFEFAF1ABF0AEECF0F900F900F90DF9164
:1022F000CF911F910F91FF90EF90DF90BF90AF9023
:102300000C94815CAF92BF92CF92DF92EF92FF92DA
:102310000F931F93CF93DF93CDB7DEB760970FB6C0
:10232000F894DEBF0FBECDBFB82EA42E6623E9F110
:102330008E010F5F1F4F80E1F80111928A95E9F736
:1023400028E0A80168E980EB0E943B11BB2041F026
:1023500025EE33E03F932F930E940B8F0F900F9049
:102360006E01F8E0CF0ED11C5CEEE52E53E0F52EA9
:10237000F80181918F011F928F93FF92EF920E943B
:102380000B8F0F900F900F900F900C151D0581F77C
:1023900088851F928F9321E434E03F932F930E940E
:1023A0000B8F0F900F900F900F90AA20E9F18E01E4
:1023B0000F5F1F4F80E1F80111928A95E9F728E03D
:1023C000A80160E880EB0E943B11BB2041F081EF47
:1023D00093E09F938F930E940B8F0F900F906E014D
:1023E000F0E1CF0ED11C4CEEE42E43E0F42EF801C8
:1023F00081918F011F928F93FF92EF920E940B8F1A
:102400000F900F900F900F900C151D0581F7888588
:102410001F928F9381E494E09F938F930E940B8F80
:102420000F900F900F900F9060960FB6F894DEBF4C
:102430000FBECDBFDF91CF911F910F91FF90EF9015
:10244000DF90CF90BF90AF900895CF93DF9300D0EF
:10245000CDB7DEB71A82198222E0AE014F5F5F4F1F
:102460006AEA8EEE0E943B11898190E0982F8827BE
:102470002A81822B90939B1B80939A1B22E0AE01B2
:102480004F5F5F4F6CEA8EEE0E943B11898190E0B6
:10249000982F88272A81822B90939D1B80939C1BC9
:1024A00022E0AE014F5F5F4F6EEA8EEE0E943B115D
:1024B000898190E0982F88272A81822B90939F1BF7
:1024C00080939E1B22E0AE014F5F5F4F60EB8EEE6C
:1024D0000E943B11898190E0982F88272A81822BC6
:1024E0009093AD1B8093AC1B22E0AE014F5F5F4F1A
:1024F00062EB8EEE0E943B11898190E0982F882735
:102500002A81822B9093AF1B8093AE1B22E0AE01F9
:102510004F5F5F4F64EB8EEE0E943B11898190E02C
:10252000982F88272A81822B9093B11B8093B01B10
:1025300022E0AE014F5F5F4F66EB8EEE0E943B11D3
:10254000898190E0982F88272A81822B9093A11B64
:102550008093A01B22E0AE014F5F5F4F68EB8EEED1
:102560000E943B11898190E0982F88272A81822B35
:102570009093A31B8093A21B22E0AE014F5F5F4F9D
:102580006AEB8EEE0E943B11898190E0982F88279C
:102590002A81822B9093A71B8093A61B22E0AE0179
:1025A0004F5F5F4F6CEB8EEE0E943B11898190E094
:1025B000982F88272A81822B9093A91B8093A81B90
:1025C00022E0AE014F5F5F4F6EEB8EEE0E943B113B
:1025D000898190E0982F88272A81822B9093AB1BCA
:1025E0008093AA1B0F900F90DF91CF9108952F92A7
:1025F0003F924F925F926F927F928F929F92AF9293
:10260000BF92CF92DF92EF92FF920F931F93CF93DF
:10261000DF93CDB7DEB76A970FB6F894DEBF0FBE73
:10262000CDBF182F488F298F19821A821B82809163
:10263000BE1B811107C06A8F0E94251281E0809322
:10264000BE1B6A8D662309F46CC04EE264EF8EEE09
:102650000E94241169E07AE180E090E00E940A5C27
:1026600022E0AE014F5F5F4F66EF8EEE0E943B119E
:102670002981822F90E0A0E0B0E02227382F492F57
:102680005A2F8A81282B8091B01B9091B11B281B57
:10269000390B41095109A091AE1BB091AF1B0E94AB
:1026A0003A886B017C018FE0F594E794D794C79446
:1026B0008A95D1F76091A81B7091A91B882777FD97
:1026C0008095982F2BE0660F771F881F991F2A95FA
:1026D000D1F72091AA1B3091AB1B442737FD4095C1
:1026E000542F2C0D3D1D4E1D5F1D0E94A788C20E4C
:1026F000D31ED092A51BC092A41B88E0C80ED11C8B
:1027000034E0D594C7943A95E1F7EE24D7FCE094F1
:10271000FE2CC092B21BD092B31BE092B41BF0927D
:10272000B51B012F0295000F000F007C0C5CA12F40
:10273000B0E0BD8BAC8BA3E0B0E0012E02C0AA0FCD
:10274000BB1F0A94E2F725E335E00E943388DC01E1
:10275000CB010296A11DB11D8C879D87AE87BF87D7
:1027600080E593ECA0E0B0E004C0B595A7959795FF
:1027700087951A95D2F7888B998BAA8BBB8B10E023
:10278000188619861A861B86A8E02A2E312CAC8959
:10279000BD892A1A3B0A988D191709F436C1402FB2
:1027A00064EF8EEE0E9424116C857D858E859F8559
:1027B0000E940A5C23E0AE014F5F5F4F66EF8EEE32
:1027C0000E943B11E091A41BF091A51BE05AFF4031
:1027D0009F01DF010E941C886B017C0180919C1B82
:1027E00090919D1B9F8B8E8BA0909A1BB0909B1BF2
:1027F00020919E1B30919F1B0E941C882B013C0145
:102800003DE075946794579447943A95D1F7A09119
:10281000A01BB091A11BA70196016CE055954795AF
:10282000379527956A95D1F70E944588BB2797FD74
:10283000B095AB2F480E591E6A1E7B1E92E0490EC2
:10284000511C611C711CB2E07594679457944794B5
:10285000BA95D1F7A0E85A0E611C711CA091AC1B6F
:10286000B091AD1BA30192010E943A88DC01CB011B
:102870002FE0B695A795979587952A95D1F78C83E4
:102880009D83AE83BF8329818A8190E0A0E0B0E080
:102890004424582E692E7A2E622A8B81482A022CD3
:1028A00004C075946794579447940A94D2F74501ED
:1028B000AA2497FCA094BA2C42E0880C991CAA1C6C
:1028C000BB1C4A95D1F7A091A21BB091A31BA701F5
:1028D00096010E9445886B017C0157E1F594E794CD
:1028E000D794C7945A95D1F72E893F89DF010E946A
:1028F0001C88EBE09595879577956795EA95D1F7D4
:10290000C60ED71EE81EF91E8C0C9D1CAE1CBF1CEB
:102910000C8804C0880C991CAA1CBB1C0A94D2F712
:1029200092E0890E911CA11CB11CF2E0B594A79411
:1029300097948794FA95D1F7481859086A087B0844
:10294000A3019201688979898A899B890E944D88AF
:1029500097FD0DC0660F771F881F991F2C813D8141
:102960004E815F810E94858849015A010CC02C81EB
:102970003D814E815F810E94858849015A01880C02
:10298000991CAA1CBB1C9927B7FC9A958B2D7A2DF4
:10299000692D9B01AC010E944D889B01AC01AEEDFD
:1029A000BBE00E943A886C01FF24D7FCF094EF2C26
:1029B000A3E4B3EEA50194010E944888BB2797FDCC
:1029C000B095AB2FC80ED91EEA1EFB1EAFECCA0E87
:1029D000AEE0DA1EE11CF11CA4E0F594E794D79474
:1029E000C794AA95D1F7C80CD91CEA1CFB1C888592
:1029F0009985AA85BB858C0D9D1DAE1DBF1D888741
:102A00009987AA87BB871F5FC6CE112391F0212F1C
:102A100030E040E050E0688579858A859B850E949A
:102A200085882093B61B3093B71B4093B81B5093F7
:102A3000B91BA98DAA2389F16091B61B7091B71BB0
:102A40008091B81B9091B91B6115710581059105A5
:102A500021F10E947E8520E836EE45EC57E40E9485
:102A6000DF8421E03EED42E45EE30E94BF879B01EC
:102A7000AC0160E070E080E89FE30E9414842BE4E6
:102A80003AE34DEB57E30E94DF846093BA1B7093E7
:102A9000BB1B8093BC1B9093BD1B6A960FB6F8942A
:102AA000DEBF0FBECDBFDF91CF911F910F91FF9081
:102AB000EF90DF90CF90BF90AF909F908F907F90DE
:102AC0006F905F904F903F902F9008950F931F93BA
:102AD000CF93DF9300D000D000D0CDB7DEB78E010A
:102AE0000F5F1F4F86E0F80111928A95E9F78091F8
:102AF000CC1A811113C040E061E386EA0E942411E0
:102B00004AE06CE286EA0E94241181E08093CC1AAC
:102B10006CE77EE380E090E00E940A5C48E06DE2B2
:102B200086EA0E9424116CE77EE380E090E00E9438
:102B30000A5C26E0A80162E386EA0E943B1147E0B6
:102B40006DE286EA0E9424118A8190E0982F8827FE
:102B50002981822B9093C71A8093C61A2C8130E06A
:102B6000322F22274B81242B3093C91A2093C81A65
:102B70004E8150E0542F44276D81462B5093CB1A41
:102B80004093CA1A5F934F933F932F939F938F93D2
:102B900085EF93E09F938F930E940B8F0FB6F8946D
:102BA000DEBF0FBECDBF26960FB6F894DEBF0FBEB8
:102BB000CDBFDF91CF911F910F910895CF92DF92FA
:102BC000EF92FF920F931F93CF93DF93CDB7DEB7B2
:102BD0002A970FB6F894DEBF0FBECDBF8E010F5FF0
:102BE0001F4F86E0F80111928A95E9F741E062E013
:102BF0008CE30E94241148E560E08CE30E942411DC
:102C000062E174E380E090E00E940A5C26E0A801A3
:102C100063E08CE30E943B1143E062E08CE30E949E
:102C20002411098110E0102F00278A81082B1093AE
:102C3000A71A0093A61AEB80F12CFE2CEE248C81AF
:102C4000E82AF092A91AE092A81ACD80D12CDC2CA7
:102C5000CC248E81C82AD092AB1AC092AA1AB8018D
:102C6000882777FD8095982F0E947E859B01AC0177
:102C7000B701882777FD8095982F2F83388749875C
:102C80005A870E947E852F81388549855A850E9402
:102C9000888420EE3EE245E652E40E945C8720E014
:102CA00030E044E353E40E9415849F938F937F9315
:102CB0006F93DF92CF92FF92EF921F930F9383E077
:102CC00094E09F938F930E940B8F0FB6F894DEBF12
:102CD0000FBECDBF2A960FB6F894DEBF0FBECDBF94
:102CE000DF91CF911F910F91FF90EF90DF90CF90E8
:102CF0000895CF93DF93EC01888199810097F9F0D3
:102D00008632904121F01982188283E063C083E803
:102D100099E00E945C53892BE1F0809173099091B6
:102D2000740993FD18C0809173099091740994FD02
:102D300043C0809173099091740995FD44C060E887
:102D400070E083E899E00E94355386E290E1998330
:102D5000888381E03FC08091CB1F82FFE4CF21E0D8
:102D600048E061E083E00E94F7128091BD1B8F93E1
:102D70008091BC1B8F938091BB1B8F938091BA1B5A
:102D80008F938091B91B8F938091B81B8F93809103
:102D9000B71B8F938091B61B8F938BE49EE09F931C
:102DA0008F930E941D8F8DB79EB70A960FB6F89429
:102DB0009EBF0FBE8DBFB7CF8091CB1F83FFB9CF12
:102DC0000E946615B6CF8091CB1F84FFB8CF0E94BA
:102DD000DE15B5CFDF91CF910895CF93C82F8CEE3C
:102DE0000E947F5C8C2F0E94895C65E375E080E027
:102DF00090E00E940A5C8DEE0E947F5C0E949A5CCB
:102E0000C82F0E94A45C2C2F30E0322F2227A9016A
:102E1000482BCA01CF910895CF93DF93C82F8CEE32
:102E20000E947F5C8C2F0E94895C62E174E380E0E9
:102E300090E00E940A5C8CEE0E947F5C80E00E9421
:102E4000895C65E375E080E090E00E940A5C8DEEAD
:102E50000E947F5C0E949A5CC82F0E949A5CD82FC7
:102E60000E94A45C4D2F50E060E070E0762F652F4B
:102E7000542F44276C2B482BCB01BA01DF91CF9103
:102E800008952F923F924F925F926F927F928F920E
:102E90009F92AF92BF92CF92DF92EF92FF920F93E9
:102EA0001F93CF93DF93CDB7DEB7CD54D1090FB6C3
:102EB000F894DEBF0FBECDBF809100029091010259
:102EC000892BD1F110920102109200028CEE0E9427
:102ED0007F5C8EE10E94895C6BE17EE480E090E0A3
:102EE0000E940A5C82EA0E94ED169093800980930A
:102EF0007F0984EA0E94ED1690937E0980937D09F4
:102F000086EA0E94ED1690937C0980937B0988EAFB
:102F10000E94ED1690937A09809379098AEA0E94BB
:102F2000ED1690937809809377098CEA0E94ED164C
:102F3000909376098093750988E40E940C176FAB13
:102F400078AF89AF9AAF88E50E940C174B015C01FE
:102F5000809177099091780920E030E040E050E0DE
:102F6000BA0126962FAF269727963FAF2797289628
:102F70004FAF289729965FAF29972A966FAF2A9768
:102F80002B967FAF2B979C0140E050E060E070E013
:102F900080E090E008E00E942E8A0E94DA893901E0
:102FA000B42FA52FF62FE72F8C019401A50160E027
:102FB00070E080E090E05301CB2EDA2EEF2EFE2E53
:102FC0000E94658A29833A832A011B014C01B101C1
:102FD000C401315041095F4F6F4F7F4F8F4F9F4F5B
:102FE000A1E0B0E02596BFAFAEAF259721153F4FCA
:102FF0004F4F5140610571058105910509F020F49D
:1030000025961FAE1EAE259725966EAC7FAC2597F4
:1030100080917509909176095C01C12CD12CE12C2D
:10302000F12C00E010E029813A81A201B101C40134
:103030000E94FD88D22EE32EF42E052F162FB72FD7
:10304000F82FE92FA0E00E948C8A84F421503109E6
:1030500040485F4F6F4F7F4F8F4F9F4FD22EE32ED1
:10306000F42E052F162FB72FF82FE92F2D2D3E2DDB
:103070004F2D502F612F7B2F8F2F9E2F07E10E9406
:10308000478A2B8F3C8F4D8F5E8F6F8F78A389A3DC
:103090009AA32053384F4F4F5F4F6F4F7F4F8F4F43
:1030A0009F4F2B8B3C8B4D8B5E8B6F8B788F898FDB
:1030B0009A8F2056304F4F4F5F4F6F4F7F4F8F4F3C
:1030C0009F4F243D30434105510561057105810540
:1030D000910541F038F025966EAC7FAC2597FFEF57
:1030E0006F1A7F0A80917D0990917E099C0140E0D2
:1030F00050E060E070E080E090E000E10E942E8A05
:103100002B833C834D835E836A8779878F8398877F
:103110004091790950917A09A980BA8062017101C0
:1031200084019A0140E050E060E070E080E090E0CF
:103130000E94FD88D22EE32EF42E052F162FB72FD6
:10314000F82FE92FA0E00E948C8A5CF4AFE70E9480
:103150006E8AD22EE32EF42E052F162FB72FF82FBE
:10316000E92F2D2D3E2D4F2D502F612F7B2F8F2F8F
:103170009E2F07E00E94478A59016A017B018C015A
:103180002B813C814D815E816A8579858F8198850F
:103190000E94658A2B833C834D835E836F8378878F
:1031A0008F87988B2E5F3F4F434051096E4F7F4F63
:1031B0008F4F9F4F22303105494F5F4F644071055B
:1031C0008105910521F018F01FEF611A710A8091B5
:1031D0007F0990918009BC0180E090E020E030E818
:1031E00040E050E00E94568929873A874B875C87E8
:1031F0006A8B798B8D879E8740917B0950917C09E2
:10320000A980BA806201710184019A0140E050E016
:1032100060E070E080E090E00E94FD88D22EE32E16
:10322000F42E052F162FB72FF82FE92FA0E00E94BC
:103230008C8A84F421503F4F4F4F5F4F6F4F7F4F29
:103240008F4F9F4FD22EE32EF42E052F162FB72F20
:10325000F82FE92F2D2D3E2D4F2D502F612F7B2F35
:103260008F2F9E2F08E00E94478A59016A017B0137
:103270008C0129853A854B855C856A8979898D859C
:103280009E850E94658A29873A874B875C876D8770
:103290007E87898B9A8B2F5F3F4F4140510961098F
:1032A000710981099109213030484C4F5F476140D5
:1032B00071058105910521F018F0BFEF6B1A7B0AAB
:1032C0002B893C894D895E896F89788D898D9A8D8E
:1032D0002F3C374041055105610571058105910578
:1032E00011F00CF0A5C1A980BA80620171018401BE
:1032F0009501A201B101C4010E94FD88A12CB12C4D
:10330000C12C10E8D12EE12CF12C00E010E00E943D
:10331000C0882BAF3CAF4DAF5EAF6FAF21967FAF94
:10332000219722968FAF229723969FAF2397AB8C3E
:10333000BC8CCD8CDE8CEF8CF8A009A11AA1950174
:10334000A601B701C8010E94FD8859016A017B01ED
:10335000E82F192F02E00E942E8A0E2F0E94658A04
:1033600069017A01162F272EF82FE92F322E8D2C86
:10337000942EAF2CB62E072F582EB92FA0E00E9406
:103380008C8A5CF4A1E00E946E8A322E832E942EE9
:10339000A52EB62E072F582EB92F232D382D492DA7
:1033A0005A2D6B2D702F852D9B2F01E00E94478A8F
:1033B0002E962FAF2E972D963FAF2D9749A75AA740
:1033C0006BA77CA78DA79EA7522E432E4BA35CA371
:1033D0006DA37EA38FA398A7B22D9601A701612F9D
:1033E000722D8F2F9E2FA0E00E948C8A4CF4A3E0B8
:1033F0000E946E8A69017A01162FB72FF82FE92FE4
:103400009601A701612F7B2F8F2F9E2F02E00E9434
:10341000478A2FA738AB49AB5AAB6BAB7CAB8DABB4
:103420009EAB19014A01B62FA72F24968FAF249780
:10343000F92F2B893C894D895E896F89788D898D1B
:103440009A8D24323A4F4F4F5F4F6F4F7F4F8F4FC0
:103450009F4F0CF08CC02B8D3C8D4D8D5E8D6F8DF4
:1034600078A189A19AA12455324F4F4F5F4F6F4FDA
:103470007F4F8F4F9F4F59016A017B018C010E9442
:10348000FD8819014A01B62FA72FFC0103E00E9415
:103490002E8A51016401EB2EFA2E8F010E947A8A46
:1034A00059016A017B018C012E962FAD2E972D9626
:1034B0003FAD2D9749A55AA56BA57CA58DA59EA5C9
:1034C0000E94658A522E432E4BA35CA36DA37EA35C
:1034D0008FA398A79101A4016B2F7A2FCF0102E04F
:1034E0000E942E8A51016401EB2EFA2E8F010E9458
:1034F0007A8A02E00E942E8A0E2F0E947A8AF22E89
:10350000032F142FD52EE62EB72FF82FE92FA0E08A
:103510000E948C8A5CF4A1E00E946E8AF22E032F36
:10352000142FD52EE62EB72FF82FE92F2F2D302F61
:10353000412F5D2D6E2D7B2F8F2F9E2F01E00E943E
:10354000478A59016A017B018C012FA538A949A935
:103550005AA96BA97CA98DA99EA90E94658A190107
:103560004A01B62FA72F24968FAF2497F92F2B81CE
:103570003C814D815E816F8178858F859889A52CEE
:10358000B42CCBA0DCA0EDA0FEA00FA118A50E943A
:103590007A8A2B833C834D835E836F8378878F8702
:1035A000988B29853A854B855C856D857E858989D3
:1035B0009A8951016401EB2EFA2E24960FAD2497BF
:1035C0001F2F0E947A8A29873A874B875C876D87ED
:1035D0007E87898B9A8B2B893C894D895E896F897F
:1035E000788D898D9A8DABACBCACCDACDEACEFAC3C
:1035F0002196FFAC219722960FAD229723961FADFF
:1036000023970E947A8A2056304F4F4F5F4F6F4F5B
:103610007F4F8F4F9F4F243D30434105510561053A
:1036200071058105910521F018F02FEF621A720AD9
:103630006FA978AD89AD9AADAB01BC0180E090E097
:10364000DC0124964FAF249725965FAF25972696E9
:103650006FAF269727967FAF279728968FAF28972B
:1036600029969FAF29972A96AFAF2A972B96BFAF7F
:103670002B97A984BA84CB84DC84ED84FE840989E9
:103680001A899A01AB0160E070E080E090E00E944E
:10369000FD88F22E032F142FD52EE62EB72FF82FEC
:1036A000E92FA0E00E948C8A84F421503109404E19
:1036B0005F4F6F4F7F4F8F4F9F4FF22E032F142F6F
:1036C000D52EE62EB72FF82FE92F2F2D302F412F93
:1036D0005D2D6E2D7B2F8F2F9E2F05E10E94478A37
:1036E000AB80BC80CD80DE80EF80F8840F851889A8
:1036F0000E947A8AF22E032F142FD52EE62EB72F92
:10370000F82FE92FA0E00E948C8A84F421503048E1
:103710004F4F5F4F6F4F7F4F8F4F9F4FF22E032FB3
:10372000142FD52EE62EB72FF82FE92F2F2D302F5F
:10373000412F5D2D6E2D7B2F8F2F9E2F0FE00E942E
:10374000478A69017A018B018A83998329011A01C9
:103750004B015C01285E334041095109610971093F
:1037600081099109283D304D4140510561057105A0
:103770008105910521F018F0BFEF6B1A7B0A0E94BA
:10378000815C672859F09601A701B8018A81998167
:103790000E94DA8929011A014B015C019201A10101
:1037A000B401C5010E94788520E030E048EC52E485
:1037B0000E94DF84C35BDF4F0FB6F894DEBF0FBEFD
:1037C000CDBFDF91CF911F910F91FF90EF90DF90D0
:1037D000CF90BF90AF909F908F907F906F905F90B1
:1037E0004F903F902F9008954F925F926F927F92EB
:1037F0008F929F92AF92BF92CF92DF92EF92FF9201
:103800002B013C0169017A0123EC35EF4CE851E4CE
:10381000C701B6010E945C874B015C0128EB3EE1C9
:1038200043E753E4C701B6010E9415849B01AC0134
:10383000C501B4010E94DF840E944C854B015C01EC
:1038400020E030E048EC52E4C301B2010E94DF8482
:1038500021E835E943EC50E40E945C87A50194011E
:103860000E945C874B015C0123E333E948E853E4A1
:10387000C701B6010E9415849B01AC01C501B401CA
:103880000E94DF8423E333EB48E553E40E945C8726
:10389000FF90EF90DF90CF90BF90AF909F908F9070
:1038A0007F906F905F904F9008954F925F926F92CC
:1038B0007F928F929F92AF92BF92CF92DF92EF92C0
:1038C000FF9269017A010E94DE8620E030E040E04C
:1038D00050E40E94148422E93CE54EED5EE30E9430
:1038E000DF844B015C0123EC35EF4CE851E4C70168
:1038F000B6010E945C872B013C0128EB3EE143E7C7
:1039000053E4C701B6010E9415849B01AC01C301B9
:10391000B2010E94DF849B01AC01C501B4010E9489
:1039200015846B017C0128EB3EE143E753E40E94E0
:103930005C874B015C01A701960163EC75EF8CE895
:1039400091E40E9414849B01AC01C501B4010E9462
:10395000DF84FF90EF90DF90CF90BF90AF909F906B
:103960008F907F906F905F904F9008954F925F92ED
:103970006F927F928F929F92AF92BF92CF92DF927F
:10398000EF92FF922B013C0169017A0123EC35EFA4
:103990004CE851E4C701B6010E945C874B015C0111
:1039A00028EB3EE143E753E4C701B6010E941584CA
:1039B0009B01AC01C501B4010E94DF840E944C85CB
:1039C0004B015C0120E030E048EC52E4C301B2015D
:1039D0000E94DF84A50194010E945C8720E030E012
:1039E00040E251E40E94148424EE38E34EE05FE3A9
:1039F0000E945C879B01AC01C701B6010E9415843F
:103A0000FF90EF90DF90CF90BF90AF909F908F90FE
:103A10007F906F905F904F90089580E80E947F5C48
:103A200081110DC08EEF0E94895C811108C06BE18D
:103A30007EE480E090E00E940A5C0C94815C0E942D
:103A4000815C8091DD239091DE23A091DF23B091F2
:103A5000E0230196A11DB11D8093DD239093DE2309
:103A6000A093DF23B093E0230895FC01DC0182E002
:103A700020E041E39D91292798E0322F330F27FF63
:103A800003C0232F242701C0232F9150B1F7815069
:103A900089F781E090E03281231711F080E090E017
:103AA0000895CF92DF92EF92FF920F931F93CF93DF
:103AB000DF930E940D1D80E80E947F5C811172C01F
:103AC0008AEF0E94895C81116DC08FE00E94895C41
:103AD000811168C065E375E080E090E00E940A5CB7
:103AE00081E80E947F5C81115DC00E949A5CC82FB2
:103AF0000E949A5C0E949A5CD82F0E949A5C0E9455
:103B00009A5C182F0E949A5C0E94A45C082F0E9465
:103B1000A45C80E80E947F5C811144C08CEF0E940D
:103B2000895C81113FC089EC0E94895C81113AC097
:103B300065E375E080E090E00E940A5C81E80E9405
:103B40007F5C0E949A5CD82E0E949A5CC82E0E94CC
:103B50009A5C0E949A5CF82E0E949A5CE82E0E9461
:103B6000A45C1F92CF921F92DF921F920F931F921D
:103B70001F931F92DF931F92CF931F92EF921F927A
:103B8000FF9288E194E09F938F930E940B8F0E9495
:103B9000815C8DB79EB742960FB6F8949EBF0FBE5C
:103BA0008DBF17C00E94815C8091DD239091DE2340
:103BB000A091DF23B091E0230196A11DB11D809358
:103BC000DD239093DE23A093DF23B093E0230E94B4
:103BD0000D1D20E030E040E050E060E070E080E06B
:103BE00090E0DF91CF911F910F91FF90EF90DF90C8
:103BF000CF900895EF92FF920F931F93CF93DF938F
:103C000000D01F92CDB7DEB78C0180E80E947F5CA8
:103C1000811154C00115110551F085EE0E94895C97
:103C200081114CC061E077E980E090E009C083EE4B
:103C30000E94895C811142C069E97AEB81E090E0E1
:103C40000E940A5C81E80E947F5C811137C00E945B
:103C50009A5CF82E89830E949A5CE82E8A830E94DF
:103C6000A45C8B830E94815CCE0101960E94351D6D
:103C7000892B21F16E2D70E07F296C7F80E090E030
:103C8000012B69F00E947C8520E030E04AEF5AE386
:103C90000E945C8720E030E040EC50E40CC00E94C1
:103CA0007C8522E538EB4FE25BE30E945C8726E6E9
:103CB00036E64BE352E40E9414841BC00E94815CF0
:103CC0008091DD239091DE23A091DF23B091E0234A
:103CD0000196A11DB11D8093DD239093DE23A09357
:103CE000DF23B093E0230E940D1D60EF7FEF89E793
:103CF00094E40F900F900F90DF91CF911F910F914F
:103D0000FF90EF9008950F931F93CF93DF93729AD4
:103D10008091540283FF08C08EE40E941D5C8111D3
:103D200063C0C0E5D0E008C0C0E5D0E00E946E09E5
:103D300021972097D9F7F0CF0E946E0921972097FD
:103D4000D9F78FE40E941D5C0E949A5C082F0F73C4
:103D50000E949A5C182F0E949A5CD82F0E94A45C43
:103D6000C82F0E94815C8091540283FF7298602F5B
:103D700070E0762F6627610F711D80E090E00E9451
:103D80007C8520E134E048EC5BE30E945C87609333
:103D9000BF1B7093C01B8093C11B9093C21B6D2FE0
:103DA00070E0762F66276C0F711D76956795769576
:103DB000679580E090E00E947C8524EA3CEF44E235
:103DC0005CE30E945C8720E030E040E252E40E9425
:103DD000148460935C2870935D2880935E28909390
:103DE0005F2880E090E002C081E090E0DF91CF9119
:103DF0001F910F9108957298729A8EE40E941D5C33
:103E000080EA0E94895C80E00E94895C80E00E94D8
:103E1000895C8FE40E941D5C0E949A5C8EE40E9483
:103E20001D5C80E80E94895C80E00E94895C80E0E3
:103E30000E94895C0E94815C80E090E008958FED93
:103E40009DE09F938F930E941D8F80916D020F9034
:103E50000F90882361F01F928F938CED9DE09F93CC
:103E60008F930E941D8F0F900F900F900F900895C9
:103E700087EB9DE09F938F930E941D8F8FE89DE0BD
:103E80009F938F930E941D8F88E69DE09F938F9351
:103E90000E941D8F8DE29DE09F938F930E941D8F46
:103EA0008BEF9CE09F938F930E941D8F8FEB9CE084
:103EB0009F938F930E941D8F89E99CE09F938F931E
:103EC0000E941D8F83E69CE09F938F930E941D8F1D
:103ED0008091CB1F9091CC1F827091702DB73EB70F
:103EE000205F3F4F0FB6F8943EBF0FBE2DBF892B0A
:103EF00041F083E39CE09F938F930E941D8F0F906E
:103F00000F9087E09CE09F938F930E941D8F8EED12
:103F10009BE09F938F930E941D8F82EB9BE09F936A
:103F20008F930E941D8F83E89BE09F938F930E9445
:103F30001D8F81E59BE09F938F930E941D8F80E2F0
:103F40009BE09F938F930E941D8F86EE9AE09F9334
:103F50008F930E941D8F80EB9AE09F938F930E9416
:103F60001D8F80E89AE09F938F930E941D8F84E5B8
:103F70009AE09F938F930E941D8F85E29AE09F9312
:103F80008F930E941D8F8CEE99E09F938F930E94D8
:103F90001D8F83EB99E09F938F930E941D8F8CE779
:103FA00099E09F938F930E941D8F8BE499E09F93DC
:103FB0008F930E941D8F8CE199E09F938F930E94B5
:103FC0001D8F8DB79EB780960FB6F8949EBF0FBE1B
:103FD0008DBF8DEE98E09F938F930E941D8F86EC8E
:103FE00098E09F938F930E941D8F80E998E09F93A4
:103FF0008F930E941D8F8AE598E09F938F930E9474
:104000001D8F84E298E09F938F930E941D8F8BEF0A
:1040100097E09F938F930E941D8F83EC97E09F936F
:104020008F930E941D8F88E997E09F938F930E9442
:104030001D8F2DB73EB7205F3F4F0FB6F8943EBFA0
:104040000FBE2DBF089587E494E00C94418F4F92EA
:104050005F926F927F928F929F92AF92BF92CF9218
:10406000DF92EF92FF92CF93DF93CDB7DEB7289721
:104070000FB6F894DEBF0FBECDBF8091D1239091D3
:10408000D223A091D323B091D42389839A83AB8385
:10409000BC834090D1235090D2236090D323709062
:1040A000D4238091D1239091D223A091D323B09196
:1040B000D4238D839E83AF83B8876091D123709181
:1040C000D2238091D3239091D4232CE3822E912C60
:1040D000A12CB12CA50194010E9485887F936F9338
:1040E00030E1C32E3EE0D32EE12CF12C6D817E8198
:1040F0008F819885A70196010E948588A50194016A
:104100000E9485883F932F9340E8842E41E5942EAA
:10411000AA24A394B12CC301B201A50194010E9469
:104120008588A70196010E9485883F932F93698116
:104130007A818B819C81A50194010E9485883F939F
:104140002F9382E797E09F938F930E941D8F0FB666
:10415000F894DEBF0FBECDBF28960FB6F894DEBF31
:104160000FBECDBFDF91CF91FF90EF90DF90CF904A
:10417000BF90AF909F908F907F906F905F904F9087
:104180000895E1E2F1E3808191818234924479F0F3
:10419000E152F143FF93EF9384E597E09F938F9370
:1041A0000E941D8F0F900F900F900F9008953A96D8
:1041B000E53F81E4F80738F30895CF93DF93EC01EE
:1041C0008C9A0E94510A9F938F937F936F9388E4F8
:1041D00097E09F938F930E941D8F0F900F900F90E9
:1041E0000F900F900F90209719F00E94610B08C05C
:1041F00086E497E09F938F930E941D8F0F900F90FE
:1042000081E00E94020A2091720230917302409173
:104210007402509175020E945C879F938F937F93E5
:104220006F938AE397E09F938F930E941D8F0F9067
:104230000F900F900F900F900F90209719F00E9401
:10424000610B08C088E397E09F938F930E941D8FB6
:104250000F900F9082E00E94020A20916E0230912E
:104260006F0240917002509171020E945C879F938F
:104270008F937F936F938CE297E09F938F930E942D
:104280001D8F0F900F900F900F900F900F90209711
:1042900019F00E94610B08C08AE297E09F938F9308
:1042A0000E941D8F0F900F9083E00E94020A9F933F
:1042B0008F937F936F938BE197E09F938F930E94EF
:1042C0001D8F8C980F900F900F900F900F900F9064
:1042D000209719F00E94610B08C089E197E09F9335
:1042E0008F930E941D8F0F900F908091CB1F87FF9F
:1042F00083C021E042E161E080ED0E94E15D9F9397
:104300008F937F936F938CE097E09F938F930E949E
:104310001D8F0F900F900F900F900F900F90209780
:1043200019F00E94610B08C08AE097E09F938F9379
:104330000E941D8F0F900F9021E042E162E080ED1E
:104340000E94E15D9F938F937F936F938DEF96E033
:104350009F938F930E941D8F0F900F900F900F903F
:104360000F900F90209719F00E94610B08C08BEFFF
:1043700096E09F938F930E941D8F0F900F9021E0E6
:1043800042E163E080ED0E94E15D9F938F937F9314
:104390006F938EEE96E09F938F930E941D8F0F90E8
:1043A0000F900F900F900F900F90CD2B19F00E944F
:1043B000610B08C08CEE96E09F938F930E941D8F37
:1043C0000F900F9021E042E164E080ED0E94E15DFA
:1043D0009F938F937F936F938FED96E09F938F932F
:1043E0000E941D8F0F900F900F900F900F900F90C5
:1043F000DF91CF910C94610BCD2BD1F3DF91CF9155
:1044000008950F931F93CF93DF93882389F049E09A
:1044100050E06FEF70E080E598E20E945F8E49E027
:1044200050E06AE070E080E598E20E948F9013C04F
:10443000C0E5D8E20AED16E089911F928F931F9391
:104440000F930E941D8F0F900F900F900F9088E296
:10445000C835D80789F7DF91CF911F910F910C9440
:10446000610BCF92DF92EF92FF92CF93DF936B01BC
:104470007C0160FF11C084E894E09F938F9384EFE8
:104480009DE09F938F930E941D8F0F900F900F9030
:104490000F9081E090E002C080E090E0C1FE09C092
:1044A000EC01219642ED58E069E874E00E94B00FFB
:1044B000CE01C2FE09C0EC01219642ED58E061E94F
:1044C00074E00E94B00FCE01C3FE09C0EC0121963A
:1044D00042ED58E069E974E00E94B00FCE01C4FEDD
:1044E00009C0EC01219642ED58E06DE974E00E94AC
:1044F000B00FCE01C5FE09C0EC01219642ED58E097
:1045000060EA74E00E94B00FCE01C6FE09C0EC0163
:10451000219642ED58E064EA74E00E94B00FCE01AB
:10452000C7FE09C0EC01219642ED58E06AEA74E04A
:104530000E94B00FCE01D0FE09C0EC01219642EDE1
:1045400058E062EB74E00E94B00FCE01D1FE09C0CA
:10455000EC01219642ED58E06AEB74E00E94B00F46
:10456000CE01D2FE09C0EC01219642ED58E06EEB7F
:1045700074E00E94B00FCE012091CB1F3091CC1F70
:1045800024703270232B59F0D3FE09C0EC01219620
:1045900042ED58E064EC74E00E94B00FCE0120912F
:1045A000CB1F23FF0BC0D4FE09C0EC01219642EDC6
:1045B00058E069EC74E00E94B00FCE012091CB1F4F
:1045C00024FF0BC0D5FE09C0EC01219642ED58E056
:1045D0006FEC74E00E94B00FCE01D6FE09C0EC0172
:1045E000219642ED58E067ED74E00E94B00FCE01D5
:1045F000B701A60144275078452B462B472B61F085
:1046000042ED58E062EE74E0DF91CF91FF90EF90C1
:10461000DF90CF900C94B00FCD28CE28CF2841F456
:1046200085ED96E09F938F930E941D8F0F900F90C2
:10463000DF91CF91FF90EF90DF90CF9008950F938F
:104640001F93CF93DF938C01C0E0D0E001151105DB
:1046500009F48AC060ED76E0C8010E943E8E892B85
:1046600009F4C16068EC76E0C8010E943E8E892B97
:1046700009F4C26060EC76E0C8010E943E8E892B8E
:1046800009F4C4606CEB76E0C8010E943E8E892B71
:1046900009F4C86069EB76E0C8010E943E8E892B60
:1046A00009F4C06165EB76E0C8010E943E8E892B5B
:1046B00009F4C0626FEA76E0C8010E943E8E892B41
:1046C00009F4C06467EA76E0C8010E943E8E892B37
:1046D00009F4C0686FE976E0C8010E943E8E892B1C
:1046E00009F4D1606BE976E0C8010E943E8E892B07
:1046F00009F4D26065E976E0C8010E943E8E892BFC
:1047000009F4D46060E976E0C8010E943E8E892BEE
:1047100009F4D8606AE876E0C8010E943E8E892BD1
:1047200009F4D06162E876E0C8010E943E8E892BD0
:1047300009F4D06267E776E0C8010E943E8E892BBB
:1047400009F4D06466E676E0C8010E943E8E892BAB
:1047500009F4D06860916B0270916C0280E090E087
:104760000E94528E8C0172CFCE01DF91CF911F91AA
:104770000F910895AF92BF92CF92DF92EF92FF9286
:104780000F931F93CF93DF93F22E032F142FE52E59
:104790005B016C01217030E040E050E060E070E0CF
:1047A00080E090E0A0E00E948C8A89F0E3EFF4E0E2
:1047B000FF93EF93E4EFFDE0FF93EF930E941D8FD3
:1047C0000F900F900F900F90E1E0F0E002C0E0E05A
:1047D000F0E08091CB1F80FF17C02F2D247030E0B8
:1047E00040E050E060E070E080E090E0A0E00E94F7
:1047F0008C8A51F0EF01219642ED58E067EF74E0AA
:10480000CF010E94B00FFE012F2D227030E040E05A
:1048100050E060E070E080E090E0A0E00E948C8AD0
:1048200051F0EF01219642ED58E06BEF74E0CF01BB
:104830000E94B00FFE012F2D287030E040E050E0C4
:1048400060E070E080E090E0A0E00E948C8A51F08F
:10485000EF01219642ED58E063E175E0CF010E943F
:10486000B00FFE012F2D207130E040E050E060E0FD
:1048700070E080E090E0A0E00E948C8A51F0EF01AF
:10488000219642ED58E06EEF74E0CF010E94B00F28
:10489000FE012F2D207230E040E050E060E070E03B
:1048A00080E090E0A0E00E948C8A51F0EF01219618
:1048B00042ED58E061E075E0CF010E94B00FFE01CB
:1048C0002F2D207430E040E050E060E070E080E0A8
:1048D00090E0A0E00E948C8A51F0EF01219642ED19
:1048E00058E067E075E0CF010E94B00FFE012F2D68
:1048F000207830E040E050E060E070E080E090E060
:10490000A0E00E948C8A51F0EF01219642ED58E020
:104910006DE075E0CF010E94B00FFE0120E0302F66
:10492000317040E050E060E070E080E090E0A0E0B6
:104930000E948C8A51F0EF01219642ED58E060E12F
:1049400075E0CF010E94B00FFE0120E0302F3270E1
:1049500040E050E060E070E080E090E0A0E00E9485
:104960008C8A51F0EF01219642ED58E065E175E047
:10497000CF010E94B00FFE0120E0302F347040E0E4
:1049800050E060E070E080E090E0A0E00E948C8A5F
:1049900051F0EF01219642ED58E06CE175E0CF0156
:1049A0000E94B00FFE0120E0302F387040E050E050
:1049B00060E070E080E090E0A0E00E948C8A51F01E
:1049C000EF01219642ED58E06FE175E0CF010E94C2
:1049D000B00FFE0120E0302F307140E050E060E089
:1049E00070E080E090E0A0E00E948C8A51F0EF013E
:1049F000219642ED58E064E275E0CF010E94B00FCD
:104A0000FE0120E0302F307240E050E060E070E0C6
:104A100080E090E0A0E00E948C8A51F0EF012196A6
:104A200042ED58E06BE275E0CF010E94B00FFE014D
:104A30008091CB1F81FF17C020E0302F307440E001
:104A400050E060E070E080E090E0A0E00E948C8A9E
:104A500051F0EF01219642ED58E062E375E0CF019D
:104A60000E94B00FFE018091CB1F9091CC1F90FF50
:104A700017C020E030E040E05E2D507160E070E053
:104A800080E090E0A0E00E948C8A51F0EF01219636
:104A900042ED58E065E375E0CF010E94B00FFE01E2
:104AA0008091CB1F9091CC1F90FF17C020E030E089
:104AB00040E05E2D507260E070E080E090E0A0E0A9
:104AC0000E948C8A51F0EF01219642ED58E068E394
:104AD00075E0CF010E94B00FFE018091CB1F909135
:104AE000CC1F90FF17C020E030E040E05E2D5074F6
:104AF00060E070E080E090E0A0E00E948C8A51F0DD
:104B0000EF01219642ED58E06EE375E0CF010E947F
:104B1000B00FFE0120E0302F307840E050E060E040
:104B200070E080E090E0A0E00E948C8A51F0EF01FC
:104B3000219642ED58E069E475E0CF010E94B00F84
:104B4000FE0120E030E0412F417050E060E070E075
:104B500080E090E0A0E00E948C8A51F0EF01219665
:104B600042ED58E06EE475E0CF010E94B00FFE0107
:104B700020E030E0412F427050E060E070E080E0E3
:104B800090E0A0E00E948C8A51F0EF01219642ED66
:104B900058E061E575E0CF010E94B00FFE0120E012
:104BA00030E0412F447050E060E070E080E090E041
:104BB000A0E00E948C8A51F0EF01219642ED58E06E
:104BC00064E575E0CF010E94B00FFE018091CB1F1C
:104BD00087FF17C020E030E0412F487050E060E0D0
:104BE00070E080E090E0A0E00E948C8A51F0EF013C
:104BF000219642ED58E067E575E0CF010E94B00FC5
:104C0000FE018091CB1F87FF17C020E030E0412FCD
:104C1000407150E060E070E080E090E0A0E00E9431
:104C20008C8A51F0EF01219642ED58E06BE575E07A
:104C3000CF010E94B00FFE018091CB1F87FF17C0EC
:104C400020E030E0412F407250E060E070E080E012
:104C500090E0A0E00E948C8A51F0EF01219642ED95
:104C600058E06FE575E0CF010E94B00FFE01809122
:104C7000CB1F87FF17C020E030E0412F407450E089
:104C800060E070E080E090E0A0E00E948C8A51F04B
:104C9000EF01219642ED58E063E675E0CF010E94F6
:104CA000B00FFE018091CB1F82FF17C020E030E0E3
:104CB000412F407850E060E070E080E090E0A0E0BC
:104CC0000E948C8A51F0EF01219642ED58E062E299
:104CD00076E0CF010E94B00FFE018091CB1F82FFD2
:104CE00017C020E030E040E05E2D517060E070E0E1
:104CF00080E090E0A0E00E948C8A51F0EF012196C4
:104D000042ED58E067E675E0CF010E94B00FFE016A
:104D10008091CB1F9091CC1F90FF17C020E030E016
:104D200040E05E2D527060E070E080E090E0A0E036
:104D30000E948C8A51F0EF01219642ED58E06AE61C
:104D400075E0CF010E94B00FFE018091CB1F9091C2
:104D5000CC1F90FF17C020E030E040E05E2D547083
:104D600060E070E080E090E0A0E00E948C8A51F06A
:104D7000EF01219642ED58E062E775E0CF010E9415
:104D8000B00FFE018091CB1F9091CC1F91FF1EC0F0
:104D900020E030E040E05E2D587060E070E080E0A0
:104DA00090E0A0E00E948C8A89F042ED58E06BE729
:104DB00075E0CF01DF91CF911F910F91FF90EF90A0
:104DC000DF90CF90BF90AF900C94B00F2F2D302F6D
:104DD000412F5E2DB501C601A0E00E948C8A41F4EE
:104DE00081E696E09F938F930E941D8F0F900F9006
:104DF000DF91CF911F910F91FF90EF90DF90CF90B7
:104E0000BF90AF900895AF92BF92DF92EF920F9351
:104E10001F93CF93DF93EC015B01FB0110826CE5E4
:104E200076E00E943E8E892B59F58091CB1F7DE460
:104E3000D72EE0E8EE2E82FD02C004E001C004E8B7
:104E400010E081FF02C060ECE62E26E04AE250E06E
:104E50006BE270E089E290E00E94315981E090E0DD
:104E60000E94EF0A882311F05DE5D52E8091CB1FBB
:104E70009091CC1F90FD16E091FF06C0186004C011
:104E8000D12CE12C00E010E06AE576E0CE010E9432
:104E90003E8E892B61F481E0F501808360916B0285
:104EA00070916C0280E090E00E94528EEC0168E507
:104EB00076E0CE010E943E8E892B61F48FEFF501E2
:104EC000808360916B0270916C0280E090E00E94A0
:104ED000528EEC01209709F41AC164E576E0CE0108
:104EE0000E943E8E892B19F4FD2DF160DF2E60E5C6
:104EF00076E0CE010E943E8E892B19F48D2D8460C0
:104F0000D82E6DE476E0CE010E943E8E892B19F4F6
:104F1000ED2DE260DE2E6BE476E0CE010E943E8E47
:104F2000892B19F4FD2DF860DF2E68E476E0CE01C0
:104F30000E943E8E892B19F48D2D8061D82E62E45B
:104F400076E0CE010E943E8E892B19F4ED2DE062B1
:104F5000DE2E6CE376E0CE010E943E8E892B19F4A2
:104F6000FD2DF064DF2E69E376E0CE010E943E8ED7
:104F7000892B19F48D2D8068D82E64E376E0CE015C
:104F80000E943E8E892B19F4EE2DE160EE2E6DE22B
:104F900076E0CE010E943E8E892B19F4FE2DF26040
:104FA000EF2E6AE276E0CE010E943E8E892B19F444
:104FB0008E2D8460E82E65E276E0CE010E943E8E62
:104FC000892B19F4EE2DE860EE2E6EE176E0CE012D
:104FD0000E943E8E892B19F4FE2DF061EF2E67E1C1
:104FE00076E0CE010E943E8E892B19F48E2D8062D0
:104FF000E82E64E176E0CE010E943E8E892B19F402
:10500000EE2DE064EE2E6FE076E0CE010E943E8E43
:10501000892B19F4FE2DF068EF2E6CE076E0CE01BE
:105020000E943E8E892B09F4016069E076E0CE0192
:105030000E943E8E892B09F4026066E076E0CE0184
:105040000E943E8E892B09F4046062E076E0CE0176
:105050000E943E8E892B09F408606EEF75E0CE0148
:105060000E943E8E892B09F400616AEF75E0CE0143
:105070000E943E8E892B09F4006266EF75E0CE0136
:105080000E943E8E892B09F4006464EF75E0CE0126
:105090000E943E8E892B09F4006861EF75E0CE0115
:1050A0000E943E8E892B09F4116069EE75E0CE01F5
:1050B0000E943E8E892B09F4126060EE75E0CE01ED
:1050C0000E943E8E892B09F4146067ED75E0CE01D5
:1050D0000E943E8E892B09F4186064ED75E0CE01C4
:1050E0000E943E8E892B09F410616EEC75E0CE01B2
:1050F0000E943E8E892B09F4106263EC75E0CE01AC
:105100000E943E8E892B09F0DCCE1064DACE2D2D64
:105110003E2DA80160E070E080E090E0DF91CF914B
:105120001F910F91EF90DF90BF90AF9008955F9225
:105130006F927F928F929F92AF92BF92CF92DF92A7
:10514000EF92FF920F931F93CF93DF93782EC5EDCD
:10515000DAE100E010E0FDEBEF2EF5E0FF2E8170CC
:10516000582E872D8270682EA8EACA2EA5E0DA2E66
:10517000B0EBAB2EB5E0BB2E8EEA882E85E0982EE4
:10518000772051F01F930F93FF92EF920E941D8F93
:105190000F900F900F900F905520A1F089858F935D
:1051A00088858F93BF92AF920E941D8F0F900F90B2
:1051B0000F900F906620C1F09F928F920E941D8FDA
:1051C0000F900F90662081F0DF92CF920E941D8F8A
:1051D000288139814A815B816C817D818E819F81AB
:1051E0000E94BA230F900F900E94610B0F5F1F4F18
:1051F0002A960430110521F6DF91CF911F910F916E
:10520000FF90EF90DF90CF90BF90AF909F908F90E6
:105210007F906F905F90089588E995E09F938F93BA
:105220000E941D8F0E9423208CEB9AE19F938F9305
:1052300080E995E09F938F930E941D8F8CE895E005
:105240009F938F930E941D8F80E00E94012287E828
:1052500095E09F938F930E941D8F0E94D80F80919D
:10526000CB1F2DB73EB7265F3F4F0FB6F8943EBF1A
:105270000FBE2DBF80FF05C041E061E081E00E94CC
:1052800082110E942720809153021F928F938EE7F4
:1052900095E09F938F930E941D8F80916F091F92BD
:1052A0008F9385E795E09F938F930E941D8F809148
:1052B0007D028F9380917C028F9380917B028F93EC
:1052C00080917A028F9387E695E09F938F930E9457
:1052D0001D8F1F9280E48F938FE495E09F938F93AF
:1052E0000E941D8F809161281F928F93809160286A
:1052F0001F928F938CE395E09F938F930E941D8F55
:10530000809152021F928F9383E395E09F938F9336
:105310000E941D8F80915402909155022DB73EB787
:10532000245E3F4F0FB6F8943EBF0FBE2DBF96FFD1
:1053300003C084E895E002C087E895E09F938F93CF
:1053400089E295E09F938F930E941D8F83E00E94D6
:1053500097280F900F900F900F901D9B03C084E82B
:1053600095E002C087E895E09F938F938DE195E0EB
:105370009F938F930E941D8F83E195E09F938F935E
:105380000E941D8F809154020F900F900F900F90EC
:105390000F900F9081FF09C08DE095E09F938F9350
:1053A0000E941D8F0F900F9013C080FF03C084E8F0
:1053B00095E002C087E895E09F938F9389E095E0A0
:1053C0009F938F930E941D8F0F900F900F900F90BF
:1053D000809154029091550297FF03C084E895E0B4
:1053E00002C087E895E09F938F9380E095E09F93BC
:1053F0008F930E941D8F89EF94E09F938F930E945B
:105400001D8F609173097091740980E090E00E9493
:1054100031220E94610B0F900F900F900F900F9010
:105420000F90779903C084E895E002C087E895E083
:105430009F938F9380EF94E09F938F930E941D8F93
:105440000E9408090E94AB0A9F938F937F936F93EA
:1054500082EE94E09F938F930E941D8F0E94650AB5
:105460009F938F937F936F9384ED94E09F938F939B
:105470000E941D8F81E090E00E94DD2080913628FF
:1054800090913728A0913828B0913928BF93AF93D5
:105490009F938F9386EC94E09F938F930E941D8F30
:1054A00080914B288F9380914A288F93809149282F
:1054B0008F93809148288F9382EB94E09F938F93F2
:1054C0000E941D8F80913A2890913B28A0913C2802
:1054D000B0913D28BF93AF939F938F9384EA94E05C
:1054E0009F938F930E941D8F8DB79EB782960FB6A4
:1054F000F8949EBF0FBE8DBF80914F288F938091EF
:105500004E288F9380914D288F9380914C288F93B4
:1055100080E994E09F938F930E941D8F61E070E07B
:1055200080E090E00E946A0B0F900F900F900F9018
:105530000F900F9061E070E081E090E00C946A0BB6
:10554000F894E0E0F0E081E2809357008491E2E09B
:10555000F0E041E2409357004491E4E0F0E091E252
:1055600090935700E49190E0A0E0B0E0DC0199272F
:10557000882750E060E070E0762F652F542F442795
:10558000840F951FA61FB71F8E0F911DA11DB11D62
:105590008093761B9093771BA093781BB093791B15
:1055A00078940895CF93DF93CDB7DEB761970FB6A8
:1055B000F894DEBF0FBECDBF48E250E068E170E076
:1055C00085ED9AE10E9471902091D51A3091D61AFA
:1055D0004091D71A5091D81A6091D91A7091DA1A5D
:1055E0008091DB1A9091DC1AAFEF0E948C8A09F04F
:1055F0005DC08DE48093D51A80E88093D61A84E04C
:105600008093D71A1092D81A1092D91A1092DA1AD7
:105610001092DB1A1092DC1A8CE390E09093DE1A61
:105620008093DD1A1092DF1A1092E01A1092E11A9C
:105630001092E21A1092E31A1092E41A1092E51AEC
:105640001092E61A1092E81A1092E71A1092E91ACC
:105650001092EA1A1092EB1A1092EC1A1092ED1AAC
:105660001092EE1A1092EF1A1092F01A1092F21A8B
:105670001092F11A1092F31A1092F41A1092F51A6D
:105680001092F61A1092F71A1092F81A1092F91A4C
:105690001092FA1A1092FC1A1092FB1A48E250E08B
:1056A00068E170E085ED9AE10E948F9042E050E061
:1056B00066E170E0CE010F960E9471908F85988907
:1056C0008F3F2FEF920779F48AE090E49093550290
:1056D0008093540242E050E066E170E084E592E09D
:1056E0000E948F9004C0909355028093540242E030
:1056F00050E060E570E0CE010F960E9471908F85BA
:1057000098898F3F2FEF920769F4109274091092D5
:10571000730942E050E060E570E083E799E00E94A1
:105720008F9004C0909374098093730949E050E00E
:105730006AE070E080E598E20E9471900E94A20CFD
:1057400044E050E064E470E0CE010B960E9471905A
:105750008B859C85AD85BE8544E050E064E470E0B7
:105760008F3F9F4FAF4FBF4F29F482E792E00E94D7
:105770008F9004C082E792E00E94719044E050E074
:1057800060E470E0CE010B960E9471908B859C8541
:10579000AD85BE8544E050E060E470E08F3F9F4FF0
:1057A000AF4FBF4F29F48EE692E00E948F9004C065
:1057B0008EE692E00E94719044E050E068E470E070
:1057C000CE010B960E9471908B859C85AD85BE8520
:1057D00044E050E068E470E08F3F9F4FAF4FBF4F11
:1057E00029F486E792E00E948F9004C086E792E059
:1057F0000E94719041E050E065E170E0CE01419679
:105800000E947190898941E050E065E170E08F3F2E
:1058100029F48FE699E00E948F9004C08FE699E00A
:105820000E94719041E050E064E170E0CE01419649
:105830000E947190898941E050E064E170E08F3FFF
:1058400029F483E592E00E948F9004C083E592E002
:105850000E94719041E050E063E170E0CE0141961A
:105860000E947190898941E050E063E170E08F3FD0
:1058700029F482E592E00E948F9004C082E592E0D4
:105880000E9471904AE050E060E070E0CE01019625
:105890000E94719089814AE050E060E070E08F3FA3
:1058A00029F48CEB9AE10E948F9004C08CEB9AE172
:1058B0000E94719044E050E06CE470E0CE010B96E1
:1058C0000E9471908B859C85AD85BE8544E050E03B
:1058D0006CE470E08F3F9F4FAF4FBF4F29F48AE7D2
:1058E00092E00E948F9004C08AE792E00E9471903B
:1058F00061960FB6F894DEBF0FBECDBFDF91CF919A
:105900000895CF92DF92EF92FF9260916B027091B7
:105910006C0280E090E00E94528E6BE875E00E947D
:10592000668E892B09F005C18DE48093D51A80E835
:105930008093D61A84E08093D71A1092D81A1092C6
:10594000D91A1092DA1A1092DB1A1092DC1A8CE330
:1059500090E09093DE1A8093DD1A1092DF1A109275
:10596000E01A1092E11A1092E21A1092E31A1092C1
:10597000E41A1092E51A1092E61A1092E81A1092A0
:10598000E71A1092E91A1092EA1A1092EB1A109282
:10599000EC1A1092ED1A1092EE1A1092EF1A109261
:1059A000F01A1092F21A1092F11A1092F31A109241
:1059B000F41A1092F51A1092F61A1092F71A109221
:1059C000F81A1092F91A1092FA1A1092FC1A109200
:1059D000FB1A48E250E068E170E085ED9AE10E9430
:1059E0008F908AE090E4909355028093540242E0B5
:1059F00050E066E170E084E592E00E948F901092A2
:105A000074091092730942E050E060E570E083E7AA
:105A100099E00E948F9042E2C42EDD24DA944CEC8F
:105A2000E42E4BE3F42EC0927202D0927302E09205
:105A30007402F092750244E050E064E470E082E7A2
:105A400092E00E948F90C0926E02D0926F02E0921C
:105A50007002F092710244E050E060E470E08EE683
:105A600092E00E948F9087ED94E3AFEEBCE38093C9
:105A7000760290937702A0937802B093790244E083
:105A800050E068E470E086E792E00E948F908AE937
:105A900099E9A9E1B0E480937A0290937B02A09304
:105AA0007C02B0937D0244E050E06CE470E08AE751
:105AB00092E00E948F9010926F0980E00E949D6694
:105AC00041E050E065E170E08FE699E00E948F9040
:105AD0008AE1809353020E94446541E050E064E112
:105AE00070E083E592E00E948F908FE080935202F5
:105AF00041E050E063E170E082E592E00E948F9027
:105B00008AE0ECEBFAE1DF011D928A95E9F74AE0C1
:105B100050E060E070E0CF010E948F9081E00E9431
:105B2000012280E090E0FF90EF90DF90CF900C9406
:105B3000B60CFF90EF90DF90CF9008952F923F9298
:105B40004F925F926F927F928F929F92AF92BF928D
:105B5000CF92DF92EF92FF920F931F93CF93DF9339
:105B6000CDB7DEB72B970FB6F894DEBF0FBECDBF13
:105B70009B878A874A01FC0180819181892B11F0E2
:105B80000C94C33E60916B0270916C02CA010E943A
:105B9000528E60E470E0C4010E94858E009759F433
:105BA00060911B3170911C318AE090E00E94D98E87
:105BB00081E00C94C83E8130910561F4F401B0801D
:105BC0001B2D110F110B012F412E512E612E712E05
:105BD000A12EBCC082309105B9F4F40180819927CF
:105BE00087FD9095982F88272181820F911D27FD91
:105BF0009A95B82E192F092F000F000B402E502E0A
:105C0000602E702EA02EA2C083309105B1F5F40154
:105C10002081922F990F990B392F492F592F692FD6
:105C2000792F892F00E10E942E8A19012A013B0158
:105C3000B82FA92F2181922F990F990B392F492F16
:105C4000592F692F792F892F08E00E942E8A590138
:105C50006A017B018C019101A201B3018B2F9A2F64
:105C60000E94658AA2801A2D110F110BB12EC12E30
:105C7000D12EE12EF12E012F55C004970CF45DC0FA
:105C8000F4012081922F990F990B392F492F592F09
:105C9000692F792F892F08E10E942E8A19012A0184
:105CA0003B01B82FA92F2181922F990F990B392FE2
:105CB000492F592F692F792F892F00E10E942E8AB1
:105CC00059016A017B018C019101A201B3018B2F63
:105CD0009A2F0E94658AA3801A2D110F110BB12EE5
:105CE000C12ED12EE12EF12E012F0E94658A1901BD
:105CF0002A013B01B82FA92F2281922F990F990BCE
:105D0000392F492F592F692F792F892F08E00E94A9
:105D10002E8A59016A017B018C019101A201B30114
:105D20008B2F9A2F0E94658AB22E132F042F452E97
:105D3000562E672E782EA92E09C07AE0B72E10E0D5
:105D400000E0412C512C612C712CA12C0E94610B84
:105D50002B2D312F402F542D652D762D872D9A2DEB
:105D60002736FFE63F07FCE64F0751056105710541
:105D70008105910511F40C940C392736EFE63E07A6
:105D8000ECE64E075105610571058105910511F09D
:105D900008F093C12936F2E73F0741055105610537
:105DA00071058105910511F40C94013C2936E2E757
:105DB0003E0741055105610571058105910511F009
:105DC00008F0A3C02536F4E63F07410551056105FB
:105DD00071058105910509F480C52536E4E63E0785
:105DE00041055105610571058105910509F0A8F589
:105DF000A6E70E948C8A09F4CDC70E948C8A09F01C
:105E000060F4A8E60E948C8A09F4ADC5A5E70E945B
:105E10008C8A09F4A9C70C94C13E2B2D312F402F39
:105E2000542D652D762D872D9A2D2A33F6E23F07C6
:105E300041055105610571058105910509F41EC3F0
:105E400024363146410551056105710581059105ED
:105E500011F40C947A3C0C94C13E2B2D312F402F21
:105E6000542D652D762D872D9A2D2737FFE63F0778
:105E700041055105610571058105910511F40C94E9
:105E8000353A2737EFE63E074105510561057105B3
:105E90008105910509F0C0F42436F9E63F07410574
:105EA0005105610571058105910509F436C725364F
:105EB0003E4641055105610571058105910511F4C5
:105EC0000C94693A0C94C13E2B2D312F402F542D48
:105ED000652D762D872D9A2D2333F1E73F07410558
:105EE0005105610571058105910511F40C947A3C09
:105EF000253632474105510561057105810591053A
:105F000011F40C94233B0C94C13E2B2D312F402FC8
:105F1000542D652D762D872D9A2D2837F4E63F07D1
:105F2000F1E64F075105610571058105910509F4F9
:105F3000B5C22837E4E63E07E1E64E0751056105A4
:105F400071058105910511F008F050C02837F4E77C
:105F50003F0741055105610571058105910509F46A
:105F60008DC22837E4E73E074105510561057105FB
:105F70008105910509F0C8F42337F2E73F07410591
:105F80005105610571058105910511F40C94523C90
:105F90002337334741055105610571058105910599
:105FA00011F40C94663C0C94C13E2B2D312F402FE4
:105FB000542D652D762D872D9A2D2133F4E63F073C
:105FC000F1E64F075105610571058105910509F459
:105FD00069C2233634464146510561057105810584
:105FE000910511F40C947A3C0C94C13E2B2D312F69
:105FF000402F542D652D762D872D9A2D2336FDE6C5
:106000003F07F8E64F0751056105710581059105C8
:1060100009F46CC22336EDE63E07E8E64E0751056B
:10602000610571058105910509F0C8F42236F5E690
:106030003F07F4E64F07510561057105810591059C
:1060400009F44BC4223732474546510561057105B5
:106050008105910511F40C948E390C94C13E2B2DC1
:10606000312F402F542D652D762D872D9A2D2336D7
:10607000F2E33F07F9E64F07510561057105810518
:10608000910509F42FC22436E3E63E07ECE64E07FD
:106090005105610571058105910511F40C940939CB
:1060A0002D36354748465105610571058105910535
:1060B00011F00C94C13E0C94903C2B2D312F402FAD
:1060C000542D652D762D872D9A2D2136EDE63E0730
:1060D000E5E74E07E8E65E07610571058105910574
:1060E00011F40C94533A2136FDE63F07F5E74F07CC
:1060F000F8E65F07610571058105910511F008F06B
:10610000DAC02437E8E73E07E4E74E0751056105AA
:1061100071058105910509F4A5C62437F8E73F0705
:10612000F4E74F075105610571058105910511F0EF
:1061300008F055C02133E1E33E07E1E74E07510582
:10614000610571058105910511F40C94CF39213356
:10615000F1E33F07F1E74F0751056105710581053F
:10616000910509F0D0F42537E3E63E07EDE64E074A
:106170005105610571058105910511F40C94CF3924
:106180002033314341475105610571058105910572
:1061900011F40C948E390C94C13E2B2D312F402FCD
:1061A000542D652D762D872D9A2D2037E5E63E0757
:1061B000E2E74E075105610571058105910511F46E
:1061C0000C94233B2C363447444751056105710537
:1061D0008105910511F40C94FE3D0C94C13E2B2DCC
:1061E000312F402F542D652D762D872D9A2D293650
:1061F000ECE63E07E1E64E07E3E65E076105710562
:106200008105910509F4A7C12936FCE63F07F1E6AF
:106210004F07F3E65F07610571058105910509F0F8
:10622000E0F42437E4E63E07E7E74E075105610551
:1062300071058105910511F40C944C3E24373F46BD
:106240004F465246610571058105910511F00C9488
:10625000C13E0C9400000C94C33E2B2D312F402FD7
:10626000542D652D762D872D9A2D2633E9E63E0790
:10627000E5E74E07E5E65E076105710581059105D5
:1062800009F475C32037FCE63F07F5E64F07F8E64B
:106290005F07610571058105910509F464C32E3618
:1062A000314648465346610571058105910509F45B
:1062B000AFC50C94C13E2B2D312F402F542D652D91
:1062C000762D872D9A2D2437F3E73F07F5E64F0704
:1062D000F2E75F07610571058105910511F40C94E2
:1062E000E33A2437E3E73E07E5E64E07E2E75E07D9
:1062F000610571058105910511F008F055C023373E
:10630000F2E73F07F7E74F07F0E75F076105710521
:106310008105910511F40C94E63A2337E2E73E0734
:10632000E7E74E07E0E75E07610571058105910526
:1063300009F0C8F42237F7E73F07F0E74F075F0798
:10634000610571058105910509F4D4C023373546EF
:1063500042475047610571058105910511F40C9480
:10636000403D0C94C13E2B2D312F402F542D652DD7
:10637000762D872D9A2D2436FDE63F07F3E64F074D
:10638000F2E75F07610571058105910509F4EAC32C
:1063900021363C4645465247610571058105910508
:1063A00009F402C30C94C13E2B2D312F402F542DE4
:1063B000652D762D872D9A2D2437F2E73F07F1E6DC
:1063C0004F07F5E75F07610571058105910509F440
:1063D0001AC42437E2E73E07E1E64E07E5E75E0729
:1063E000610571058105910509F0C8F42437F3E7CB
:1063F0003F07F5E64F07F4E75F0761057105810583
:10640000910509F458C52737304748475447610577
:1064100071058105910509F4D3C40C94C13E2B2D5F
:10642000312F402F542D652D762D872D9A2D2F3607
:10643000FCE63F07FFE54F07F6E75F0761057105DB
:106440008105910509F439C32C36E1E63E07E4E7FE
:106450004E07E8E75E07610571058105910511F4B6
:106460000C94C83D223737464047554761057105B2
:106470008105910511F00C94C13EA8C683E080937C
:106480003E281092402810923F284EE358E262E1E5
:1064900084E392E00E94B6500C94C33E0E946615BD
:1064A0000C94C33E21E042E161E080ED0E94E15D99
:1064B00021E042E161E080ED0E94E15D21E042E106
:1064C00061E080ED0E94E15D21E042E161E080ED6C
:1064D0000E94E15D21E042E161E080ED0E94E15D2A
:1064E0000C94C33E0E94D80F0C94C33E0E94DE154C
:1064F0000C94C33E60916B0270916C0280E090E05E
:106500000E94528E8C0164E875E00E94668E892B91
:1065100019F477980C94C33E67E875E0C8010E94AF
:10652000668E892B19F4779A0C94C33E779903C031
:1065300084E895E002C087E895E09F938F938AE70F
:1065400094E09F938F930E941D8F0F900F900F9058
:106550000F900C94C33E60916B0270916C0280E0CE
:1065600090E00E94528E8C016EE475E00E94668E6F
:10657000892B09F077C060916B0270916C0280E00A
:1065800090E00E94528E8C01009711F40C94C33E4F
:1065900062E975E00E94668E892BB1F482E29FEF7A
:1065A000ACECBBE38093720290937302A0937402ED
:1065B000B093750244E050E064E470E082E792E05A
:1065C0000E948F900C94C33E68E975E0C8010E9458
:1065D000668E892BB1F482E29FEFACECBAE3809334
:1065E000720290937302A0937402B093750244E018
:1065F00050E064E470E082E792E00E948F900C9497
:10660000C33EC8010E943C8D2B013C0120E030E0DC
:10661000A9010E94DB848823D9F081E00E94020A4C
:106620009B01AC01C301B2010E94DF84609372023E
:1066300070937302809374029093750244E050E06B
:1066400064E470E082E792E00E948F900C94C33E75
:1066500086EE92E09F938F930E941D8F0F900F9074
:106660000C94C33E61E575E0C8010E94668E892BDB
:1066700009F077C060916B0270916C0280E090E04D
:106680000E94528E8C01009711F40C94C33E62E973
:1066900075E00E94668E892BB1F482E29FEFACEC2C
:1066A000BBE380936E0290936F02A0937002B0934D
:1066B000710244E050E060E470E08EE692E00E94F7
:1066C0008F900C94C33E68E975E0C8010E94668E05
:1066D000892BB1F482E29FEFACECBAE380936E02B7
:1066E00090936F02A0937002B093710244E050E067
:1066F00060E470E08EE692E00E948F900C94C33EBE
:10670000C8010E943C8D2B013C0120E030E0A90132
:106710000E94DB848823D9F082E00E94020A9B0158
:10672000AC01C301B2010E94DF8460936E027093DA
:106730006F02809370029093710244E050E060E435
:1067400070E08EE692E00E948F900C94C33E89ED3B
:1067500092E09F938F930E941D8F0F900F900C9447
:10676000C33E69E475E0C8010E94668E892B09F07A
:1067700073C060916B0270916C0280E090E00E94A7
:10678000528E8C01009711F40C94C33E62E975E0BF
:106790000E94668E892BB1F487ED94E3AFEEBCE3E3
:1067A0008093760290937702A0937802B093790257
:1067B00044E050E068E470E086E792E00E948F9049
:1067C0000C94C33E68E975E0C8010E94668E892B6F
:1067D00051F48AEC92E09F938F930E941D8F0F904B
:1067E0000F900C94C33EC8010E943C8D2B013C01CC
:1067F00020E030E0A9010E94DB84882319F180E0C9
:106800000E94020A4B015C0121EE3AE744E95EE393
:10681000C301B2010E941484A50194010E94DF8487
:106820006093760270937702809378029093790256
:1068300044E050E068E470E086E792E00E948F90C8
:106840000C94C33E8DEB92E09F938F930E941D8F1B
:106850000F900F900C94C33E0E94510A9F938F9308
:106860007F936F9386EB92E09F938F930E941D8F8F
:1068700082E00E94020A20916E0230916F024091E4
:106880007002509171020E945C87162F072FF82E1C
:10689000E92E81E00E94020AEF92FF920F931F936C
:1068A00020917202309173024091740250917502EE
:1068B0000E945C879F938F937F936F938AEA92E005
:1068C0009F938F930E941D8F0E94610B0FB6F894C7
:1068D000DEBF0FBECDBF0C94C33E60916B027091C2
:1068E0006C0280E090E00E94528E0097C1F00E94FE
:1068F0001F2320917309309174098217930709F1BE
:10690000909374098093730942E050E060E570E071
:1069100083E799E00E948F9083E794E002C08CE6C1
:1069200094E09F938F930E941D8F609173097091E3
:10693000740980E090E00E9431220E94610B0F9068
:106940000F9081E694E09F938F930E941D8F6FEFCD
:106950007FEF80E090E00E9431220E94610B0F9057
:106960000F900C94C33E0E94381F0C94C33EF40158
:106970008481843329F440E061E080E00E94821148
:1069800080916D02882311F40C94C33E1F928F9363
:106990008EE594E09F938F930E941D8F0F900F9030
:1069A0000F900F900C94C33EF4018481893709F055
:1069B00070C060916B0270916C0280E090E00E9468
:1069C000528E8C0164E875E00E94668E892B31F44A
:1069D000809154029091550290640CC067E875E074
:1069E000C8010E94668E892B91F480915402909187
:1069F00055029F7B909355028093540242E050E0F1
:106A000066E170E084E592E00E948F9042C06DE9FB
:106A100075E0C8010E94668E892B21F58091D41AF9
:106A20008F938091D31A8F938091D21A8F938091F4
:106A3000D11A8F938091D01A8F938091CF1A8F9310
:106A40008091CE1A8F938091CD1A8F938FE792E029
:106A50009F938F930E941D8F0FB6F894DEBF0FBED9
:106A6000CDBF17C0809154029091550296FF03C08C
:106A700084E895E002C087E895E09F938F938BE7C9
:106A800092E09F938F930E941D8F0F900F900F9015
:106A90000F9080916D02882311F40C94C33E1F92D5
:106AA0008F938BE594E09F938F930E941D8F0F909F
:106AB0000F900F900F900C94C33EF40184818737A0
:106AC000E9F560916B0270916C0280E090E00E94A9
:106AD000528E0097D9F00E943C8D2B013C0120E0A2
:106AE00030E0A9010E94DB84882381F040927A0281
:106AF00050927B0260927C0270927D0244E050E0F2
:106B00006CE470E08AE792E00E948F9080917D02B1
:106B10008F9380917C028F9380917B028F938091E1
:106B20007A028F938DE692E09F938F930E941D8F40
:106B30000F900F900F900F900F900F9080916D021B
:106B4000882311F40C94C33E1F928F9388E594E040
:106B50009F938F930E941D8F0F900F900F900F9017
:106B60000C94C33E60916B0270916C0280E090E0E7
:106B70000E94528E5C0164E875E00E94668E00916E
:106B8000540210915502892B11F4106808C067E86F
:106B900075E0C5010E94668E892B71F41F771093F2
:106BA00055020093540242E050E066E170E084E553
:106BB00092E00E948F9013C017FF03C084E895E015
:106BC00002C087E895E09F938F9389E692E09F93B8
:106BD0008F930E941D8F0F900F900F900F908091B8
:106BE0006D02882311F40C94C33E1F928F9385E5A8
:106BF00094E09F938F930E941D8F0F900F900F90A2
:106C00000F900C94C33E60916B0270916C0280E017
:106C100090E00E94528E5C0163EA75E00E94668EED
:106C2000892B11F489E108C067EA75E0C5010E946B
:106C3000668E892B49F480E18093C4001092C500D0
:106C400082E08093C00055C06BEA75E0C5010E94E8
:106C5000668E892B11F488E0EFCF60EB75E0C501FB
:106C60000E94668E892B39F065EB75E0C5010E94A4
:106C7000668E892B11F483E0DFCF8091C4008931C7
:106C800041F484E692E09F938F930E941D8F0F90B2
:106C90000F908091C400803141F48FE592E09F9382
:106CA0008F930E941D8F0F900F908091C4008830A9
:106CB00041F489E592E09F938F930E941D8F0F907E
:106CC0000F908091C400833041F483E592E09F935C
:106CD0008F930E941D8F0F900F908091C400883079
:106CE00041F48DE492E09F938F930E941D8F0F904B
:106CF0000F9080916D02882311F40C94C33E1F9273
:106D00008F9382E594E09F938F930E941D8F0F9045
:106D10000F900F900F900C94C33E60916B02709196
:106D20006C0280E090E00E94528E62E975E00E9461
:106D3000668E892B11F481E001C080E00E9401225F
:106D400080916D02882311F40C94C33E1F928F939F
:106D50008FE494E09F938F930E941D8F0F900F906C
:106D60000F900F900C94C33E0E94272080916D02DB
:106D7000882311F40C94C33E1F928F938CE494E00B
:106D80009F938F930E941D8F0F900F900F900F90E5
:106D90000C94C33E0E94232080916D02882311F43D
:106DA0000C94C33E1F928F9389E494E09F938F933A
:106DB0000E941D8F0F900F900F900F900C94C33E68
:106DC00060916B0270916C0280E090E00E94528EA4
:106DD0000E94408D803168F480936F090E949D6607
:106DE00041E050E065E170E08FE699E00E948F900D
:106DF000CAC780916F091F928F9383E492E09F939B
:106E00008F930E941D8F0F900F900F900F90BBC714
:106E100060916B0270916C0280E090E00E94528E53
:106E20000E94408D95EF980F903168F48093530243
:106E30000E94446541E050E064E170E083E592E047
:106E40000E948F90A0C7809153021F928F938AE374
:106E500092E09F938F930E941D8F0F900F900F9041
:106E60000F9091C760916B0270916C0280E090E08E
:106E70000E94528E009781F04AE050E0BC018CEBFA
:106E80009AE10E94768E4AE050E060E070E08CEB80
:106E90009AE10E948F9077C78CEB9AE19F938F9332
:106EA0008AEB95E09F938F930E940B8F0F900F902A
:106EB0000F900F9068C760916B0270916C0280E038
:106EC00090E00E94528E5C016AED73E00E94668E33
:106ED000892B99F4219A80915402909155028061F6
:106EE000909355028093540242E050E066E170E0D6
:106EF00084E592E00E948F9046C762E575E0C50187
:106F00000E94668E892B99F4229A80915402909166
:106F100055028062909355028093540242E050E003
:106F200066E170E084E592E00E948F902CC76CEBE4
:106F300073E0C5010E94668E892B99F4239A809193
:106F400054029091550280649093550280935402AC
:106F500042E050E066E170E084E592E00E948F90AC
:106F600012C769EF74E0C5010E94668E892B99F4FF
:106F7000239A809154029091550280689093550213
:106F80008093540242E050E066E170E084E592E0D4
:106F90000E948F90F8C66BE179E0C5010E94668E71
:106FA000892B31F581E08093E22385ED9AE190937E
:106FB000E4238093E3231092E6231092E52380914B
:106FC000540290915502916090935502809354021F
:106FD00042E050E066E170E084E592E00E948F902C
:106FE00042EE53E262E184E392E00E94B650CBC6E7
:106FF00063EE73E0C5010E94668E892BD1F4E5E053
:10700000FBE1119211922BE1E532F207D1F7809169
:1070100054029091550292609093550280935402CD
:1070200042E050E066E170E084E592E00E948F90DB
:10703000AAC667E875E0C5010E94668E20915402D9
:1070400030915502892BA1F42F703C7F309355026B
:10705000209354022B9A42E050E066E170E084E510
:1070600092E00E948F90809147280E9459658BC6BC
:1070700024FF03C084E895E002C087E895E09F9371
:107080008F938FE292E09F938F930E941D8F809148
:1070900054020F900F900F900F9085FF03C084E86B
:1070A00095E002C087E895E09F938F9384E292E099
:1070B0009F938F930E941D8F809154020F900F9089
:1070C0000F900F9086FF03C084E895E002C087E828
:1070D00095E09F938F9389E192E09F938F930E9415
:1070E0001D8F809154020F900F900F900F9087FF8B
:1070F00003C084E895E002C087E895E09F938F93F2
:107100008EE092E09F938F930E941D8F8091540296
:10711000909155020F900F900F900F9090FF03C029
:1071200084E895E002C087E895E09F938F9383E021
:1071300092E09F938F930E941D8F809154029091B3
:1071400055020F900F900F900F9091FF03C084E8AD
:1071500095E002C087E895E09F938F9388EF91E0D8
:107160009F938F930E941D8F80915402909155029E
:107170000F900F900F900F9091FF05C682EC95E055
:107180000E94418F55E0A52E5BE1B52E0BE010E08B
:107190006AEC862E65E0962EF50180819181F2E001
:1071A000AF0EB11C9F938F931F930F939F928F925B
:1071B0000E940B8F0F5F1F4F0F900F900F900F903B
:1071C0000F900F900B31110539F7DDC585E494E080
:1071D0009F938F930E941D8F80916D020F900F904F
:1071E000882361F01F928F9382E494E09F938F93A2
:1071F0000E941D8F0F900F900F900F9088E10FB697
:10720000F89480936000109260000FBE0C94007C94
:10721000BAC50E94925DB7C560916B0270916C0215
:1072200080E090E00E94528E8C0164E875E00E943C
:10723000668E892BA9F40E94436480915402909138
:1072400055028D7F8160909355028093540242E0F5
:1072500050E066E170E084E592E00E948F9093C573
:1072600067E875E0C8010E94668E892BA1F40E9430
:10727000FB6380915402909155028C7F909355024C
:107280008093540242E050E066E170E084E592E0D1
:107290000E948F9078C565ED75E0C8010E94668EEA
:1072A000892BA9F40E94FB638091540290915502AE
:1072B0008E7F8260909355028093540242E050E0AA
:1072C00066E170E084E592E00E948F905CC5809159
:1072D000540281FF0FC085ED95E09F938F9384EF5B
:1072E00091E09F938F930E941D8F0F900F900F90AE
:1072F0000F9049C580FF03C084E895E002C087E88D
:1073000095E09F938F9380EF91E09F938F930E94DE
:107310001D8F0F900F900F900F9035C58091E02337
:107320008F938091DF238F938091DE238F938091C1
:10733000DD238F938091DC238F938091DB238F93C8
:107340008091DA238F938091D9238F938091D823D2
:107350008F938091D7238F938091D6238F938091A1
:10736000D5238F938FE194E09F938F930E941D8F7D
:1073700080916D020FB6F894DEBF0FBECDBF88239B
:1073800009F401C51F928F938CE194E09F938F9332
:107390000E941D8F0F900F900F900F90F4C4F894DF
:1073A00081E090E029E0FC0120935700C895E02C93
:1073B00080E090E0FC0120935700C895F02C789471
:1073C000F89483E090E0FC0120935700C895002DCD
:1073D00082E090E0FC0120935700C895102D78942E
:1073E0008091791B8F938091781B8F938091771B6D
:1073F0008F938091761B8F9322E134E03F932F93FC
:107400000E941D8F1F92EF921F92FF921F920F9367
:107410001F921F938BEE93E09F938F930E941D8F7B
:107420000E94C120809166001F928F938FED93E0A0
:107430009F938F930E941D8F0E94610B80916D021C
:107440000FB6F894DEBF0FBECDBF882309F49BC4EE
:107450001F928F938CED93E09F938F930E941D8FCB
:107460000F900F900F900F908EC460E070E080E05E
:1074700090E00E946A0B60E070E081E090E00E9482
:107480006A0B80916D02882309F47DC41F928F934B
:1074900089ED93E09F938F930E941D8F0F900F9023
:1074A0000F900F9070C40E94FB1E0E94610B809190
:1074B0006D02882309F467C41F928F9386ED93E0D1
:1074C0009F938F930E941D8F0F900F900F900F909E
:1074D0005AC460916B0270916C0280E090E00E944F
:1074E000528E6AED75E00E94668E892B31F5F89414
:1074F0008AEA99E00E94A3515C01009769F0C501F6
:107500000F960E94A754B50184E092E00E945D515D
:10751000C5010E944B52F0CF8AEA99E00E94305296
:10752000892B29F08AEA99E00E94DC51F5CF8AEA9A
:1075300099E00E949F51789434C08AEA99E00E94B1
:10754000A3515C0100EE15E0A114B10451F1F50165
:1075500086811F928F9380851F928F9385811F92C2
:107560008F9381851F928F9387811F928F93848140
:107570001F928F9383811F928F9382811F928F938B
:1075800082851F928F931F930F930E940B8FC501CB
:107590000E944B525C010FB6F894DEBF0FBECDBF08
:1075A000D3CF80916D02882309F4EDC31F928F938E
:1075B00083ED93E09F938F930E941D8F0F900F9008
:1075C0000F900F90E0C30E94812CDDC360916B028D
:1075D00070916C0280E090E00E94528E8C016FE10D
:1075E00076E00E94668E892B91F4809154029091EE
:1075F0005502977F909355028093540242E050E0E9
:1076000066E170E084E592E00E948F90BCC368E977
:1076100075E0C8010E94668E892B91F48091540216
:10762000909155029860909355028093540242E0E5
:1076300050E066E170E084E592E00E948F90A3C381
:107640000E940809A0C360916B0270916C0280E0F7
:1076500090E00E94528EFC0120812332B1F44AE076
:1076600050E060E070E001960E94F48A1B01609196
:107670006B0270916C0280E090E00E94528EF4E008
:107680002F1631040CF094C002C0212C312C00972D
:1076900009F48EC01982BE016F5F7F4F0E940327DD
:1076A00029013A014B01B82FA92F8AE0829DF001F0
:1076B000839DF00D1124EB52F54E20812A833181F8
:1076C0003B8382818C8393819D8324812E833581AA
:1076D0003F8386818887978199879201A301B401AE
:1076E0008B2F9A2FAA80BB80CC80DD80EE80FF801C
:1076F000088519850E94838A09F45DC089818823E1
:1077000051F18CF02A81422A3B81532A8C81682ACC
:107710009D81792A2E81822A3F81932A8885B82BE0
:107720009985A92B18C040945094609470948094CB
:107730009094B095A0952A8142223B8153228C815E
:1077400068229D8179222E8182223F819322888521
:10775000B8239985A92340825182628273828482F0
:107760009582B683A78348E250E068E170E085ED3A
:107770009AE10E948F908BEC93E09F938F930E94ED
:107780001D8F8AE0829DF001839DF00D1124EB5244
:10779000F54E2081318142815381648175818681DA
:1077A00097810E94BA230E94610B0F900F9003C033
:1077B00082E00E9497288FEB93E09F938F930E9423
:1077C0001D8F2FEF3FEF4FEF5FEF60E070E080E045
:1077D00090E00E94BA230E94610B80916D020F908D
:1077E0000F90882309F4CFC21F928F938CEB93E004
:1077F0009F938F930E941D8F0F900F900F900F906B
:10780000C2C260916B0270916C0280E090E00E94B5
:10781000528EFC0120812332A1F44AE050E060E066
:1078200070E001960E94F48A8B0160916B02709166
:107830006C0280E090E00E94528E04301105ECF45E
:1078400002C000E010E00097C1F04AE050E060E0C4
:1078500070E00E94288C2AE0209FF001219FF00D0B
:107860001124EB52F54E7187608748E250E068E1E1
:1078700070E085ED9AE10E948F9081E00E94972848
:1078800080916D02882309F47EC21F928F9389EB49
:1078900093E09F938F930E941D8F0F900F900F90F6
:1078A0000F9071C20E94E05480916D02882309F408
:1078B0006AC21F928F9386EB93E09F938F930E94EF
:1078C0001D8F0F900F900F900F905DC20E940C299A
:1078D00080916D02882309F456C21F928F9383EB27
:1078E00093E09F938F930E941D8F0F900F900F90A6
:1078F0000F9049C280E090E00E94DD2080916D02EF
:10790000882309F440C21F928F9380EB93E09F93EA
:107910008F930E941D8F0F900F900F900F9033C286
:107920008091CB1F81FF2DC00E94831E892B49F5BA
:107930008091C21B8F938091C11B8F938091C01B3C
:107940008F938091BF1B8F9385EA93E09F938F93D2
:107950000E941D8F80915F288F9380915E288F9366
:1079600080915D288F9380915C288F9388E993E0C4
:107970009F938F930E941D8F0FB6F894DEBF0FBEAA
:10798000CDBF0E94610B8091CB1F9091CC1F90FFC7
:1079900063C081E090E00E94FA1D3B014C0180E051
:1079A00090E00E94FA1D1B012C010E94511D9F9224
:1079B0008F927F926F9287E893E09F938F930E94BC
:1079C0001D8F5F924F923F922F9287E793E09F9394
:1079D0008F930E941D8F222D332D442D552D662D02
:1079E000772D882D992D0E94F41B9F938F937F9361
:1079F0006F938CE693E09F938F930E941D8F222DAF
:107A0000332D442D552D662D772D882D992D0E94CF
:107A1000551C9F938F937F936F938EE593E09F9375
:107A20008F930E941D8F222D332D442D552D662DB1
:107A3000772D882D992D0E94B61C9F938F937F934D
:107A40006F938BE493E09F938F930E941D8F0FB6EB
:107A5000F894DEBF0FBECDBF0E94610B80916D0216
:107A6000882309F490C11F928F9388E493E09F9339
:107A70008F930E941D8F0F900F900F900F9083C1D6
:107A80008091CB1F82FF2BC021E048E061E083E0C2
:107A90000E94F7128091BD1B8F938091BC1B8F9326
:107AA0008091BB1B8F938091BA1B8F938091B91BE0
:107AB0008F938091B81B8F938091B71B8F93809188
:107AC000B61B8F9381E393E09F938F930E941D8F4A
:107AD0000E94610B0FB6F894DEBF0FBECDBF809140
:107AE000CB1F9091CC1F91FF41C00E944117B62E31
:107AF000A72E982E892E20E030E048EC52E4D501E4
:107B0000F4016B2F7A2F8F2F9E2F0E945C8720E825
:107B100036EE45EC57E40E94DF8421E03EED42E47E
:107B20005EE30E94BF879B01AC0160E070E080E8EB
:107B30009FE30E9414842BE43AE34DEB57E30E9449
:107B4000DF849F938F937F936F938F929F92AF92D7
:107B5000BF9288E193E09F938F930E941D8F0E94B4
:107B6000610B0FB6F894DEBF0FBECDBF80916D02E2
:107B7000882309F408C11F928F9385E193E09F93B6
:107B80008F930E941D8F0F900F900F900F90FBC04E
:107B900060916B0270916C0280E090E00E94528EC6
:107BA00064E276E00E94668E892BB1F460916B02EC
:107BB00070916C0280E090E00E94528E009709F470
:107BC000E2C00E94408D803108F0DDC090915201EA
:107BD000982B90935201D7C0809152018F701F92C1
:107BE0008F9383EE91E09F938F930E941D8F0E944D
:107BF000610B0F900F900F900F90C5C060916B02BA
:107C000070916C0280E090E00E94528E009711F11A
:107C10004AE050E060E070E00E94F48A603198F43D
:107C2000609352021F926F9388E093E09F938F932B
:107C30000E941D8F41E050E063E170E082E592E038
:107C40000E948F9011C0809152021F928F938FEFEC
:107C500092E006C0809152021F928F9386EF92E0CD
:107C60009F938F930E941D8F0F900F900F900F90F6
:107C70000E94610B80916D02882309F484C01F92D9
:107C80008F9383EF92E09F938F930E941D8F0F90AD
:107C90000F900F900F9077C060916B0270916C0203
:107CA00080E090E00E94528E8C0164E875E00E94B2
:107CB000668E892BA1F40E94AC628091540290914F
:107CC00055029061909355028093540242E050E037
:107CD00066E170E084E592E00E948F9054C067E80E
:107CE00075E0C8010E94668E892B41F5F8940E94C8
:107CF000BA6288E10FB6F894809360001092600039
:107D00000FBE84B7877F84BF8091600088618093B5
:107D10006000109260007894809154029091550216
:107D20009F7E909355028093540242E050E066E1BA
:107D300070E084E592E00E948F9025C069E276E0D1
:107D4000C8010E94668E2091540230915502892B01
:107D500021F434FF18C0F894FFCF34FF03C084E847
:107D600095E002C087E895E09F938F938FED91E0B7
:107D70009F938F930E941D8F0F900F900F900F90E5
:107D800002C00E941F1FEA85FB851182108283E0DA
:107D90002B960FB6F894DEBF0FBECDBFDF91CF910B
:107DA0001F910F91FF90EF90DF90CF90BF90AF9019
:107DB0009F908F907F906F905F904F903F902F900B
:107DC00008950F931F93CF93DF93EC018A0188816D
:107DD0009981009711F18431904121F01982188224
:107DE00083E020C06231E9F4A80162E170E08BE930
:107DF00099E00E949E2D84E080933E2810924028B6
:107E000010923F2810934228009341284EE358E2F5
:107E100062E184E392E00E94B65084E190E19983AC
:107E2000888381E0DF91CF911F910F9108950E9487
:107E3000A0626C9A6B9A6A9A6F9A729A749A739A01
:107E4000779A809880B3897F80BB8398849887E0F5
:107E500080937E00549A0E94A02A0E94D22A81E038
:107E60000E94760980E090E00E94B60C0E94175CA8
:107E70000E94650A6093CD237093CE238093CF2315
:107E80009093D0238091540286FD239A0895CF9336
:107E9000DF93EC0188819981009741F08F3F9F40EB
:107EA00009F48CC01982188283E093C00E94173FA6
:107EB0008091540280FD05C081FF01C01D9B0E947E
:107EC000FB63809170008C7F809370008091B6007E
:107ED00080628093B6001092B20082E08093B1007D
:107EE0008091B6008770E1F7809170008160809387
:107EF000700062E279E080E090E00E948A620E9475
:107F0000232080E00E94012286E69EE09F938F93CB
:107F10000E941D8F0E94D80F8091CB1F0F900F9051
:107F200086FD0E943E5D8091CB1F9091CC1F90FDFD
:107F30000E940D1D8091CB1F87FF06C021E04CE001
:107F400061E080ED0E94E15D80916F090E949D6675
:107F5000809153020E9444650E94416580939A0972
:107F6000809153020E94446580916F091F928F9304
:107F700080919A091F928F938EE296E09F938F9340
:107F80000E940B8F10929C0910929B090F900F90EA
:107F90000F900F900F900F9088E492E090935A28E2
:107FA0008093592883E290E09093AD118093AC11B7
:107FB0008FEF9FE09983888381E00BC06332E1F704
:107FC00046EF53E260E070E08BE999E00E949E2D5D
:107FD000E3CFDF91CF9108958436910514F19F93FB
:107FE0008F9380E496E09F938F930E940B8F8091F4
:107FF000D5239091D623A091D723B091D823019671
:10800000A11DB11D8093D5239093D623A093D72390
:10801000B093D8230F900F900F900F9081E090E0D5
:10802000089580E090E008952F923F924F925F92E2
:108030006F927F928F929F92AF92BF92CF92DF9278
:10804000EF92FF920F931F93CF93DF93CDB7DEB7DD
:10805000C859D1090FB6F894DEBF0FBECDBFC157C6
:10806000DF4F99838883CF58D0408A01633871F4F9
:108070008FE999E0C956DF4F6883C759D0400E9405
:10808000F94EC956DF4F6881C759D040C157DF4FFD
:10809000A881B981CF58D0402D913C912D3ABFE0B5
:1080A0003B0709F483C340F42115310581F02330E7
:1080B0003E4009F4C1C3B5C32E3B4FE0340709F479
:1080C00091C3253C3F4011F40C94104CAAC344EEDC
:1080D00052E061E870E08FE999E00E94DF4E83E0B2
:1080E0009EE05BC3E3E0F0E0EC0FFD1FE00FF11F4B
:1080F0001082C8010E94EC3F892B89F720E030E014
:1081000040E050E0652D627070E080E090E0A0E01B
:108110000E948C8A09F0CEC5C257DF4F2881CE5805
:10812000D040287030E040E050E060E070E080E057
:1081300090E0A0E00E948C8AA1F127E04AE250E0A2
:108140006BE270E089E290E00E94315980E598E2AC
:108150000E949F5BBC01882777FD8095982F0E9425
:108160007E8520E030E048EC52E40E94DF849F935B
:108170008F937F936F9384E796E09F938F931F92E3
:1081800087E78F93CE01800F911F03969F938F9364
:108190000E946E8F080F191F0FB6F894DEBF0FBE36
:1081A000CDBFC257DF4F2881CE58D040207130E07C
:1081B00040E050E060E070E080E090E0A0E00E94ED
:1081C0008C8AF1F126E04AE250E06BE270E089E24D
:1081D00090E00E94315981E090E00E94EF0A809384
:1081E0006E098EE29BE10E949F5BBC01882777FDB0
:1081F0008095982F0E947E8520E030E048EC52E484
:108200000E94DF849F938F937F936F938EE796E016
:108210009F938F931F9287E78F93C8010296E1E0A7
:10822000F0E0EC0FFD1F8E0F9F1F9F938F930E9416
:108230006E8F080F191F0FB6F894DEBF0FBECDBFAB
:10824000C657DF4F2881CA58D04030E040E050E0A8
:1082500060E070E080E090E0A0E00E948C8A01F194
:108260000E94AB0A9F938F937F936F9389E896E068
:108270009F938F931F9287E78F93C801029641E0E7
:1082800050E04C0F5D1F840F951F9F938F930E94AA
:108290006E8F080F191F0FB6F894DEBF0FBECDBF4B
:1082A000C257DF4F2881CE58D040207430E040E0E4
:1082B00050E060E070E080E090E0A0E00E948C8AF6
:1082C00031F18091D0238F938091CF238F93809130
:1082D000CE238F938091CD238F9387E996E09F9350
:1082E0008F931F9287E78F93C8010296A1E0B0E0B9
:1082F000AC0FBD1F8A0F9B1F9F938F930E946E8FA1
:10830000080F191F0FB6F894DEBF0FBECDBFC257BE
:10831000DF4F2881CE58D040207830E040E050E058
:1083200060E070E080E090E0A0E00E948C8A41F183
:10833000F8948091362890913728A0913828B091F0
:1083400039287894BF93AF939F938F9385EA96E0F3
:108350009F938F931F9287E78F93C801029621E026
:1083600030E02C0F3D1F820F931F9F938F930E942D
:108370006E8F080F191F0FB6F894DEBF0FBECDBF6A
:1083800020E0372D317040E050E060E070E080E0A8
:1083900090E0A0E00E948C8A09F09DC420E0372D77
:1083A000327040E050E060E070E080E090E0A0E0FB
:1083B0000E948C8A09F017C520E0372D347040E008
:1083C00050E060E070E080E090E0A0E00E948C8AE5
:1083D00009F03AC520E0372D387040E050E060E009
:1083E00070E080E090E0A0E00E948C8A09F05BC51C
:1083F00020E0372D307140E050E060E070E080E038
:1084000090E0A0E00E948C8A09F0D5C520E0372DCD
:10841000307240E050E060E070E080E090E0A0E08A
:108420000E948C8A09F0F7C520E0CD56DF4F3881D5
:10843000C359D04040E050E060E070E080E090E060
:10844000A0E00E948C8A09F013C620E0CC56DF4FD2
:108450003881C459D04040E050E060E070E080E0F6
:1084600090E0A0E00E948C8A09F030C620E030E065
:10847000482D417050E060E070E080E090E0A0E0C6
:108480000E948C8A09F050C620E030E0482D4270EE
:1084900050E060E070E080E090E0A0E00E948C8A14
:1084A00009F075C620E030E0CE56DF4F4881C25952
:1084B000D04050E060E070E080E090E0A0E00E94FA
:1084C0008C8A09F097C620E030E0482D487050E0D3
:1084D00060E070E080E090E0A0E00E948C8A09F00B
:1084E000B3C620E030E0482D407150E060E070E01D
:1084F00080E090E0A0E00E948C8A09F0D5C620E0E0
:1085000030E0482D407250E060E070E080E090E0A4
:10851000A0E00E948C8A09F0F7C620E030E0482DE8
:10852000407450E060E070E080E090E0A0E00E94E5
:108530008C8A09F019C7F82DF078EF2E20E030E092
:108540004F2F50E060E070E080E090E0A0E00E94FB
:108550008C8A09F039C7292D2170F22E20E030E0F5
:1085600040E05F2D60E070E080E090E0A0E00E94DD
:108570008C8A09F033C720E030E04E2D50E060E0F7
:1085800070E080E090E0A0E00E948C8A09F031C7A2
:1085900020E030E040E05F2D60E070E080E090E0BF
:1085A000A0E00E948C8A09F056C720E030E040E04D
:1085B000592D527060E070E080E090E0A0E00E94F1
:1085C0008C8A09F07AC720E030E040E0592D5470E1
:1085D00060E070E080E090E0A0E00E948C8A09F00A
:1085E0009CC720E030E040E0592D507160E070E021
:1085F00080E090E0A0E00E948C8A09F0BEC720E0F5
:1086000030E040E0592D507260E070E080E090E092
:10861000A0E00E948C8A09F0EDC720E030E040E045
:10862000592D507460E070E080E090E0A0E00E947E
:108630008C8A11F00C94374B20E030E040E0592D4B
:10864000587060E070E080E090E0A0E00E948C8ACA
:1086500011F00C94764B20E030E040E0CB56DF4F39
:108660005881C559D04060E070E080E090E0A0E023
:108670000E948C8A11F00C94A74B779A8091730911
:108680009091740992FD749AC257DF4F2881CE5899
:10869000D040372DA401652DCF56DF4F7881C159C9
:1086A000D040842D962DA0E0FE0133967F010E94DC
:1086B0008C8A11F00C94DE4B809152028061898388
:1086C000809193098A83F701E00FF11F1082809156
:1086D00073099091740998012D5F3F4F790180FFD4
:1086E0000CC0FF922F9386E098E09F938F930E9497
:1086F0000B8F0F900F900F900F90B701CE01019646
:108700000E9428588091540282FF0AC026E334E276
:10871000A701BE016F5F7F4F8BE592E00E94AE5CC8
:10872000809173099091740982FD73980E9443644B
:108730008FE999E00E94FB4E80915402909155027E
:1087400090FF3BC00F5F1F4F0E944165F82E89E1EB
:108750000E945965209154023091550230FF29C082
:108760007398809193098F5F809393098A83B801EE
:108770006F5F7F4FCE0101960E9428588FE999E0E4
:108780000E94FB4E40E050E065E88091B01190916E
:10879000B1110E94B6508DEA9FE0C157DF4FA8810A
:1087A000B981CF58D0408D939C9338C000E010E041
:1087B000D1CF8F2D0E945965739A80917009909145
:1087C0007109892B11F00E94FB63809193098F5FDF
:1087D00080939309809173099091740982FF7FCCF3
:1087E000739A7DCC8BE899E00E945C53892BB1F0A1
:1087F0000E9443648091540287FD2B9860E470E0EE
:108800008BE899E00E94355385EC9FE0C157DF4F1C
:10881000E881F981CF58D0409183808381E00C9426
:10882000234CC157DF4FA881B981CF58D0401D924A
:108830001C9283E00C94234C623181F780915402A6
:108840009091550291FD4BCC20917A0230917B02A0
:1088500040917C0250917D026091CD237091CE2396
:108860008091CF239091D0230E94DB8487FF14C096
:108870008091D9239091DA23A091DB23B091DC235E
:108880000196A11DB11D8093D9239093DA23A09363
:10889000DB23B093DC2323CCF80180818130D1F439
:1088A0000180F281E02D2081C257DF4F2883CE580E
:1088B000D04071808280938054803581CF56DF4FC5
:1088C0003883C159D0404680678020843184A12CF0
:1088D000B12C3DC0823081F4A380B480212C312C96
:1088E000B1E0C257DF4FB883CE58D040712C812CF5
:1088F00020E8922E512C24C0833099F0843009F066
:10890000EECB212C312CA12CB12CE5E0C257DF4F4E
:10891000E883CE58D040712C812C912C92E0592EB6
:108920000FC0212C312CA12CB12CF5E0C257DF4F08
:10893000F883CE58D040712C812C912C552453941F
:10894000CF56DF4F1882C159D040412C612C282DC1
:108950002470CE56DF4F2883C259D04020E030E04B
:10896000CE56DF4F4881C259D04050E060E070E001
:1089700080E090E0A0E00E948C8A09F08C9AC257B7
:10898000DF4F3881CE58D0403072C657DF4F388322
:10899000CA58D040232F30E040E050E060E070E063
:1089A00080E090E0A0E00E948C8A11F00E94AB0A67
:1089B000472D4074CD56DF4F4883C359D04020E047
:1089C000342F40E050E060E070E080E090E0A0E014
:1089D0000E948C8A11F00E94831E572D5078CC562D
:1089E000DF4F5883C459D04020E0352F40E050E09D
:1089F00060E070E080E090E0A0E00E948C8A51F09E
:108A00000E94510A6093432870934428809345281C
:108A100090934628C257DF4F2881CE58D04021700E
:108A200030E040E050E060E070E080E090E0A0E006
:108A30000E948C8AF1F08CEB9AE19F938F9384E5EE
:108A400096E09F938F931F9287E78F93CE010396B3
:108A50009F938F930E946E8F7C010E94EC3F0FB614
:108A6000F894DEBF0FBECDBF892B09F038CB87014C
:108A700002C000E010E0C257DF4F2881CE58D0403E
:108A8000227030E040E050E060E070E080E090E094
:108A9000A0E00E948C8A09F442C0C80102966CE5ED
:108AA00076E0A1E0B0E0AC0FBD1F8A0F9B1F0E94D3
:108AB0006F8E0D5F1F4FB0E5CB2EB8E2DB2E8CEE34
:108AC000E82E83E0F82E27E7F60181916F011F92CF
:108AD0008F93FF92EF921F922F93C801029641E06D
:108AE00050E04C0F5D1F840F951F9F938F93C856C6
:108AF000DF4F2883C859D0400E946E8F080F191F7E
:108B00000FB6F894DEBF0FBECDBFC856DF4F288129
:108B1000C859D04078E5C71678E2D706A9F6C257FB
:108B2000DF4F2881CE58D040247030E040E050E044
:108B300060E070E080E090E0A0E00E948C8A09F4A0
:108B400061C0C801029660E676E0A1E0B0E0AC0F3B
:108B5000BD1F8A0F9B1F0E946F8E0C5F1F4F7E01EF
:108B6000BAE7EB0EF11C80E1F70111928A95E9F763
:108B700028E0A70168E980EB0E943B116701F8E05B
:108B8000CF0ED11C4CEE53E027E7D7018D917D012C
:108B90001F928F935F934F931F922F93C80102965A
:108BA000E1E0F0E0EC0FFD1F8E0F9F1F9F938F936E
:108BB000C856DF4F2883C859D040CA56DF4F488374
:108BC000C659D040C956DF4F5883C759D0400E947C
:108BD0006E8F080F191F0FB6F894DEBF0FBECDBF02
:108BE000C856DF4F2881C859D040CA56DF4F488148
:108BF000C659D040C956DF4F5881C759D040EC14F0
:108C0000FD0419F6792D7078CB56DF4F7883C5595E
:108C1000D04020E030E040E0572F60E070E080E09E
:108C200090E0A0E00E948C8AE1F48091700990911C
:108C300071099F938F9385E696E09F938F931F9280
:108C400087E78F93CE01800F911F03969F938F9399
:108C50000E946E8F080F191F0FB6F894DEBF0FBE6B
:108C6000CDBF20E030E040E050E0652D617070E065
:108C700080E090E0A0E00E948C8A09F43FCAE3E023
:108C8000F0E0EC0FFD1FE00FF11F80E28083E9EFC1
:108C9000F3E280810F5F1F4F882309F423CA80818C
:108CA000A1E0B0E0AC0FBD1FA00FB11F12968C93D6
:108CB0003196EFCFCE01800F911F6CE676E00396E0
:108CC0000E946F8E095F1F4FC8010E94EC3F892BE5
:108CD00009F005CA21CA2114310409F45FCBF894C4
:108CE00060913628709137288091382890913928E2
:108CF000C657DF4F688379838A839B83CA58D040E5
:108D000078948091261B9091271BA091281BB091ED
:108D1000291BC657DF4F288139814A815B81CA5898
:108D2000D040281B390B4A0B5B0BCA01B9010E94CA
:108D30007C856B017C01B10180E090E00E947C8524
:108D40009B01AC01C701B6010E94DF847C01FF9248
:108D50008F937F936F9380EB96E09F938F931F92F7
:108D600087E78F939E01200F311F2D5F3F4F3F9369
:108D70002F93C956DF4F6883C759D040CA56DF4F7B
:108D80007883C659D0400E946E8F080F191FC956AC
:108D9000DF4F6881C759D040CA56DF4F7881C65926
:108DA000D040862F972FAE2DBF2D809348289093CB
:108DB0004928A0934A28B0934B28C657DF4F4881D3
:108DC00059816A817B81CA58D0404093261B5093B9
:108DD000271B6093281B7093291B0FB6F894DEBFE6
:108DE0000FBECDBFDBCA2114310409F4E5CAF894E3
:108DF0008091FD1A9091FE1AA091FF1AB091001B6C
:108E000078949F938F93809159028F938091580209
:108E10008F938DEB96E09F938F931F9287E78F93AD
:108E2000C8010296A1E0B0E0AC0FBD1F8A0F9B1FE6
:108E30009F938F930E946E8F080F191F0FB6F8949F
:108E4000DEBF0FBECDBFB8CAF89480913A2890918A
:108E50003B28A0913C28B0913D287894BF93AF93D4
:108E60009F938F938DEC96E09F938F931F9287E74C
:108E70008F93C801029621E030E02C0F3D1F820F36
:108E8000931F9F938F930E946E8F080F191FC80125
:108E90000E94EC3F0FB6F894DEBF0FBECDBF892B0A
:108EA00009F01DC997CA2114310409F4A1CAF89424
:108EB00060913A2870913B2880913C2890913D2800
:108EC000C657DF4F688379838A839B83CA58D04013
:108ED000789480912A1B90912B1BA0912C1BB09110
:108EE0002D1BC657DF4F288139814A815B81CA58C3
:108EF000D040281B390B4A0B5B0BCA01B9010E94F9
:108F00007C856B017C01B10180E090E00E947C8552
:108F10009B01AC01C701B6010E94DF847C01FF9276
:108F20008F937F936F9388ED96E09F938F931F921B
:108F300087E78F939E01200F311F2D5F3F4F3F9397
:108F40002F93C956DF4F6883C759D040CA56DF4FA9
:108F50007883C659D0400E946E8F080F191FC956DA
:108F6000DF4F6881C759D040CA56DF4F7881C65954
:108F7000D040862F972FAE2DBF2D80934C289093F5
:108F80004D28A0934E28B0934F28C657DF4F4881F5
:108F900059816A817B81CA58D04040932A1B5093E3
:108FA0002B1B60932C1B70932D1B0FB6F894DEBF08
:108FB0000FBECDBF1DCA232809F428CAF89480919A
:108FC000011B9091021BA091031BB091041B78948C
:108FD0009F938F93809157028F93809156028F9326
:108FE00085EE96E09F938F931F9287E78F93C8013A
:108FF0000296A1E0B0E0AC0FBD1F8A0F9B1F9F93AC
:109000008F930E946E8F080F191F0FB6F894DEBF62
:109010000FBECDBFFBC98091D1239091D223A091E7
:10902000D323B091D423BF93AF939F938F9385EFB6
:1090300096E09F938F931F9287E78F93C8010296C4
:1090400021E030E02C0F3D1F820F931F9F938F93E1
:109050000E946E8F080F191FC8010E94EC3F0FB6C7
:10906000F894DEBF0FBECDBF892B09F038C8DCC92C
:109070008091C21B8F938091C11B8F938091C01BE5
:109080008F938091BF1B8F9380E097E09F938F9386
:109090001F9287E78F93C801029661E070E06C0F22
:1090A0007D1F860F971F9F938F930E946E8F080FCF
:1090B000191FC8010E94EC3F0FB6F894DEBF0FBE27
:1090C000CDBF892B11F00C946F40BFC98091462809
:1090D0008F93809145288F93809144288F9380911E
:1090E00043288F938BE097E09F938F931F9287E79E
:1090F0008F93C8010296E1E0F0E0EC0FFD1F8E0FA8
:109100009F1F9F938F930E946E8F080F191FC80196
:109110000E94EC3F0FB6F894DEBF0FBECDBF892B87
:1091200011F00C946F40A2C981E00E94020A2091C4
:1091300072023091730240917402509175020E9444
:109140005C879F938F937F936F9388E197E09F93C2
:109150008F931F9287E78F93C801029641E050E0FA
:109160004C0F5D1F840F951F9F938F930E946E8FEE
:10917000080F191FC8010E94EC3F0FB6F894DEBF1C
:109180000FBECDBF892B11F00C946F407DC982E0DA
:109190000E94020A20916E0230916F02409170028B
:1091A000509171020E945C879F938F937F936F937E
:1091B00085E297E09F938F931F9287E78F93C80173
:1091C0000296A1E0B0E0AC0FBD1F8A0F9B1F9F93DA
:1091D0008F930E946E8F080F191FC8010E94EC3FE9
:1091E0000FB6F894DEBF0FBECDBF892B11F00C94E3
:1091F0006F4058C983E00E94020A9F938F937F9328
:109200006F9382E397E09F938F931F9287E78F93EB
:10921000C801029621E030E02C0F3D1F820F931F02
:109220009F938F930E946E8F080F191F8C98C8010F
:109230000E94EC3F0FB6F894DEBF0FBECDBF892B66
:1092400011F00C946F403FC98091CB1F87FF49C933
:1092500021E042E161E080ED0E94E15D9F938F9308
:109260007F936F938FE397E09F938F931F9287E78E
:109270008F93C801029661E070E06C0F7D1F860F2E
:10928000971F9F938F930E946E8F080F191FC8011D
:109290000E94EC3F0FB6F894DEBF0FBECDBF892B06
:1092A00011F00C946F401DC98091CB1F87FF27C917
:1092B00021E042E162E080ED0E94E15D9F938F93A7
:1092C0007F936F938DE497E09F938F931F9287E72F
:1092D0008F93C8010296E1E0F0E0EC0FFD1F8E0FC6
:1092E0009F1F9F938F930E946E8F080F191FC801B5
:1092F0000E94EC3F0FB6F894DEBF0FBECDBF892BA6
:1093000011F00C946F40FBC88091CB1F87FF05C9FB
:1093100021E042E163E080ED0E94E15D9F938F9345
:109320007F936F938BE597E09F938F931F9287E7CF
:109330008F93C801029641E050E04C0F5D1F840FEF
:10934000951F9F938F930E946E8F080F191FC8015E
:109350000E94EC3F0FB6F894DEBF0FBECDBF892B45
:1093600011F00C946F40D9C88091CB1F87FFE3C8E0
:1093700021E042E164E080ED0E94E15D9F938F93E4
:109380007F936F9389E697E09F938F931F9287E770
:109390008F93C8010296A1E0B0E0AC0FBD1F8A0F09
:1093A0009B1F9F938F930E946E8F080F191FC801F8
:1093B0000E94EC3F0FB6F894DEBF0FBECDBF892BE5
:1093C00011F00C946F40B7C88091CB1F82FFC3C8C7
:1093D00046E061E083E00E94F712BDC88091CB1F98
:1093E00082FFC9C821E046E061E083E00E94F712F5
:1093F000C2C88091CB1F82FFCBC88091B91B8F93CD
:109400008091B81B8F938091B71B8F938091B61B6F
:109410008F9387E797E09F938F931F9287E78F93B0
:10942000C801029641E050E04C0F5D1F840F951F6C
:109430009F938F930E946E8F080F191FC8010E947F
:10944000EC3F0FB6F894DEBF0FBECDBF892B11F0F5
:109450000C946F409DC88091CB1F82FFA6C880915D
:10946000BD1B8F938091BC1B8F938091BB1B8F93EF
:109470008091BA1B8F938FE797E09F938F931F92F2
:1094800087E78F93C8010296A1E0B0E0AC0FBD1F43
:109490008A0F9B1F9F938F930E946E8F080F191F37
:1094A000C8010E94EC3F0FB6F894DEBF0FBECDBFDF
:1094B000892B11F00C946F4078C88091CB1F90914C
:1094C000CC1F90FF80C880E090E00E94FA1D9F931F
:1094D0008F937F936F938AE897E09F938F931F9268
:1094E00087E78F93C801029621E030E02C0F3D1FE3
:1094F000820F931F9F938F930E946E8F080F191FE7
:10950000C8010E94EC3F0FB6F894DEBF0FBECDBF7E
:10951000892B11F00C946F4056C88091CB1F90910D
:10952000CC1F90FF5EC881E090E00E94FA1D9F93DF
:109530008F937F936F938AE997E09F938F931F9206
:1095400087E78F93C801029661E070E06C0F7D1F82
:10955000860F971F9F938F930E946E8F080F191F7E
:10956000C8010E94EC3F0FB6F894DEBF0FBECDBF1E
:10957000892B11F00C946F4034C88091CB1F9091CF
:10958000CC1F90FF3CC881E090E00E94FA1D6B0167
:109590007C0180E090E00E94FA1D9B01AC01C701B4
:1095A000B6010E94F41B9F938F937F936F938BEA76
:1095B00097E09F938F931F9287E78F93C80102963E
:1095C000E1E0F0E0EC0FFD1F8E0F9F1F9F938F9344
:1095D0000E946E8F080F191FC8010E94EC3F0FB642
:1095E000F894DEBF0FBECDBF892B11F00C946F40F5
:1095F0000C94FF428091CB1F9091CC1F90FF0DC81F
:1096000081E090E00E94FA1D6B017C0180E090E017
:109610000E94FA1D9B01AC01C701B6010E94551CB6
:109620009F938F937F936F9386EB97E09F938F9396
:109630001F9287E78F93C801029641E050E04C0FDC
:109640005D1F840F951F9F938F930E946E8F080F4D
:10965000191FC8010E94EC3F0FB6F894DEBF0FBE81
:10966000CDBF892B11F00C946F400C940D43809169
:10967000CB1F9091CC1F90FD02C00C941C4381E045
:1096800090E00E94FA1D6B017C0180E090E00E9456
:10969000FA1D9B01AC01C701B6010E94B61C9F9345
:1096A0008F937F936F9384EC97E09F938F931F9298
:1096B00087E78F93C8010296A1E0B0E0AC0FBD1F11
:1096C0008A0F9B1F9F938F930E946E8F080F191F05
:1096D000C8010E94EC3F0FB6F894DEBF0FBECDBFAD
:1096E000892B11F00C946F400C941C438091CB1F7C
:1096F0009091CC1F91FD02C00C942B430E94411706
:109700009F938F937F936F9387ED97E09F938F93B2
:109710001F9287E78F93C801029621E030E02C0F5B
:109720003D1F820F931F9F938F930E946E8F080F90
:10973000191FC8010E94EC3F0FB6F894DEBF0FBEA0
:10974000CDBF892B11F00C946F400C942B43D501A5
:1097500016968C9116971F928F9315968C9115974C
:109760001F928F9313968C9113971F928F9312963B
:109770008C911F928F9388EE97E09F938F931F9207
:1097800087E78F93C8010296E1E0F0E0EC0FFD1F40
:109790008E0F9F1F9F938F930E946E8F080F191F2C
:1097A000C8010E94EC3F0FB6F894DEBF0FBECDBFDC
:1097B000892B11F00C946F400C943D4380917309F8
:1097C0009091740982FD0CC08091540280FD08C004
:1097D00081FD02C00C945C431D9902C00C945C4353
:1097E000FF92EF928FEF97E09F938F930E940B8FE2
:1097F00080916D020F900F900F900F90882311F4BD
:109800000C945C431F928F9383E69EE09F938F930B
:109810000E941D8F0F900F900F900F900C945C433F
:109820008BE899E00E945C53892B11F40C940E4450
:109830000E94FB638091540287FD02C00C946F402C
:109840002B9A0C946F40C856DF4F0FB6F894DEBFCA
:109850000FBECDBFDF91CF911F910F91FF90EF9081
:10986000DF90CF90BF90AF909F908F907F906F9040
:109870005F904F903F902F9008950C94224F4F92FD
:109880005F926F927F928F929F92AF92BF92CF9290
:10989000DF92EF92FF920F931F93CF93DF93CDB799
:1098A000DEB760970FB6F894DEBF0FBECDBF6B0179
:1098B0000E944165E82FF0E0EE0FFF1FE151F54EE9
:1098C0008081918101969183808380917309909129
:1098D000740981FD749880905402909055020E9402
:1098E0007C577C01FC018081982F92959F7091306C
:1098F00099F48F7051F48091D31A9091D41A0196F3
:109900009093D41A8093D31A00C1B60180E698E2EE
:109910000E94984E892B51F08091D11A9091D21AC1
:1099200001969093D21A8093D11AEFC0C40184E0BB
:10993000989F812D99271124F82FF1708F2E8AEA94
:1099400099E00E94A3518C01009709F448C0B60128
:10995000C80102960E94984E892BE9F198014CE3C8
:1099600059E060E074E6C8010F960E942354F701A5
:109970009181F8018481981321C082858F5F82874D
:109980008091CF1A9091D01A01969093D01A80931B
:10999000CF1A84E00E949958F801208530E02817FA
:1099A000390708F0A1C184E00E949958F801808726
:1099B000F70180818F70F8018187A7C0F8011286B6
:1099C00084E00E949958F8018087F70180818F70A8
:1099D000F80181878AC1C8010E944B52B4CF84E04C
:1099E00092E00E9438518C01009709F48EC0B601B4
:1099F000C80102960E948F4EF70181818150F801C3
:109A0000848380E091E0A0E0B0E083879487A5871D
:109A1000B687128684E00E949958F8018087F70182
:109A200080818F70F8018187B8018AEA99E00E94ED
:109A3000035298014CE359E060E074E6C8010F96C8
:109A40000E94235499249394F7018181F80184831F
:109A5000F70180818F70F801878384E00E94995814
:109A6000F801858383E00E9499585C01F8018683A0
:109A700087818F3009F0912CF7014180F8018481B2
:109A8000481A512C612C712C56E0440C551C661C54
:109A9000771C5A95D1F72385348545855685A0ECEA
:109AA000B0E00E943A88BB27A92F982F872F480E35
:109AB000591E6A1E7B1E4386548665867686809173
:109AC00073099091740981FD2AC08091540280FD30
:109AD00026C081FD22C0809154029091550297FDCD
:109AE000CEC0992091F082E08093E2231092E4238B
:109AF0001092E3231093E6230093E52342EE53E212
:109B000062E184E392E00E94B650809173099091E3
:109B1000740981FFECC0749AEAC01D9BDCCFA4E6F7
:109B2000B0E0A30192010E943A88672F782F892F15
:109B3000992724E630E040E050E00E9485887F933A
:109B40006F93452C562C672C77245F924F92BB2441
:109B5000BF92AF92F80185811F928F93F7018081A8
:109B60008F701F928F9381811F928F93F601818155
:109B70001F928F9380811F928F93C70102969F93AC
:109B80008F9387E198E09F938F930E940B8F809132
:109B90006D020FB6F894DEBF0FBECDBF882361F013
:109BA0001F928F9380E69EE09F938F930E941D8F5C
:109BB0000F900F900F900F9080915402909155024A
:109BC00096FF2DC0882059F1F7012081322F3F7078
:109BD000832F90E00297D4F08FEF830F207F822BAA
:109BE00080838FE999E00E943D4C8091CD1A90913D
:109BF000CE1A01969093CE1A8093CD1A8091730954
:109C00009091740996FF0BC0739809C08091D31A84
:109C10009091D41A01969093D41A8093D31A80917C
:109C2000CB1F86FF58CF0E94305DC70105960E946A
:109C3000FC5CF70181811F928F93F80186811F924E
:109C40008F9385811F928F938BE598E09F938F93DD
:109C50001F9280E18F939E012F5F3F4F6901DF923A
:109C60002F930E946E8F82E00E94165DC6010E94B3
:109C7000FC5C0FB6F894DEBF0FBECDBF2CCF8CEBD3
:109C80009AE12091BC1A222309F42BCF9F938F9342
:109C90008EE698E09F938F93FE0131966F01DF92DD
:109CA000EF930E94AB8F5C01B601C70102960E9440
:109CB000908E0F900F900F900F900F900F90009735
:109CC00009F40FCF95012F5F3F4F280F391FA901CE
:109CD0002F5F3F4FFA0180818032C9F362E18CE04F
:109CE00092E00E94B650FDCE812C912CADCE6096B4
:109CF0000FB6F894DEBF0FBECDBFDF91CF911F919D
:109D00000F91FF90EF90DF90CF90BF90AF909F901A
:109D10008F907F906F905F904F9008950895FB0112
:109D20002081FC012083FB012181FC012183089516
:109D3000FC019081DB018C91981309C081E090E0D7
:109D4000318111962C91321721F080E0089580E046
:109D500090E00895BC0180E698E20C948F4EDC01FF
:109D60001996ED91FC911A970280F381E02D3097BE
:109D700009F0099408950F931F93CF93DF9300D0B8
:109D8000CDB7DEB78C0188E10E94AC58BC01CE0192
:109D900001960E948F4ED8011996ED91FC911A9769
:109DA0000190F081E02DBE016F5F7F4FC8010995E2
:109DB0000F900F90DF91CF911F910F910895EF9227
:109DC000FF920F931F93CF93DF93EC018B017A01E6
:109DD0004CEF52E00E94084FFA86E98660E073E09B
:109DE000C801DF91CF911F910F91FF90EF900C94DC
:109DF000614F0C94204FCF93DF93EC0160E678E243
:109E000088E10E94A258CE01DF91CF910C94224F9D
:109E1000EF92FF920F931F93CF93DF93EC018B018F
:109E20007A010E943D4FF886EF8264E073E0C8013A
:109E3000DF91CF911F910F91FF90EF900C94614FA4
:109E40000C94454F0C94BD69DC011796ED91FC9183
:109E500018970190F081E02D0994DC011796ED919F
:109E6000FC9118970280F381E02D309709F0099456
:109E700008958EEA91E10C949F51FC0173836283F3
:109E8000BC018EEA91E10C940352BC018EEA91E18F
:109E90000C94E851CF93DF93EC018EEA91E10E949C
:109EA000A351009749F0FC01228133812C173D0713
:109EB00029F00E944B52F5CF80E090E0DF91CF91E6
:109EC00008950F931F93CF93DF938B010E944A4F06
:109ED000EC01009731F01D830C83C8010E94EE6BEA
:109EE0008E83DF91CF911F910F9108951F93CF9390
:109EF000DF93EC01162FEC81FD813097D1F0909328
:109F0000B1118093B01182E08887CE010696099541
:109F1000992787FD90950297029710F0133839F42E
:109F2000BE01CE01DF91CF911F910C94A34F81E030
:109F30008887DF91CF911F910895FC01208520FD36
:109F40000C94764F0895CF92DF92EF92FF920F9389
:109F50001F93CF93DF93EC016B01E090B011F09071
:109F6000B1110091B2111091B311F801EC17FD0776
:109F700039F0309709F44AC00190F081E02DF6CF16
:109F8000209709F443C08885882309F118860115B4
:109F9000110561F0C017D10729F0AE0167E8C801CB
:109FA0000E949D4FF80100811181F1CFEC81FD816C
:109FB000309769F0CC15DD0551F0D093B111C09305
:109FC000B01140E050E063E8CE0106960995E091BB
:109FD000B211F091B311CE17DF0769F4888199812E
:109FE0009093B3118093B2110DC0808191818C1731
:109FF0009D0721F0FC013097C1F704C08881998149
:10A0000091838083F092B111E092B011DF91CF91F2
:10A010001F910F91FF90EF90DF90CF9008951F93C5
:10A02000CF93DF931092BC11C091B211D091B311B4
:10A0300011E0209779F08985882341F018871986E7
:10A0400040E050E062E8CE010E94764F0990D8814E
:10A05000C02DEFCFDF91CF911F91089580915F12B6
:10A0600091E0980F90935F1208956091B0117091F4
:10A07000B1110C94A34F8AE880935F1210925D1285
:10A0800010925E121092B3111092B2111092B1118F
:10A090001092B01108958091BC1181110E940F504F
:10A0A00070915E12772309F451C0E0915D122E2F5A
:10A0B00030E085E0E89FF0011124E354FE4E60811A
:10A0C0006093BB11418152815093BA114093B911F1
:10A0D000838194819093B8118093B7112F5F3F4F84
:10A0E0002F71332720935D12715070935E12009789
:10A0F00031F58091B2119091B3119093B611809384
:10A10000B5118091B5119091B611892BF9F080911C
:10A11000BC1181110E940F504091B9115091BA1198
:10A120006091BB118091B5119091B6110E949D4F25
:10A13000E091B511F091B61180819181DECF613847
:10A1400019F421E0FC0120870E949D4F8091BC11F1
:10A1500020915E1290E0820F911D08958091BC11B4
:10A1600020915E1290E0820F911D089520915E1261
:10A170002032B9F0E0915D12E20FEF71E093B4117B
:10A1800035E0E39FF0011124E354FE4E60835283D7
:10A190004183948383832F5F20935E1280E090E05D
:10A1A000089581E090E00895CF93DF93C091B011BE
:10A1B000D091B1110E949D4FD093B111C093B011B5
:10A1C000DF91CF910895AB013091B2112091B3117D
:10A1D000E32FF22FE817F907B1F0309721F0019043
:10A1E000F081E02DF7CF009771F0FC0130832183DF
:10A1F0009093B3118093B21121E0208717821682C9
:10A2000061E80C94D4500895009749F0FC01208532
:10A210002150223020F421E021872093BC110895A1
:10A2200021E030E0FC018085811102C020E030E0B7
:10A23000C9010895CF93DF93EC014A815B8160E00F
:10A2400070E08C819D810E945F8E2A813B81888194
:10A250009981289FA001299F500D389F500D1124EE
:10A2600060E070E08E819F81DF91CF910C945F8ED2
:10A27000FC018281938120E030E028173907D1F07A
:10A28000A481B581A20FB31F4C91411110C081E090
:10A290008C9380819181289FA001299F500D389F28
:10A2A000500D112486819781840F951F08952F5F8B
:10A2B0003F4FE3CF80E090E00895FC012681378195
:10A2C0004281538180E090E084179507C9F02617FA
:10A2D000370781F4A481B581A80FB91F2C911216FC
:10A2E00014F421502C930480F581E02DE80FF91F20
:10A2F00080810895A081B1812A0F3B1F0196E4CF90
:10A300008FEF0895FC018681978168177907A0F087
:10A31000A081B18142815381A49F9001A59F300DFE
:10A32000B49F300D1124280F391F81E090E062178F
:10A33000730720F080E0089580E090E00895FC012C
:10A34000118210820895FC01808191810895FB01A2
:10A3500020813181FC01318320830895DC01ED915E
:10A36000FC91309731F080819181009729F0FC01B8
:10A37000FACF80E090E00895CF010895DC01ED91DF
:10A38000FC9111973097A9F020813181232B21F482
:10A390001D921C92CF010895A081B1818D919C9155
:10A3A0001197892B11F0FD01F7CF11821082CD0199
:10A3B000089580E090E00895DC01ED91FC91119703
:10A3C000309721F0208131812D933C93CF01089566
:10A3D000DC01ED91FC913097A9F0A0E0B0E0208184
:10A3E0003181E617F70741F4109709F4DC012D934A
:10A3F0003C931182108208952115310519F0DF0177
:10A40000F901EDCF08950F931F93CF93DF938C0144
:10A41000EB010E94E85119821882C8010E94AE51D6
:10A42000009711F4F80101C0FC01D183C083DF91D2
:10A43000CF911F910F9108950F931F93CF93DF93A7
:10A44000EC018B010E94E85188819981F801918388
:10A45000808319830883DF91CF911F910F91089515
:10A46000DC01ED91FC9180E090E0309729F00196BD
:10A470000190F081E02DF9CF0895FB01309719F498
:10A48000BA010C941C5280819181DA018D939C93C6
:10A49000518340830895009721F0FC0180819181D0
:10A4A000089580E090E00895809162129091631287
:10A4B000892B29F4109261121092601208950E9463
:10A4C0004861E0916212F0916312228133814081F0
:10A4D0005181240F351F281B390B0480F581E02D95
:10A4E000309769F04281538160817181460F571F17
:10A4F000481B590B4217530780F79A01EECF280FDC
:10A50000391F3093611220936012089580E892E021
:10A510000C940451EF92FF920F931F93CF93DF930C
:10A520008C01FC0180819181009799F08A35910519
:10A53000D9F0F8011182108283E068C0868197818A
:10A540008417950709F049C00480F581E02D309704
:10A55000A9F710926312109262128AE590E0F80156
:10A560009183808381E052C0673891F16238A9F706
:10A57000C0916212D0916312E12CF12C209769F303
:10A58000CE010E94BF6F892BF1F0AE0168E88E8189
:10A590009F810E94B650892BA1F41F821E828C815C
:10A5A0009D81E114F10421F0F7019583848304C0B7
:10A5B00090936312809362121D821C820E945452F7
:10A5C000D7CF0E9486527E010C80DD81C02DD6CF70
:10A5D000E0916212F0916312BACFF0936312E093AC
:10A5E0006212A481B581109709F4B7CF16968D91A8
:10A5F0009C9117978417950711F0FD01F2CF1496DF
:10A600008D919C91159795838483EBCFDF91CF91AA
:10A610001F910F91FF90EF900895CF93DF93EC017E
:10A620000E9486528E819F81309162122091631226
:10A63000892B59F0E32FF22F309739F0EC17FD07F3
:10A6400081F00480F581E02DF7CF8091B0119091D9
:10A65000B1119F838E833C832D83D0936312C0936B
:10A660006212DF91CF910C945452CF93DF93EC019F
:10A670000E949F6FCE01DF91CF910C940D53CF9329
:10A68000DF93EC010E94AB6FCE01DF91CF910C9470
:10A690000D53CF93DF93EC010E94B56FCE01DF9194
:10A6A000CF910C940D53FC0120813181260F371F6F
:10A6B000318320830C94545221E030E0FC018681E8
:10A6C0009781892B11F020E030E0C9010895FC0149
:10A6D0002281338180819181820F931F0895FC0133
:10A6E00080819181089581E090E020916212309103
:10A6F0006312232B11F480E090E0089580916212A0
:10A7000090916312892B29F08091601290916112CF
:10A71000089580E090E00895CF93DF93EC01E091FD
:10A720006212F09163128E179F0769F48C819D81EC
:10A7300090936312809362120DC0848195818C176F
:10A740009D0721F0FC013097C1F706C08C819D81E7
:10A75000958384830E9454521D821C821F821E8214
:10A76000DF91CF910895EF92FF920F931F93CF93B4
:10A77000DF938C017A01FC0180819181009741F087
:10A780008B34910501F1F8011182108283E048C0F9
:10A7900085E692E10E94A351EC01209751F06C8173
:10A7A0007D81CE0102960E9435530990D881C02D3B
:10A7B000F4CF81E0809364128BE490E0F801918300
:10A7C000808381E02DC06838E1F785E692E10E9440
:10A7D000A351EC01209781F3CE010296E816F90609
:10A7E000D9F4BE0185E692E10E94E851E090B011F3
:10A7F000F090B1118A859B859093B1118093B0112F
:10A80000EC85FD85309719F08E859F850995F0922E
:10A81000B111E092B011D0CF0990D881C02DDACF1C
:10A82000DF91CF911F910F91FF90EF9008951092BB
:10A83000641285E692E10E949F5160E070E08AE830
:10A8400092E00C94E3500F931F93CF93DF93EC01AE
:10A850000091B0111091B1111B870A875D874C8759
:10A860003F872E8780916412882379F08AE892E0EE
:10A870009093B1118093B011CE0102960E9435538E
:10A880001093B1110093B01102C07D836C83BE019F
:10A8900085E692E10E94E851BE0185E692E1DF91F2
:10A8A000CF911F910F910C9403520F931F93CF934D
:10A8B000DF93EC0180916412882391F00091B01134
:10A8C0001091B1118AE892E09093B1118093B01188
:10A8D000CE0102960E943F531093B1110093B01124
:10A8E000BE0185E692E10E94E851BE0185E692E153
:10A8F000DF91CF911F910F910C9403520F931F93EF
:10A90000CF93DF93EC0180916412882391F0009142
:10A91000B0111091B1118AE892E09093B111809337
:10A92000B011CE0102960E9449531093B1110093C9
:10A93000B011BE0185E692E10E94E851BE0185E6B4
:10A9400092E1DF91CF911F910F910C940352CF931D
:10A95000DF93EC0180916412882329F0CE010296E6
:10A960000E948C5304C01F821E8219861886BE0165
:10A9700085E692E1DF91CF910C94E851CF93DF937C
:10A98000EC0180916412882331F0CE010296DF91B0
:10A99000CF910C945C5385E692E10E94A3510097FD
:10A9A00039F08C179D0739F0FC0180819181F7CF38
:10A9B00081E090E002C080E090E0DF91CF910895C7
:10A9C0002F923F924F925F926F927F928F929F92BF
:10A9D000AF92BF92CF92DF92EF92FF920F931F93AD
:10A9E000CF93DF93CDB7DEB7E8970FB6F894DEBF0D
:10A9F0000FBECDBFE7E9FAE2208131814281538168
:10AA0000E3E9FAE25080418032802380EFE8FAE205
:10AA10008081898391819A83A281AB836380EBE8F3
:10AA2000FAE2B081BC8381818D8392819E83A38170
:10AA3000AF83E7E8FAE2B081B887818189879281A4
:10AA40009A87A381AB87E3E8FAE2B081BC87818172
:10AA50008D8792819E87A381AF87EFE7FAE2B0816D
:10AA6000B88B8181898B92819A8BA381AB8BEBE729
:10AA7000FAE2B081BC8B81818D8B92819E8BA38108
:10AA8000AF8BE7E7FAE2B081B88F8181898F92813D
:10AA90009A8FA381AB8FE3E7FAE2B081BC8F81810B
:10AAA0008D8F92819E8FA381AF8FEFE6FAE2B08106
:10AAB000B8A3818189A392819AA3A381ABA3EBE67A
:10AAC000FAE2B081BCA381818DA392819EA3A38170
:10AAD000AFA3E7E6FAE2B081B8A7818189A79281A6
:10AAE0009AA7A381ABA7E3E6FAE2B081BCA7818174
:10AAF0008DA792819EA7A381AFA7EFE5FAE2B0816F
:10AB0000B8AB818189AB92819AAB7380EBE5FAE2B5
:10AB1000B080A18092808380E7E5FAE2F080E18056
:10AB2000D280C380E3E5FAE2A081AFABB181B8AFD8
:10AB3000128103812BAB3CAB4DAB5EAB0E947661C7
:10AB40005EA95F934DA94F933CA93F932BA92F93E7
:10AB50002F923F924F925F926F922B812F932A8177
:10AB60002F9329812F932F812F932E812F932D8126
:10AB70002F932C812F932B852F932A852F93298513
:10AB80002F9328852F932F852F932E852F932D85F7
:10AB90002F932C852F932B892F932A892F932989E3
:10ABA0002F9328892F932F892F932E892F932D89C7
:10ABB0002F932C892F932B8D2F932A8D2F93298DB3
:10ABC0002F93288D2F932F8D2F932E8D2F932D8D97
:10ABD0002F932C8D2F932BA12F932AA12F9329A153
:10ABE0002F9328A12F932FA12F932EA12F932DA127
:10ABF0002F932CA12F932BA52F932AA52F9329A513
:10AC00002F9328A52F932FA52F932EA52F932DA5F6
:10AC10002F932CA52F937F922AA92F9329A92F93A5
:10AC200028A92F938F929F92AF92BF92CF92DF92DB
:10AC3000EF92FF920F931F9328AD2F932FA92F937D
:10AC40009F938F937F936F93A1E6B8E28C911F92AD
:10AC50008F93E0E6F8E280811F928F938BED9EE068
:10AC60009F938F930E941D8FE7ECFAE22081318140
:10AC700042815381E3ECFAE25080418032802380AC
:10AC8000E7EBFAE29080818072806380E3EBFAE286
:10AC90008081898391819A83A281AB83B381BC83B4
:10ACA000EFEAFAE280818D8391819E83A281AF8356
:10ACB000B381B887EBEAFAE28081898791819A872C
:10ACC000A281AB87B381BC87E7EAFAE280818D87F6
:10ACD00091819E87A281AF87B381B88BE3EAFAE2C4
:10ACE0008081898B91819A8BB280A380EFE9FAE20F
:10ACF000F080E180D280C380EBE9FAE2A081AB8BE7
:10AD0000B181BC8B128103810FB6F894DEBF0FBEF8
:10AD1000CDBF2BAB3CAB4DAB5EAB0E9476615EA969
:10AD20005F934DA94F933CA93F932BA92F932F924B
:10AD30003F924F925F926F927F928F929F922C815F
:10AD40002F932B812F932A812F9329812F9328854D
:10AD50002F932F812F932E812F932D812F932C852D
:10AD60002F932B852F932A852F9329852F9328891D
:10AD70002F932F852F932E852F932D852F93AF9271
:10AD8000BF922A892F9329892F93CF92DF92EF9236
:10AD9000FF920F931F932C892F932B892F939F93AF
:10ADA0008F937F936F93A1E6B8E28C911F928F935C
:10ADB000E0E6F8E280811F928F938CE69EE09F93FD
:10ADC0008F930E941D8F0FB6F894DEBF0FBECDBFCC
:10ADD000E8960FB6F894DEBF0FBECDBFDF91CF91DE
:10ADE0001F910F91FF90EF90DF90CF90BF90AF90A9
:10ADF0009F908F907F906F905F904F903F902F909B
:10AE0000089580E380931B130895CF93DF9360919F
:10AE10001B1370E0C0E3D0E0C61BD70B67597D4E13
:10AE2000AE010E94568ECE01DF91CF910895CF9250
:10AE3000DF92EF92FF920F931F93CF93DF937C01EA
:10AE4000C0901E13D0901F1360911B1370E0E60199
:10AE5000E096C61BD70BC138D105D8F400E310E04B
:10AE6000061B170B67597D4EA8010E94568E6091F4
:10AE700067127091681280911C1390911D13680FD6
:10AE8000791FA601C701800F911F0E94568ECE0127
:10AE900002C080E090E0DF91CF911F910F91FF9071
:10AEA000EF90DF90CF90089590911B13980F90939F
:10AEB0001B13089540911E1350911F1348175907F3
:10AEC00098F020911C1330911D13280F391F3093D7
:10AED0001D1320931C13481B590B50931F134093B1
:10AEE0001E1381E090E0089580E090E00895909333
:10AEF0001F1380931E13089580911C1390911D13AE
:10AF000087569D4E089580911B1390E087599D4E62
:10AF1000089581E090E020916712309168122959DC
:10AF2000324111F480E090E008950E948957892B06
:10AF300061F0609167127091681240911E135091F8
:10AF40001F1389E992E10C94568E20911C133091C5
:10AF50001D1321153105B9F080911E1390911F1317
:10AF6000C096E9E9F2E1AF01495652414817590745
:10AF700034F4DF01A20FB31F4C914193F4CF109230
:10AF80001D1310921C1308958091671290916812FE
:10AF9000089580911E1390911F13089590911B1393
:10AFA00080E3891B089520E380911B13281B809167
:10AFB0001E1390911F13820F911D08951F93CF931D
:10AFC000DF93EC0110911B13812F90E08C179D07EC
:10AFD0006CF00E94D3578C0F9D1F8138910530F47F
:10AFE0001C1B10931B1381E090E002C080E090E0F6
:10AFF000DF91CF911F910895CF93DF93EAE6F8E2B6
:10B000001192119288E2EA39F807D1F7C2E6D8E244
:10B010006AEF72E0CE010E948F4E229688E2CA3615
:10B02000D807B1F7DF91CF91089510921D131092B8
:10B030001C1310921F1310921E1380E380931B1396
:10B0400089E992E190936812809367120C94FC57FF
:10B05000EF92FF920F931F93CF93DF9300D0CDB762
:10B06000DEB78C0169837A830E9415586981E62EC8
:10B070007A81F72E81E8E816F10418F080E8E82ECE
:10B08000F12CA701B80180916712909168120E947B
:10B09000568EF0921F13E0921E13C7010F900F906F
:10B0A000DF91CF911F910F91FF90EF9008950F9333
:10B0B0001F93CF93DF938C01EB010E9415581093DF
:10B0C000681200936712D0931F13C0931E13DF9171
:10B0D000CF911F910F91089520E3EAE6F8E2DC0199
:10B0E00001900D922A95E1F788E0E2E6F8E2DB01B3
:10B0F00001900D928A95E1F7089520E3FC01AAE6FC
:10B10000B8E201900D922A95E1F788E0FB01A2E6F2
:10B11000B8E201900D928A95E1F70895E82FF0E0EA
:10B12000EE0FFF1FE659F74D7183608381E090E0D9
:10B130000895E82FF0E0EE0FFF1FE659F74D8081EC
:10B140009181089590E0880F991F8E5C974D0E9421
:10B150008F4E81E090E0089590E0880F991F8E5CFB
:10B16000974D08958115910511F00197F1F7089514
:10B17000E0919D28F0919E28908180919C288923C0
:10B180000895E0919A28F0919B28808190919C28C5
:10B19000892B8083E0919F28F091A0288081909155
:10B1A0009C28892B80830895E0919A28F0919B2810
:10B1B000908180919C28809589238083E0919F28AD
:10B1C000F091A028908180919C288095892380838C
:10B1D00008951F93CF93DF93E0919A28F0919B28D5
:10B1E000908180919C28809589238083E0919F287D
:10B1F000F091A028808190919C28892B80838FEBEF
:10B2000093E00E94B2581FB7F894E0919F28F09104
:10B21000A028908180919C2880958923808383E851
:10B2200090E00E94B258E0919D28F0919E28D08134
:10B23000C0919C281FBF78948BE393E00E94B25882
:10B24000E0919D28F0919E28908180919C289823E0
:10B2500019F08D2F8C2301C081E0DF91CF911F91D8
:10B2600008955093A02840939F2870939B28609343
:10B270009A2890939E2880939D2881E001C0880F92
:10B280002A95EAF780939C280C94E958CF93DF9392
:10B29000C82FDFB7F894E0919F28F091A028808113
:10B2A00090919C28892B808383E090E00E94B25883
:10B2B000CC2351F0E0919F28F091A02880819091BB
:10B2C0009C2890959823908387E190E00E94B25843
:10B2D000E0919D28F0919E28808190919C2889235F
:10B2E00009F4C0E089E590E00E94B258E0919F28FF
:10B2F000F091A028808190919C289095982390832C
:10B30000DFBF8BE390E00E94B2588C2FDF91CF918A
:10B310000895CF93DF93C82FD8E08C2F81700E94BF
:10B320004659C6958111C068D150B9F78C2FDF916D
:10B33000CF9108958FEF0C948959DF92EF92FF928D
:10B340000F931F93CF93DF93E82EEB010E94E958F0
:10B3500081112FC080EF0E948959F12C10E488EFF1
:10B36000D82ED10E81E00E944659082F81E00E941C
:10B370004659882319F0002361F01DC0011109C04E
:10B380001E1528F0888180FF04C0E11611F0F12E0F
:10B3900001E0802F0E94465998819695011190688E
:10B3A000988311501D11DECF21961111D8CF8F2D0A
:10B3B00003C08FEF01C08EEFDF91CF911F910F91EE
:10B3C000FF90EF90DF900895FF920F931F93CF931C
:10B3D000DF93F82EEB010E94E958209769F085E58C
:10B3E0000E9489598E01085F1F4F89910E948959D7
:10B3F000C017D107D1F703C08CEC0E9489598F2D5B
:10B40000DF91CF911F910F91FF900C9489590F9369
:10B410001F93CF93DF93DB01EC9111969C911197D1
:10B42000F0E0F92B803181F4BF016E7FE3E0660F1D
:10B43000771FEA95E1F716969C911697ECE0F0E0FD
:10B44000E91BF109E60FF71FF7FF07C091E0EA01DA
:10B450009883F195E195F10902C0EA0118828832DA
:10B4600079F414968C91982F9076903649F086FF57
:10B4700002C0EE7F05C085FF02C0EC7F01C0E87FFF
:10B48000CF0144E0969587954A95E1F7D9018C93D1
:10B49000EF70E801E88380E0DF91CF911F910F9179
:10B4A00008950F931F93CF93DF93EC018B01B801A5
:10B4B00088810E949D59888381508D3F30F4F80126
:10B4C0008081883211F0803191F7DF91CF911F9107
:10B4D0000F910895CF93DF93EC010E94E958BE01CC
:10B4E00084EB0E94E45981E00E944659C82F0E94D3
:10B4F000E95881E0C11101C080E0DF91CF9108954A
:10B500001F93CF93DF9300D0CDB7DEB7182F698399
:10B510007A830E94E9580E94B85869817A81882309
:10B5200041F084E40E94E459113029F00E94C1588E
:10B5300002C082E001C080E00F900F90DF91CF91B8
:10B540001F9108954F925F926F927F928F929F9278
:10B55000AF92BF92CF92DF92EF92FF920F931F9321
:10B56000CF93DF93CDB7DEB729970FB6F894DEBF40
:10B570000FBECDBF6C015B014A0189010E94E958F1
:10B58000B6018EEB0E94E459CE0101967C013E018A
:10B590009AE0690E711C27010E949A59F701819364
:10B5A0007F01E615F705C1F769E070E0C2010E946E
:10B5B0003074811109C09401A501B201F6018081A6
:10B5C0000E94075A80E001C083E029960FB6F894E4
:10B5D000DEBF0FBECDBFDF91CF911F910F91FF90C6
:10B5E000EF90DF90CF90BF90AF909F908F907F9023
:10B5F0006F905F904F9008955F926F927F928F92BD
:10B600009F92AF92BF92CF92DF92EF92FF920F93F1
:10B610001F93CF93DF93CDB7DEB729970FB6F8947A
:10B62000DEBF0FBECDBF582E6B015A01890160E00D
:10B6300070E08EEB0E94E459CE0101967C014E0130
:10B640009AE0890E911C37010E949A59F701819363
:10B650007F01E815F905C1F769E070E0C3010E94B8
:10B660003074811108C09501A601B301852D0E9497
:10B67000075A80E001C083E029960FB6F894DEBF38
:10B680000FBECDBFDF91CF911F910F91FF90EF9033
:10B69000DF90CF90BF90AF909F908F907F906F90F2
:10B6A0005F9008950F931F93CF93DF93CDB7DEB7CD
:10B6B00028970FB6F894DEBF0FBECDBF182F062F08
:10B6C00098E0E6E0F3E0DE01119601900D929A9584
:10B6D000E1F7242F332727FD309541E752E0249FDF
:10B6E000C001259F900D349F900D112464E670E0F9
:10B6F0000E947188CB0144E6049F800D911D1124A6
:10B70000FE013196AE01475F5F4F619170E02617F1
:10B71000370711F4019603C0E417F507B1F71123B9
:10B7200019F091958195910928960FB6F894DEBF8E
:10B730000FBECDBFDF91CF911F910F910895EF9272
:10B74000FF920F931F93CF93DF93CDB7DEB72B9765
:10B750000FB6F894DEBF0FBECDBFF82EE92E682FCE
:10B76000792F88E08F0D0E94805A882319F084E396
:10B7700091E243C066E471E48FE090E00E940A5CCD
:10B780008E01075F1F4F9801AE01465F5F4FBE01FC
:10B79000655F7F4F8F2D9E2D0E94A25A8111E7CFAA
:10B7A00088E0E6E0F3E0DE01119601900D928A95C3
:10B7B000E1F7498521E732E0429FC001439F900DA8
:10B7C000112464E670E00E9471888A8594E6899F5E
:10B7D000600D711D1124FE0131968191481303C043
:10B7E0006F5F7F4F03C0E017F107B9F78B858823A0
:10B7F00019F0719561957109CB012B960FB6F894EC
:10B80000DEBF0FBECDBFDF91CF911F910F91FF9093
:10B81000EF900895DC01CB0181159105A105B105DB
:10B8200029F081509040A040B040D9F7089510927F
:10B83000B90080E28093B800089594EA9093BC0028
:10B8400040EA56E861E070E09091BC0097FD0BC0C3
:10B850004150510961097109411551056105710591
:10B8600099F781E008959091B900987F983011F090
:10B870009031B9F78093BB0084E88093BC0080EAE4
:10B8800096E8A1E0B0E02091BC0027FD08C0019738
:10B89000A109B1090097A105B105A9F7E2CF8091EF
:10B8A000B900887F883111F08034D9F680E008959E
:10B8B00024EA34E844E92093BC009091BC0097FF4F
:10B8C000FCCF9091B900987F983011F0903199F7A2
:10B8D0008093BB003093BC009091BC0097FFFCCFDD
:10B8E0009091B900987F903211F0983539F44093D7
:10B8F000BC009091BC0094FDFCCFDDCF08950C946A
:10B900001D5C84E98093BC008091BC0084FDFCCF69
:10B9100008958093BB0084E88093BC008091BC00B4
:10B9200087FFFCCF9091B900987F81E0983209F4AD
:10B9300080E0089584EC8093BC008091BC0087FF78
:10B94000FCCF8091BB00089584E88093BC00809177
:10B95000BC0087FFFCCF8091BB000895E0E1DC01D3
:10B96000FD91CD01F0933F01E150C9F780913C0179
:10B970008F7D80933C0180913C01877F80933C01C7
:10B98000FB0180E1919190933E018150D9F7809124
:10B990003C01806880933C0180913D0180FFFCCF99
:10B9A0004051510980913C01806280933C0180911B
:10B9B0003C01877F80933C01141615069CF4FB0123
:10B9C00080E1919190933E018150D9F780913C01A3
:10B9D000806880933C0180913D0180FFFCCF405105
:10B9E0005109EACFF90180E190913E019193815094
:10B9F000D9F781E090E008950F931F93CF93DF93E1
:10BA0000EC018CE70E94585C8CE70E94895C8E01F7
:10BA1000005F1F4F89910E94895CC017D107D1F741
:10BA2000DF91CF911F910F910C94815C813019F4BB
:10BA300040E050E002C040EC50E060E070E08CE795
:10BA400090E00C942411813019F44EE050E002C0D3
:10BA500048E050E060E070E08CE790E00C94241146
:10BA600041E050E060E070E08CE790E00E9424113B
:10BA70006AE67AE080E090E00C940A5C48E350E0EB
:10BA800060E070E08CE790E00E94241149E350E010
:10BA900060E070E08CE790E00E94241144E150E007
:10BAA00060E070E08CE790E00E94241148E750E0ED
:10BAB00060E070E08CE790E00E9424114EE550E0D9
:10BAC00060E070E08CE790E00E9424114DE650E0C9
:10BAD00060E070E08CE790E00E9424116CE17AE174
:10BAE00086E090E00E940A5C4CE050E060E070E08C
:10BAF0008CE790E00E94241141E050E060E070E0AB
:10BB00008CE790E00E94241146E050E060E070E095
:10BB10008CE790E00E9424116AE67AE080E090E0F1
:10BB20000C940A5CCF93DF93CDB7DEB7A2970FB624
:10BB3000F894DEBF0FBECDBF81E1EFEEF8E0DE018D
:10BB4000529601900D928A95E1F781E1E0E0F9E0EB
:10BB5000DE01119601900D928A95E1F70E943E5DFB
:10BB6000CE0142960E94FC5C82E00E94165D6AE66D
:10BB70007AE080E090E00E940A5CCE0101960E948B
:10BB8000FC5C60E17EEA88E290E00E940A5C80E072
:10BB90000E94235D60E17EEA88E290E00E940A5CF8
:10BBA0004EE050E060E070E08CE790E00E942411ED
:10BBB000A2960FB6F894DEBF0FBECDBFDF91CF9136
:10BBC0000895CF92DF92EF92FF920F931F93CF933E
:10BBD000DF9300D01F92CDB7DEB7F82E042F122FBF
:10BBE000213031F0223031F0243031F0283031F082
:10BBF00090E005C091E003C092E001C093E00C30FA
:10BC000059F00E3011F4946007C0003111F49860BF
:10BC100003C0023109F49C60613059F0623011F4C4
:10BC2000906207C0633011F4906403C0643009F47B
:10BC300090669068692F70E023E030E0AE014F5FBE
:10BC40005F4F8F2D90E00E943B1169E07AE180E028
:10BC500090E00E940A5C8F2D8160F82E0E941D5C8E
:10BC60000E949A5C89830E949A5C8A83023119F44B
:10BC70000E949A5C8B830E949A5C87FDF1CF0E94A0
:10BC8000A45C0E94815C69E07AE180E090E00E941F
:10BC90000A5C8F2D0E941D5C0E949A5C89830E9421
:10BCA0009A5C8A83023119F40E94A45C8B830E94FF
:10BCB000A45C0E94815C39812A81023149F5832F7D
:10BCC00090E0A0E0B0E04B817727662731FF0EC0FF
:10BCD00030E0322F2227620F731F811D911D640FE8
:10BCE000711D811D911D8C6F9F6F0BC030E0322F35
:10BCF0002227620F731F811D911D640F711D811D0D
:10BD0000911D0E947E8520E83FEF4FEF57E420C051
:10BD1000632F70E0762F6627620F711D882777FDED
:10BD20008095982F0E947E850C3029F420E030EE1B
:10BD30004FEF54E40DC00E3029F420E038EF4FEF00
:10BD400055E406C0003131F420E03EEF4FEF56E4F9
:10BD50000E94DF842FE632E143E050E40E945C87DA
:10BD60006B017C01612F70E080E090E00E947E8595
:10BD70009B01AC01C701B6010E94DF840F900F90B8
:10BD80000F90DF91CF911F910F91FF90EF90DF9077
:10BD9000CF900895E6E4F1E08081208190813081A8
:10BDA000829586958695837022952F70822B832BA2
:10BDB00092959F70892B08950F931F93CF93DF93D4
:10BDC00000D0CDB7DEB746E06CE080E00E940C62A8
:10BDD00089E18093C4001092C50082E08093C00086
:10BDE00080E00E9497620E94386184B784B784B76C
:10BDF00084B784B7E1E2F1E322E432E431832083C3
:10BE00003A968DB79EB70A97E817F907B8F381E11C
:10BE100099E09F938F9388E290E19F938F930E9484
:10BE20001D8F0E9473700E943B5060E070E080E8BC
:10BE300092E00E94E3500E941754E0910E03F091AB
:10BE40000F0309950E94CA5E90E00E94AF70CE0178
:10BE500001960E946D600F900F900F900F908823B5
:10BE600041F088E090E19F938F930E941D8F0F9087
:10BE70000F90CE0101960E94AA4E0E947B608C0119
:10BE80000E947760AE014F5F5F4FB8010E9463650B
:10BE90000E94E75F0E9444650E947F600E949D6649
:10BEA0008BEF9FE09F938F930E941D8F8A811F923B
:10BEB0008F9307EF1FE01F930F930E941D8F8981BF
:10BEC0001F928F931F930F930E941D8F85EF9FE00A
:10BED0009F938F930E941D8F0E94B370E0914B033C
:10BEE000F0914C030995E0913D03F0913E030995D3
:10BEF000E0912403F091250309950E94A466182F70
:10BF00000E9441651F921F931F928F9380914A0355
:10BF10008F93809149038F9380913C038F938091FD
:10BF20003B038F938AED9FE09F938F930E941D8F19
:10BF3000E0915503F09156030FB6F894DEBF0FBEA3
:10BF4000CDBF309791F00995BC0180E890E00E9448
:10BF50005D887F936F9387EC9FE09F938F930E9400
:10BF60001D8F0F900F900F900F9085EC9FE09F9387
:10BF70008F930E941D8F60E070E086ED92E00E943A
:10BF8000E3508AEE92E00E94836F8DEB9FE09F93D7
:10BF90008F930E941D8F0F900F900F900F900F9016
:10BFA0000F90DF91CF911F910F9108957F936F9321
:10BFB0009F938F9387EB9FE09F938F930E941D8F9A
:10BFC0000F900F900F900F900F900F9008951F9368
:10BFD000CF93DF93CDB7DEB7A0970FB6F894DEBF4F
:10BFE0000FBECDBF87E590E00E948990182F282FC3
:10BFF00035EF380F303108F0982F9095291709F454
:10C0000061C083E490E19F938F930E941D8FE8E8C5
:10C01000F0E10F900F90DE01119684918D9331968F
:10C0200080E1E039F807C9F7F89448E050E063E7A9
:10C0300070E0CE0101960E948F90EAE7F0E1DE0108
:10C04000119684918D93319680E1E838F807C9F70D
:10C050004EE050E065E670E0CE0101960E948F90C0
:10C06000E0E7F0E1DE01119684918D93319680E155
:10C07000EA37F807C9F74AE050E06BE570E0CE0117
:10C0800001960E948F906DEC7BEA85E590E00E941E
:10C09000A79060E070E083E590E00E94A79060E0E8
:10C0A00082E590E00E94999060E070E089E590E080
:10C0B0000E94A7901AE16AE175EE87E590E00E9480
:10C0C000A7907894812FA0960FB6F894DEBF0FBE8C
:10C0D000CDBFDF91CF911F910895F89442E050E0D9
:10C0E00063E770E00E947190789480E0089585E5A0
:10C0F00090E00C94899083E590E00C94899082E51F
:10C1000090E00C9481904091AF285091B0286091BC
:10C11000B1287091B22890E0A0E0B0E0480F591F1C
:10C120006A1F7B1F4093AF285093B0286093B128BB
:10C130007093B2284091AB285091AC286091AD2803
:10C140007091AE28480F591F6A1F7B1F4093AB2880
:10C150005093AC286093AD287093AE2820914F2A5D
:10C160002223A1F04091A7285091A8286091A928E6
:10C170007091AA28480F591F6A1F7B1F4093A72858
:10C180005093A8286093A9287093AA2808951F9215
:10C190000F920FB60F9211240BB60F922F933F936D
:10C1A0004F935F936F937F938F939F93AF93BF93BF
:10C1B000EF93FF9380912213909123130196909314
:10C1C000231380932213809121138F5F8093211377
:10C1D0008038A9F4109221138091AF289091B02853
:10C1E000A091B128B091B2280196A11DB11D8093F4
:10C1F000AF289093B028A093B128B093B228809133
:10C200004F2A8823E1F0809120138F5F80932013C1
:10C210008038A9F4109220138091A7289091A82823
:10C22000A091A928B091AA280196A11DB11D8093C3
:10C23000A7289093A828A093A928B093AA280E9481
:10C240007353892B11F00E948652FF91EF91BF9199
:10C25000AF919F918F917F916F915F914F913F919E
:10C260002F910F900BBE0F900FBE0F901F9018953F
:10C27000F8941092B60016BC83EF87BD82E084BDAF
:10C2800094E095BD95B395BB80936E007894089526
:10C290008091221390912313209122133091231324
:10C2A00082179307A9F70895009751F022E330E031
:10C2B00000002150310921153105D1F70197F4CF44
:10C2C00008950F931F93CF93DF93EC010E94486171
:10C2D0008C010E944861801B910B8C179D07C8F34D
:10C2E000DF91CF911F910F91089508950F931F93A0
:10C2F0006091AF287091B0288091B1289091B228B8
:10C300000091AF281091B0282091B1283091B22827
:10C31000601771078207930759F71F910F910895CE
:10C320001F920F920FB60F9211241092AC020F9031
:10C330000FBE0F901F9018951F920F920FB60F927D
:10C3400011240BB60F922F933F934F935F936F93EC
:10C350007F938F939F93AF93BF93EF93FF93E0915E
:10C36000A202F091A3028081E091AD02F091AE02B1
:10C37000309709F00995FF91EF91BF91AF919F918F
:10C380008F917F916F915F914F913F912F910F907E
:10C390000BBE0F900FBE0F901F9018951F920F921B
:10C3A0000FB60F9211241092B9020F900FBE0F908A
:10C3B0001F9018951F920F920FB60F9211240BB673
:10C3C0000F922F933F934F935F936F937F938F932E
:10C3D0009F93AF93BF93EF93FF93E091AF02F091E0
:10C3E000B0028081E091BA02F091BB02309709F06F
:10C3F0000995FF91EF91BF91AF919F918F917F919F
:10C400006F915F914F913F912F910F900BBE0F90C5
:10C410000FBE0F901F9018959DE0899FF001112489
:10C42000EE55FD4FA281B3811C92A481B5816C931E
:10C43000A681B78188ED8C93A085B1854C93128637
:10C440001486138608959DE0899FF0011124EE550E
:10C45000FD4F81E08287A081B1816C933A96808103
:10C460008111FDCF08951F93CF93DF93182FEB0118
:10C47000FE016491662329F0812F0E942362219698
:10C48000F7CFDF91CF911F9108951F93CF93DF9343
:10C49000182FEB018881882369F08A3021F46DE040
:10C4A000812F0E94236269916D30A1F3812F0E9438
:10C4B0002362F0CFDF91CF911F910895CF93DF9347
:10C4C000CDB7DEB79E01285F3F4F4E815F8160E4AC
:10C4D00070E084E293E10E94DA8F64E273E18D817F
:10C4E0000E944562DF91CF910895CF93C82F8A3083
:10C4F00031F46DE0809164130E94236202C08D309C
:10C5000029F06C2F809164130E94236280E090E0F8
:10C51000CF9108959DE0899FF0011124EE55FD4FC4
:10C52000748763870895682F80E00C94236280935A
:10C53000641384E992E090931C3180931B31089539
:10C5400084B7877F84BF88E10FB6F894809360003A
:10C55000109260000FBE08952FE088E190E00FB6C2
:10C56000F894A895809360000FBE20936000089512
:10C57000A895089588E10FB6F89480936000109212
:10C5800060000FBE0895F89428E088E190E00FB6AF
:10C59000F894A895809360000FBE20936000FFCFB1
:10C5A0008091BA288091BA2890E0089540E06FE128
:10C5B00081E491E00C943968E9E3F1E080818081C5
:10C5C0008D7F80838DE090E00197F1F723E040E0DC
:10C5D0006FE182E491E00E94436883E090E001977C
:10C5E000F1F708959091390191FD0AC0282F80310B
:10C5F00008F02FE040E06FE085E491E00C944368A0
:10C6000008958091390181FD0EC040E06FE181E421
:10C6100091E00E943968282F2F7E81E090E0213040
:10C6200021F080E0089580E090E008958091390144
:10C6300081FD10C040E06FE181E491E00E94396823
:10C640008F3131F0982F9F7E915081E0923018F415
:10C6500080E0089581E008950E9416638823E1F345
:10C660000895CF93DF93C82F0E942C630E94D66257
:10C67000D82FC81789F1C83019F40E94DC6225C090
:10C68000C93121F4863189F429E005C0C63169F445
:10C69000893159F426E040E06FE182E491E00E94A4
:10C6A0004368E3E0F0E03197F1F72C2F40E06FE1D1
:10C6B00082E491E00E944368D83019F4E9E6F1E0A1
:10C6C00002C0E3E0F0E03197F1F70E94D6628C17E8
:10C6D00019F083E490E002C080E490E0DF91CF9114
:10C6E00008950E942C6310924F2A0E94DC62809170
:10C6F00039018260809339018091D22A8823D9F14F
:10C7000080919400909195004091E32A5091E42A01
:10C7100084179507A0F48091AF2A9091B02AA09138
:10C72000B12AB091B22A8C57914EAF4FBF4F809330
:10C73000AF2A9093B02AA093B12AB093B22A209145
:10C74000940030919500241B350B8091AF2A909175
:10C75000B02AA091B12AB091B22A820F931FA11DD5
:10C76000B11D8093AF2A9093B02AA093B12AB093C1
:10C77000B22A1092D22A8091D42A8823D9F18091AA
:10C780009400909195004091E72A5091E82A8417EF
:10C790009507A0F48091B72A9091B82AA091B92A60
:10C7A000B091BA2A8C57914EAF4FBF4F8093B72AA2
:10C7B0009093B82AA093B92AB093BA2A20919400F2
:10C7C00030919500241B350B8091B72A9091B82A9F
:10C7D000A091B92AB091BA2A820F931FA11DB11D51
:10C7E0008093B72A9093B82AA093B92AB093BA2A13
:10C7F0001092D42A089580914F2A882381F0809145
:10C80000E813811104C00E941663811106C081E003
:10C810008093E61381E090E008950E94716380E0C8
:10C8200090E0089580919400909195009093E82A6B
:10C830008093E72A21E02093D42A8091390181FD59
:10C8400008C08091390181FD1AC086E10E943163E0
:10C8500016C020934E2A8091940090919500909359
:10C86000E42A8093E32A2093D22A809139018D7F94
:10C870008093390180914E2A8111FCCFE2CF81E073
:10C8800080934F2A089580914F2A81110AC0809188
:10C89000E813882321F081E08093E71302C00E940F
:10C8A000126481E090E008951F93CF93DF931F926D
:10C8B000CDB7DEB78FB789838091E813811126C089
:10C8C000F89480914F2A882351F08091390181FD9D
:10C8D0001BC00E9416638823B9F080E003C00E9449
:10C8E000436481E02091470191E02E3008F090E010
:10C8F000192F119581110E94FB63107429F0898111
:10C900008FBF81E090E004C089818FBF80E090E01C
:10C910000F90DF91CF911F9108958091E7138823A5
:10C9200021F00E9412641092E7138091E61388238D
:10C9300021F00E9471631092E6131092E81308959B
:10C940000F931F93AB0121E02093E8130091932AEA
:10C950001091942A2091952A3091962A0F5F1F4FAB
:10C960002F4F3F4F0093932A1093942A2093952A98
:10C970003093962A22E0260F27FF0CC080914C2A84
:10C9800090914D2A019690934D2A80934C2A0FEF57
:10C990001FEF07C0BC0185E693E10E94568E00E0C0
:10C9A00010E00E948D64C8011F910F91089580933B
:10C9B000EA1308950E94D662823011F0823111F498
:10C9C00080E0089581E0089508958FEF80934E01EF
:10C9D00022E044E060EF8CE691E00E94436825E0AD
:10C9E00041E06EE08CE290E00E94436880E8809332
:10C9F0006F018091460180936D0121E045E060E286
:10CA000084E491E00C9443688DEF93E00197F1F793
:10CA10000E942F681092C328109245291092C729AE
:10CA20001092C2281092C128E9E3F1E080818E7F44
:10CA3000808380818D7F80838DE090E00197F1F786
:10CA4000E9E3F1E080818160808323E040E06FE1F1
:10CA500082E491E00E9443688DEF93E00197F1F743
:10CA600080915D0180915E010E94E56460E070E06C
:10CA70008CEB92E00E94E3500E94126481E090E00F
:10CA800008958091E9130895CF93DF931F92CDB756
:10CA9000DEB789830E942C6389818093E913282F54
:10CAA00040E06FE188E491E00F90DF91CF910C942A
:10CAB00043680E9444658091390181FD03C086E08E
:10CAC0000C9431630895FA0180936201909363019D
:10CAD00060936001709361013097C1F08081809311
:10CAE0006B01818180936A018281809369018381D6
:10CAF00080936801848180936701858180936601BA
:10CB000086818093650187818093640108958CEB11
:10CB100092E00E94045181E08093BA288091BB2862
:10CB20009091BC2801969093BC288093BB2881E00B
:10CB300090E008958091C22892E8899FF001112425
:10CB4000ED53F74D10828F5F833018F48093C22825
:10CB500002C01092C228E091C22882E8E89FF0014A
:10CB60001124ED53F74D808181110C94876510924B
:10CB7000BA2808951F93CF93DF932091C22812E81B
:10CB8000129F90011124D901AD53B74D4C91411121
:10CB900003C00E949A6593C05091390151FD8FC026
:10CBA00050914F2A552309F48AC047FF16C00E94AE
:10CBB0009A658091832A9091842AA091852AB091C8
:10CBC000862A0196A11DB11D8093832A9093842A01
:10CBD000A093852AB093862A72C04330B0F40E9495
:10CBE0009A6580917F2A9091802AA091812AB091A4
:10CBF000822A0196A11DB11D80937F2A9093802ADD
:10CC0000A093812AB093822A5AC050E0EA01229769
:10CC10006C177D07B0F40E949A6580917B2A9091F1
:10CC20007C2AA0917D2AB0917E2A0196A11DB11D7A
:10CC300080937B2A90937C2AA0937D2AB0937E2AAE
:10CC40003EC0B9016C53774D0E94568EE091C228C8
:10CC50001E9FF0011124ED5BF64D80818093B32877
:10CC60000E949A65809147018093B4289091B928D9
:10CC7000992311F0891710F48093B9286091B42892
:10CC800070E084E00E948E586091B32870E083E0E9
:10CC90000E948E584091972A5091982A6091992A23
:10CCA00070919A2A4F5F5F4F6F4F7F4F4093972A43
:10CCB0005093982A6093992A70939A2A02C0C0E0F0
:10CCC000D0E0CE01DF91CF911F910895CF93DF93F4
:10CCD000EC01888199810097E9F08730954021F037
:10CCE0001982188283E026C06238C1F41092BA28F3
:10CCF0000E9415580E947C5760E870E00E94BA6557
:10CD0000181619066CF40E947757E0914F03F091C2
:10CD10005003099587E095E09983888381E00AC0F4
:10CD20008091B7289091B82801969093B828809365
:10CD3000B728F0CFDF91CF91089591E09093E81359
:10CD40000E94F2620C948D648091390181FD06C0CD
:10CD500040E06FE085E491E00C94396880E108954B
:10CD60000F931F93CF93DF93182F21E02093E813A5
:10CD700000914F2A8091390181FF16C08091940063
:10CD8000909195009093E42A8093E32A2093D22AED
:10CD900020934E2A809139018D7F809339018091B3
:10CDA0004E2A8111FCCF00E00E942C6380914F2A13
:10CDB000882309F43FC08091D42A8823D9F1809137
:10CDC000940090919500E091E72AF091E82A8E175F
:10CDD0009F07A0F44091B72A5091B82A6091B92AD0
:10CDE0007091BA2A4C57514E6F4F7F4F4093B72ADC
:10CDF0005093B82A6093B92A7093BA2A209194006C
:10CE0000309195002E1B3F0B4091B72A5091B82AC4
:10CE10006091B92A7091BA2A420F531F611D711D8A
:10CE20004093B72A5093B82A6093B92A7093BA2ACC
:10CE30001092D42A8091390181FD03C089E10E94BA
:10CE4000316386E00E949958892B51F00E94A466B4
:10CE5000C82F86E00E94995881500E94F26202C059
:10CE6000C0E0D0E020919400309195003093E62A04
:10CE70002093E52A81E08093D32AF89480913901A8
:10CE8000826080933901809139018D7F80933901CF
:10CE900062E0610F85E693E10E94746878942091C6
:10CEA000492A30914A2A2F5F3F4F30934A2A2093D4
:10CEB000492A0E942C6345E060EE82E491E00E94E2
:10CEC0003968182F86E00E949958892B19F08C2F09
:10CED0000E94F262002319F00E94126402C00E94B4
:10CEE00071638091D32A8823D9F180919400909125
:10CEF0009500E091E52AF091E62A8E179F07A0F4AD
:10CF00004091B32A5091B42A6091B52A7091B62A03
:10CF10004C57514E6F4F7F4F4093B32A5093B42AD2
:10CF20006093B52A7093B62A2091940030919500B1
:10CF30002E1B3F0B4091B32A5091B42A6091B52A21
:10CF40007091B62A420F531F611D711D4093B32A81
:10CF50005093B42A6093B52A7093B62A1092D32ABC
:10CF600080914F2A882361F02091940030919500A0
:10CF70003093E82A2093E72A81E08093D42A07C0DF
:10CF800023E040E06FE182E491E00E9443680E9468
:10CF90008D641130E9F01330A9F480918B2A9091BF
:10CFA0008C2AA0918D2AB0918E2A0196A11DB11DC7
:10CFB00080938B2A90938C2AA0938D2AB0938E2AEB
:10CFC00012E009C0153031F0173029F411E003C028
:10CFD00010E001C013E0812F90E0DF91CF911F910D
:10CFE0000F910895CF93DF93EB010E94A064009707
:10CFF00029F4CE010E94B066009751F020914C2A8E
:10D0000030914D2A2F5F3F4F30934D2A20934C2A69
:10D01000DF91CF910895CF93DF9380914F2A8111B3
:10D0200004C00E944364D1E001C0D0E00E94D662F7
:10D03000863111F0813119F4C091470109C040E0F7
:10D040006FE186E491E00E943968C82FCC0FC80FC9
:10D05000D1110E94FB638C2FDF91CF910895109224
:10D06000EC131092EB13EFE6F0E080818062808396
:10D070000895FC018081862390E002C095958795F4
:10D080004A95E2F70895F894FC015081362F3095C7
:10D090005323042E01C0220F0A94EAF72623522BB1
:10D0A00050837894089540917B01FC014193A0E85E
:10D0B000B1E050E8540F9D012F5F3F4F6C91619399
:10D0C000521711F0D901F7CF4150E42FF0E0E058AA
:10D0D000FE4F2181FC01E058FF4F2083FC01EF57F8
:10D0E000FF4F21E02083089560938001E1E8F1E0A3
:10D0F00061589F012F5F3F4FDC014D91CD0140836F
:10D10000621711F0F901F5CF08951F920F920FB633
:10D110000F9211240BB60F922F933F934F935F936F
:10D120006F937F938F939F93AF93BF93EF93FF93EF
:10D13000809147018093B4288091C12822E8829F82
:10D14000C00111248D53974D0E9453688091C128CE
:10D150008F5F833018F48093C12802C01092C128D9
:10D160000E948765FF91EF91BF91AF919F918F9141
:10D170007F916F915F914F913F912F910F900BBED7
:10D180000F900FBE0F901F9018951F920F920FB621
:10D190000F9211240F900FBE0F901F9018951F92A1
:10D1A0000F920FB60F9211240F900FBE0F901F9089
:10D1B00018951F920F920FB60F9211240F900FBE69
:10D1C0000F901F9018951F920F920FB60F92112477
:10D1D00010924E2A0F900FBE0F901F9018951F921D
:10D1E0000F920FB60F92112410924E2A0F900FBE7D
:10D1F0000F901F9018951F920F920FB60F92112447
:10D200008F9381E08093BA288F910F900FBE0F907B
:10D210001F9018951F920F920FB60F921124109223
:10D220004E2A0F900FBE0F901F9018951F920F92CD
:10D230000FB60F9211248F939F938091EB139091CF
:10D24000EC1301969093EC138093EB139F918F91C5
:10D250000F900FBE0F901F901895CF92DF92EF9214
:10D26000FF920F931F93CF93DF937C018B016A0191
:10D270008DEE93E10E94A351EC01009751F0EC81F7
:10D28000FD81309711F0C8010995CE010E944B52E3
:10D29000F3CFA601B801C701DF91CF911F910F9184
:10D2A000FF90EF90DF90CF900C942D4F0F931F9332
:10D2B000CF93DF9300D0CDB7DEB78091572A9091FE
:10D2C000582AA091592AB0915A2A0196A11DB11D40
:10D2D0008093572A9093582AA093592AB0935A2A98
:10D2E0000E94C06B8C018DEE93E10E94A3510097C8
:10D2F00079F0DC011296ED91FC911397309729F0AB
:10D3000089839A8309959A8189810E944B52EFCF34
:10D310000115110549F0C8010F900F90DF91CF91D1
:10D320001F910F910C94244F0F900F90DF91CF918C
:10D330001F910F9108950E94B3700E9415580E948A
:10D34000E7698BE393E09093522A8093512A0E94DD
:10D35000BE6B2FEF31E040E05EE160E074E082E020
:10D3600090E00C94876BBC018DEE93E10C9403521A
:10D37000BC018DEE93E10C94E851CF93DF93EC0167
:10D380004091532A5091542A6091552A7091562AFF
:10D390004F5F5F4F6F4F7F4F4093532A5093542AF4
:10D3A0006093552A7093562A0E94D36B009761F0C0
:10D3B0000E949557E0913F03F0914003BE018DE23A
:10D3C00099E6099581E090E0DF91CF91089583EF90
:10D3D00093E10C949F510F93CF93DF93EC017B83E8
:10D3E0006A8318865F834E83BC0183EF93E10E94BA
:10D3F0000352E091EF13F091F013309749F04C8114
:10D400005D8101E020E030E068858A819B8109959B
:10D41000DF91CF910F910895BC0183EF93E10C94BC
:10D42000E8510F93DC0118961C921897E091EF13C6
:10D43000F091F013309759F000E020E030E040E048
:10D4400050E060E012968D919C91139709950F9191
:10D4500008950F93DC01AB0114962D913C91159723
:10D4600081E018968C93189715967C936E93149779
:10D47000E091EF13F091F013309739F000E061E0A4
:10D4800012968D919C91139709950F9108950F9382
:10D49000DC01E091EF13F091F013309771F01496E6
:10D4A0004D915C91159701E09A0118966C9118972F
:10D4B00012968D919C91139709950F910895E09183
:10D4C000F113F091F213309709F0099408959093B5
:10D4D000F2138093F11308959093F0138093EF1358
:10D4E000089583EF93E10C94A351EF92FF920F9371
:10D4F0001F93CF93DF938C01EB017A0183EF93E1CC
:10D500000E94A3510097D9F0DC0112962D913C9115
:10D5100013972C173D0781F41696ED91FC91179700
:10D52000309769F09701AE01B801DF91CF911F915B
:10D530000F91FF90EF9009940E944B52E3CFDF913F
:10D54000CF911F910F91FF90EF9008950895CF9381
:10D55000DF93C6E2D4E16881798120E030E046ECD7
:10D560005AE680E194E10E9423540E94B1706881E0
:10D5700079810E945D8820E030E04AED5AE6BC01E6
:10D5800080E094E1DF91CF910C9423548091261494
:10D59000909127142091241430912514880F991FFD
:10D5A0002817390708F4C90190932714809326148B
:10D5B0000C94A76ACF93DF930E9415580E947C5762
:10D5C000EC01198218820E94716A288139810097C2
:10D5D00019F1FC0140854423F9F0FC01428153819B
:10D5E000F901EE0FFF1FEE0FFF1FEC0FFD1F53831E
:10D5F0004283FC01448155812F5F3F4FF901EE0FBB
:10D60000FF1FEE0FFF1FEC0FFD1F51834083398377
:10D6100028830E944B52D9CFC901880F991F880FC8
:10D62000991F02960E94775788819981892B31F042
:10D6300085EF93E1DF91CF910C94FB4EDF91CF9179
:10D640000895AF92BF92CF92DF92EF92FF920F9325
:10D650001F93CF93DF9300D0CDB7DEB76B010E944D
:10D660007C57FC01008111811A8309830C3011055C
:10D6700018F4E12CF12C0DC01F930F938FE299E069
:10D680009F938F930E940B8F0F900F900F900F908E
:10D6900021C0E016F106F1F00E947C57F701EE0F71
:10D6A000FF1FEE0FFF1FE80FF91FA280B3800E943B
:10D6B0007C57FFEFEF1AFF0AF701EE0FFF1FEE0F87
:10D6C000FF1FE80FF91F40815181B501C6010E947B
:10D6D000756ADFCF0F900F90DF91CF911F910F915F
:10D6E000FF90EF90DF90CF90BF90AF9008950F9391
:10D6F000013059F4809120149091211490932714B3
:10D70000809326140F910C94A76A0F910895EF92BD
:10D71000FF920F931F93CF93DF938B01EA0179015F
:10D7200048E253E0BC0185EF93E10E94DF4E109385
:10D73000211400932014D0932314C0932214F09248
:10D740002514E092241487E79BE6DF91CF911F9187
:10D750000F91FF90EF900C946C6A80E194E10E942D
:10D76000A75480E094E10E94A75485EF93E10C94C4
:10D77000F94E809126149091271408950C94394FF6
:10D78000CF93DF93E0912C03F0912D030995EC01E9
:10D79000009729F06A817B8181E00E948E58CE013A
:10D7A000DF91CF9108950F931F93CF93DF93EC01F7
:10D7B000E0912E03F0912F0309958C016A817B8102
:10D7C00081E00E948E5881E090E0012B11F480E00E
:10D7D00090E0DF91CF911F910F910895E091300378
:10D7E000F0913103099420E030E00296FC01329779
:10D7F0004081442331F0FC0131974081240F311DD9
:10D80000F4CFC9010895FC01208130E0322F222796
:10D810008181282B02C0220F331F6A95E2F7832FE4
:10D820009927FA01EE5CFC4F208130E0822393239C
:10D8300028E030E0241B350B02C0969587952A9589
:10D84000E2F708956F927F928F929F92AF92BF926C
:10D85000CF92DF92EF92FF920F931F93CF93DF93BC
:10D860008C01EB016A0179012830310524F4A9010A
:10D87000B601CE014AC0590123E0B594A7942A9578
:10D88000E1F74115510521F04801612C712C03C0CD
:10D89000D801FB0120C048E050E0B601CE01860D62
:10D8A000971D0E94036CF40181934F01FFEF6F1AE3
:10D8B0007F0A6A147B047CF3C501B7FE02C080E0D6
:10D8C00090E0A701477055274115510511F1080F48
:10D8D000191FB60118C0CF018C1B9D0B8A159B0523
:10D8E0001CF481918D93F7CFC501B7FE02C080E093
:10D8F00090E0A701477055274115510551F0080FD9
:10D90000191F60E070E08C0F9D1F0E94036CF801EE
:10D910008083DF91CF911F910F91FF90EF90DF9067
:10D92000CF90BF90AF909F908F907F906F90089511
:10D930008F929F92AF92BF92CF92DF92EF92FF921F
:10D940000F931F93CF93DF9300D0CDB7DEB70E9424
:10D950007C578C0182E090E00E945A57892B19F481
:10D9600080E090E05DC0F801818190E0982F8827E9
:10D970002081820F911D0E944A4F7C01009781F304
:10D980000E947C574C01F7012681822F869586954F
:10D99000869590E0422F477021E030E011F420E0BE
:10D9A00030E0820F931F0E945A57892BC9F2F7016A
:10D9B00004811581C12CD12CF8018081882379F153
:10D9C000F801A180B12CB60133E0759567953A95C1
:10D9D000E1F7A60147705527680D791D883168F079
:10D9E0009501CE0101960E94226CBE016F5F7F4FB0
:10D9F000F80180810E94A2580DC01A8219829501F7
:10DA0000CE0101960E94226C69817A81F8018081A1
:10DA10000E948E58CA0CDB1C0E5F1F4FCDCFC70172
:10DA20000F900F90DF91CF911F910F91FF90EF908A
:10DA3000DF90CF90BF90AF909F908F900895DC01C2
:10DA400050E0E0E1F0E0E61BF70BE21BF30B02C055
:10DA5000440F551FEA95E2F78C91852B8C93119614
:10DA60008C911197842B11968C9308956F927F92CD
:10DA70008F929F92AF92BF92CF92DF92EF92FF92DE
:10DA80000F931F93CF93DF938C016B01EA01790110
:10DA9000283031051CF44881C8015CC0390153E0CD
:10DAA000759467945A95E1F76115710521F04E015F
:10DAB000A12CB12C03C0D801FE0127C0F401419173
:10DAC0004F0128E030E0B601C8018A0D9B1D0E947D
:10DAD0001F6DFFEFAF1ABF0AA614B7047CF3C30192
:10DAE00077FE02C080E090E0970127703327211570
:10DAF000310509F43FC0C80FD91F488150E0B60175
:10DB0000621B730B685F7F4F1CC0CF018C1B9D0B8A
:10DB1000861597051CF481918D93F7CFC30177FE8D
:10DB200002C080E090E0970127703327211531056E
:10DB300009F1C80FD91F488150E068E070E0621B0E
:10DB4000730B02C0559547956A95E2F760E070E067
:10DB5000800F911FDF91CF911F910F91FF90EF9058
:10DB6000DF90CF90BF90AF909F908F907F906F90FD
:10DB70000C941F6DDF91CF911F910F91FF90EF904B
:10DB8000DF90CF90BF90AF909F908F907F906F90DD
:10DB900008956F927F928F929F92AF92BF92CF9291
:10DBA000DF92EF92FF920F931F93CF93DF9300D0FA
:10DBB000CDB7DEB78C01FC018681E82EE694E694B1
:10DBC000E694F12C282F277081E090E011F480E09A
:10DBD00090E0E80EF91EC70102960E94DE570097FA
:10DBE00009F445C00E948357F8012281FC0120837B
:10DBF000F8012381FC0121830E94835702965C0176
:10DC0000A70160E070E00E945F8EF8010481158139
:10DC1000E12CF12CF8018081882339F1F801818011
:10DC2000912C670163E0D594C7946A95E1F73701B9
:10DC3000F7E06F227724CA0CDB1C883128F00E94A1
:10DC4000AC589401AC0108C00E9499589A8389830A
:10DC50009401AE014F5F5F4FB301C6010E94366D64
:10DC6000E80CF91C0E5F1F4FD5CF81E090E00F90BC
:10DC70000F90DF91CF911F910F91FF90EF90DF9068
:10DC8000CF90BF90AF909F908F907F906F900895AE
:10DC9000E0914D03F0914E030994E0912603F09139
:10DCA00027030994E0915103F09152030994E09104
:10DCB0005303F0915403099480E090E0089508958F
:10DCC000E0911E03F0911F03099480E090E0089515
:10DCD0000F931F93CF93DF93CDB7DEB7E0970FB6C7
:10DCE000F894DEBF0FBECDBF0E94C9578C010E94C1
:10DCF0007C57AE014F5F5F4F602F0E9438768823BC
:10DD000009F446C088A99801281B3109C9010E945D
:10DD10005A57892BE9F12E8121110CC0BE016A5E90
:10DD20007F4F88E10E94A258E0914103F0914203A5
:10DD300009952EC08A859B858D3C3BEA930711F09F
:10DD4000019631F5223019F088E090E002C082E0BF
:10DD500090E001979C012F5F3F4F12161306F4F6D7
:10DD6000E1E0F0E0EC0FFD1FE80FF91F23852F3FE6
:10DD700081F3BE01645F7F4F89E10E94A25889E16F
:10DD80000E94AC5860E678E20E94984E892B31F6EA
:10DD9000E0960FB6F894DEBF0FBECDBFDF91CF91F6
:10DDA0001F910F910895AF92BF92CF92DF92EF92A1
:10DDB000FF920F931F93CF93DF93CDB7DEB7E0971A
:10DDC0000FB6F894DEBF0FBECDBF8C016B01CE0144
:10DDD00001967C0180E3F70111928A95E9F781E0D1
:10DDE00089838CE00E9499588C831D821F828091C8
:10DDF0002A1491E0980F90932A14898783E0B82E13
:10DE0000B8868DEC9BEA9B878A8789E10E94AC5893
:10DE10006AEF72E00E94984E892B31F082E08E8387
:10DE20008FEF8C878D8709C089E10E94AC58BC01B7
:10DE3000CE010C960E948F4EBE828DEC9BEA9D8B8C
:10DE40008C8B60E678E2CE0146960E948F4E0E944F
:10DE50007C579FA78EA70E94C95788ABC7010E9415
:10DE60003175B82E90E00E94DE57892B31F10E9467
:10DE70008357BC014B2DC7010E944F75E0901403DE
:10DE8000F09015030E94D3575C010E948357B5019F
:10DE9000F70109950115110581F0009739F00197F7
:10DEA00061F441E050E064E070E004C041E050E023
:10DEB00060E070E0C601F8010995E0960FB6F894AD
:10DEC000DEBF0FBECDBFDF91CF911F910F91FF90AD
:10DED000EF90DF90CF90BF90AF9008950E94B17007
:10DEE00080932A14E0911E03F0911F030994892B5B
:10DEF00029F0E0911E03F0911F0304C0E09120037C
:10DF0000F09121030994CF93DF93EC0189919991CA
:10DF1000009729F060E070E00E94E350F7CFDF91B6
:10DF2000CF910895CF93DF93EC0189919991009758
:10DF300019F00E943550F9CFDF91CF910895CF931A
:10DF4000DF93EC017B836A830E9448619983888315
:10DF5000DF91CF910895FC018081918122813381ED
:10DF6000820F931F918380830895CF93DF93EC01F9
:10DF70000E94486199838883DF91CF910895CF9360
:10DF8000DF93EC010E94486128813981821B930B49
:10DF90009C012F5F3F4F81E090E04A815B814217F7
:10DFA000530710F080E090E0DF91CF910895CF9378
:10DFB000DF93FC01C281D38180819181C80FD91F79
:10DFC0000E9448619E01281B390BC901DF91CF9146
:10DFD0000895CF93DF93E9EDFAE2CBE9DAE2ADEC15
:10DFE000BAE21192119219921992199219921D92F4
:10DFF0008AE2E13FF807A9F7DF91CF910895CF9327
:10E00000DF93FC01E353F54D40819C01220F331F48
:10E01000220F331F442301F1A0919400B091950089
:10E02000FC01EE0FFF1FE752F54D80819181AD019C
:10E03000481B590BCA01E901C556D54D4881598184
:10E040006A817B81480F591F611D711D4883598367
:10E050006A837B83B183A083F901E556F54D608126
:10E06000718182819381DF91CF91089560E070E0AA
:10E07000CB010895FC01EE0FFF1FEE0FFF1FE556C9
:10E08000F54D40835183628373830895CF93DF936B
:10E090002DEC3AE2CBE9DAE2E9EDFAE2D9018D9131
:10E0A0009D018823B9F040919400509195008081A2
:10E0B0009181BA01681B790B88819981AA81BB8102
:10E0C000860F971FA11DB11D88839983AA83BB83E7
:10E0D0005183408324963296BAE2293D3B07F1F6FC
:10E0E000DF91CF9108950C94C0740F931F93FC019E
:10E0F000CB0140912B1450912C1433832283158330
:10E10000048371836083F0932C14E0932B14452BCC
:10E1100011F40E94DA7480E090E01F910F9108954D
:10E1200080912B1490912C140097C1F010922C1414
:10E1300010922B14DC0114966D917C911597129618
:10E14000ED91FC9113970995E0912B14F0912C140B
:10E15000309721F0808191810C94DA7408950C94A9
:10E16000E98A0C94E58A8EEC92E00E941A5186ECC2
:10E1700092E00C941A51CF93DF930E948957892B18
:10E18000A9F086EC92E00E943851EC01009721F151
:10E190000E94C957998388830E94C4579B838A83AE
:10E1A000CE0104960E9405578CAB14C08EEC92E011
:10E1B0000E943851EC01009779F002960E9417579F
:10E1C00099838883BE016E547F4FCE018E579F4F37
:10E1D0000E946C58CE0102C080E090E0DF91CF91A8
:10E1E0000895BC016E547F4F8E579F4F0C946C580E
:10E1F000CF93DF93EC01BC018EEC92E00E94825140
:10E20000BE01892B19F08EEC92E009C086EC92E0F9
:10E210000E948251892B39F0BE0186EC92E0DF9199
:10E22000CF910C945D51DF91CF9108950F931F937F
:10E23000CF93DF93EC01BC018EEC92E00E948251FF
:10E24000892B91F0FE0161917191CF010E942858B4
:10E25000BE016E547F4FCE018E579F4FDF91CF91FD
:10E260001F910F910C947D58BE0186EC92E00E94A4
:10E270008251892BD1F00E941558688179818A8159
:10E280009B810E9428588CA990E00E94DE570CA91F
:10E2900010E00E948357BE016C5F7F4FA801DF91A1
:10E2A000CF911F910F910C94568EDF91CF911F91BA
:10E2B0000F910895CF93DF93EC01BC018EEC92E0B7
:10E2C0000E948251892B19F0CE0102960CC0BE012A
:10E2D00086EC92E00E948251892B19F08A819B8101
:10E2E00002C080E090E0DF91CF910895FC01808131
:10E2F00091810895860F911D860F911D8E579F4F16
:10E300000895860F911D860F911D8E579F4FFC011A
:10E3100080819181089508958AE89AE10E945C5372
:10E32000892B21F08AE89AE10C9449530895E091F1
:10E33000761AF091771A309709F0099480E00895E1
:10E34000EF92FF920F931F93CF93DF937C01EA012B
:10E35000FC0180819181009741F08C30934071F1F4
:10E36000F7011182108283E0F2C080E024E0829FF6
:10E37000F0011124E858F54E118210828F5F84302D
:10E38000A8F38093751A8091B0119091B111909378
:10E39000891A8093881A0E942E508093F12A60E493
:10E3A00070E08AE89AE10E9435530E94AE778CE0D3
:10E3B00093E0F7019183808381E0C9C06230D9F492
:10E3C0008091F22A9091F32A892B89F38091032B73
:10E3D000863029F480911B2B81FD0E948C7181E095
:10E3E0000E94EC788091F22A9091F32A892BF9F21D
:10E3F0000E94B073DCCF633060F5611114C02097C8
:10E40000B1F2D0930030C093FF2F83E00E94EC78EC
:10E410008091F22A9091F32A892B11F00E94977132
:10E420000E948C71C4CF613011F6209709F4BFCFE0
:10E43000D093FC2FC093FB2F85E00E94EC78809155
:10E44000F22A9091F32A892B09F4B1CF0E94977197
:10E45000AECF6738E9F51092741A08E71AE1809197
:10E46000741A8430B8F4F801828193818C179D0767
:10E4700049F4808191810E94B978F801118210825B
:10E48000138212820C5F1F4F8091741A8F5F8093EA
:10E49000741AE5CFEAE1F0E3838194818C179D073C
:10E4A00019F4148213821082B09620E3EA39F2073D
:10E4B00099F7E7E9F0E3818592858C179D0711F4C0
:10E4C000158214823D9681E3E931F807A1F76FCFF9
:10E4D000683809F06CCFCA58DA4109F068CF8AE889
:10E4E0009AE10E945C53892B09F461CF1092741A4F
:10E4F000E091741AE43008F05ACF20E2E29FF00174
:10E500001124EF5FFF4C818D8823D9F08AE89AE1CE
:10E510000E9449538091741AE0E28E9FC001112439
:10E520008F5F9F4C909300308093FF2F82E00E947A
:10E53000EC788091F22A9091F32A892B11F00E94B5
:10E5400097718091741A8F5F8093741AD1CFDF9185
:10E55000CF911F910F91FF90EF9008959093771AAC
:10E560008093761A08952091B0113091B11160E036
:10E57000E8E7FAE1643098F440815181481759077F
:10E5800059F4428153814217530731F46093731A4F
:10E59000118210820C94B97834966F5FEBCF609340
:10E5A000731A089540E0E8E7FAE14430A8F451E036
:10E5B000540F20813181232B61F44093721A91838F
:10E5C00080832091B0113091B111338322830C9458
:10E5D000D3783496452FE9CF4093721A089520914D
:10E5E000B0113091B111FC01358F248F778F668F78
:10E5F00008952091B0113091B111FC01328721872B
:10E60000748763870895CF93DF93EA010E945C7853
:10E61000009749F02091B0113091B111FC0132877F
:10E620002187D487C387DF91CF9108950F931F93DC
:10E63000CF93DF9300D000D0CDB7DEB78C01AB0114
:10E640008FEF89838A838B838C83B801CE010196F7
:10E650000E940373009719F0FC01158304830F9047
:10E660000F900F900F90DF91CF911F910F91089510
:10E6700040E050E062E086ED92E00E94D4501092BB
:10E68000F32A1092F22A0895AC0161E086ED92E03F
:10E690000C94B650AC0160E086ED92E00C94B6505C
:10E6A0000F931F93CF93DF938A010E94DA77EC01D7
:10E6B000009759F08091B0119091B1119D8F8C8F7E
:10E6C0001F8F0E8FCE010E944A73CE01DF91CF9132
:10E6D0001F910F910895CF93DF93A091FF2FB091D9
:10E6E0000030109719F0ED016C9605C0C091FB2F1A
:10E6F000D091FC2F29968091FA2F86FF22C010928C
:10E70000711A40E0E8E7FAE14430B8F42081318141
:10E7100014968D919C9115972817390759F4828189
:10E720009381009739F04093711A998388831B82F3
:10E730001A8205C034964F5FE7CF4093711A0E944A
:10E740008C7188819981009741F04A815B81609149
:10E75000F12ADF91CF910C94D450DF91CF9108959D
:10E760000F931F93CF93DF938091032B863009F093
:10E7700071C08091F22A9091F32A8115954009F099
:10E7800069C0C4E9D2E0D093F32AC093F22A02E030
:10E790000093FC2A14E91093FD2A10921F2B10926B
:10E7A0001E2B0E94A8778095909590931F2B8093A5
:10E7B0001E2B1092052B1092042B0E9497778095A8
:10E7C00090959093052B8093042B0E949771D09382
:10E7D000F32AC093F22A0093FC2A1093FD2AA091F9
:10E7E000FD2FB091FE2FFD01E459FD4F8CE692E024
:10E7F00001900D920197E1F76CE672E082E19BE2F5
:10E800000E9456778091F62A8093122B8091F72AE6
:10E810008093132B8091F82A8093142B8091F92AEE
:10E820008093152B10921F2B10921E2B0E94A877FD
:10E830008095909590931F2B80931E2B1092052B03
:10E840001092042B0E949777809590959093052BBA
:10E850008093042BDF91CF911F910F910C949771AE
:10E86000FC01680F791F80E048E1E617F70781F0A7
:10E87000219198E0322F3827532F517030FD842793
:10E880008695513009F480682695915099F7EDCF1F
:10E8900008951F920F920FB60F9211240BB60F928C
:10E8A0002F933F934F935F936F937F938F939F9398
:10E8B000AF93BF93EF93FF93809194009091950055
:10E8C0009093DE2A8093DD2A81E08093CF2A809185
:10E8D0007100807D809371000E9490708091CF2A9A
:10E8E0008823D9F180919400909195004091DD2A80
:10E8F0005091DE2A84179507A0F48091A32A909165
:10E90000A42AA091A52AB091A62A8C57914EAF4F68
:10E91000BF4F8093A32A9093A42AA093A52AB093D3
:10E92000A62A2091940030919500241B350B8091EC
:10E93000A32A9091A42AA091A52AB091A62A820F79
:10E94000931FA11DB11D8093A32A9093A42AA09385
:10E95000A52AB093A62A1092CF2AFF91EF91BF91DA
:10E96000AF919F918F917F916F915F914F913F9167
:10E970002F910F900BBE0F900FBE0F901F90189508
:10E980009FB7F894E1E7F0E08081807D808388B3D1
:10E990008F6288BB10929000E1E9F0E01082109243
:10E9A000920010929500109294008081856080837F
:10E9B0009FBF08952FB7F894909399008093980083
:10E9C00088B38F6288BBE1E7F0E08081826080835A
:10E9D0002FBF0895CF93DF93FC01DB0185E0EB01AE
:10E9E00019928A95E9F78581837011F082E08C9302
:10E9F0008781837021F082E012968C931297858133
:10EA0000837081F08781837069F0238934898185DF
:10EA100092852817390731F481E0848312961C927D
:10EA2000129701C0148285818370823021F0833077
:10EA300021F080E003C082E001C088E011968C9351
:10EA4000119787818370823021F0833021F080E03C
:10EA500003C082E001C088E013968C93DF91CF91D0
:10EA60000895CF93DF9300D000D01F92CDB7DEB7CB
:10EA7000BE016F5F7F4F0E94EA7489819A81890F7E
:10EA80008D5F9B81890F9C81890F9D81890F0F90DC
:10EA90000F900F900F900F90DF91CF9108954F92AC
:10EAA0005F926F927F928F929F92AF92BF92CF921E
:10EAB000DF92EF92FF920F931F93CF93DF9300D0DB
:10EAC00000D000D0CDB7DEB78C017B01BE016F5FF7
:10EAD0007F4F4E830E94EA74B981AA815B804C808B
:10EAE0008B2F90E003962A2F30E0820F931F850D25
:10EAF000911D642D70E0860F971F5D81850F911D1C
:10EB00004E8150E0481759070CF49AC0F8018181F2
:10EB100080FB662460F8712C43E0660C771C4A95F4
:10EB2000E1F7828180FB882480F8912C54E0880CE6
:10EB3000991C5A95E1F7862880818770882A8381FD
:10EB400080FBAA24A0F8B12C85E0AA0CBB1C8A95F6
:10EB5000E1F78A28848180FBCC24C0F8D12C96E090
:10EB6000CC0CDD1C9A95E1F78C28F7018082F80126
:10EB700045814370F4E04F9FA0011124F801868184
:10EB80008370F0E18F9FC0011124482BF801878129
:10EB9000F0E48F9FC0011124482BF7014183F80155
:10EBA0008085F7018283B23059F4F8018185F7013D
:10EBB0008383F8018285F701848395E0C92E02C022
:10EBC00083E0C82EB0E080E090E0200F311FDB2E04
:10EBD000DC0C0197BA1761F0A901480F591FFA011F
:10EBE000B384A7014D0D511DFA01B082BF5FEFCF75
:10EBF0009D2DF2E05F120EC0D701AD0DB11DF801E1
:10EC000083898C9381E08D0DD701A80FB11D9E5F84
:10EC100084898C9340E020E030E0060F171F842F9A
:10EC2000890F21503109441561F0D801A20FB31F9B
:10EC300055965C91D701A80FB11D5C934F5FEFCF44
:10EC400080E026960FB6F894DEBF0FBECDBFDF91F1
:10EC5000CF911F910F91FF90EF90DF90CF90BF90D9
:10EC6000AF909F908F907F906F905F904F9008959E
:10EC7000BF92CF92DF92EF92FF920F931F93CF93A9
:10EC8000DF937C01D62EEA0182E0861708F0B2C03D
:10EC9000F701808186FBBB24B0F89181292F26954E
:10ECA00026952370C92EC294C694C69453E0C522FB
:10ECB000382F3770388383FB332730F9398384FB4F
:10ECC000332730F93A8385FB882780F98B83BC8210
:10ECD0002D83892F829583708E83CF82828188874E
:10ECE000222391F13381848190E0982F8827830F2C
:10ECF000911D9A87898787010B5F1F4F223079F416
:10ED00006AEF72E0CE010B960E948F4EF70186816A
:10ED10008B8785818C878701095F1F4F20C0233037
:10ED2000F1F4F7013D9680E090E03E2F2F2F4291C5
:10ED3000DE01A80FB91F1B964C93019688309105F0
:10ED4000B1F7032F122F0BC087010D5F1F4F6AEF22
:10ED500072E0CE010B960E948F4E1A861986CC2047
:10ED6000B9F1B1100DC0F8012081818190E0982F98
:10ED70008827820F911D9C8B8B8B0E5F1F4F04C0C9
:10ED800089859A859C8B8B8BF2E0CF120EC06AEF3F
:10ED900072E0CE0145960E948F4EF80181818D8BE5
:10EDA00080818E8B0E5F1F4F1BC0F3E0CF1218C007
:10EDB000085F1F4FF80180E090E02291DE01A80F6C
:10EDC000B91F55962C93019688309105B1F708C06C
:10EDD0006AEF72E0CE0145960E948F4E1C8A1B8A14
:10EDE000C8018E199F092D2D281B2FA71EA70DA71F
:10EDF000D81608F480E0DF91CF911F910F91FF901A
:10EE0000EF90DF90CF90BF900895FB0141505109E2
:10EE1000460F571FE417F50778F4208130E0322FB2
:10EE200022276181260F311D820F931F82179307BE
:10EE300008F401963296EECFE417F50751F42081DD
:10EE400030E0322F2227820F931F8217930708F496
:10EE500001960895CF93DF93C091FD2AD0E0649787
:10EE60002091FC2A30E0322F2227C20FD31F48E026
:10EE700050E066E07BE29E01280F311DC9010E942F
:10EE80000577AE016EE07BE20E940577009721F0E6
:10EE900098278927982702C08FEF9FEFDF91CF91A6
:10EEA00008959093A31A8093A21A0895FC015381A8
:10EEB000560F5093F92A872F99274281480F409384
:10EEC000F82AA181A093F72AE081E093F62A242F63
:10EED00030E02817390748F481E08A0F8093F72A39
:10EEE000811103C0EF5FE093F62A852F90E077272A
:10EEF0008617970788F44F5F4093F82A41110CC09A
:10EF00008091F72A8F5F8093F72A811105C0809145
:10EF1000F62A8F5F8093F62A0895AB01BC0180E04A
:10EF200090E00E940577982789279827089544E163
:10EF300050E06AEF7AE280E090E00E940577009767
:10EF400021F098278927982708958FEF9FEF08953C
:10EF500086E00C942A7781E10C942A7780E0E82FF0
:10EF6000F0E0EE0FFF1FEF57FF4C118210828F5F12
:10EF70008430A8F380E090E2899FF0011124EF5FD4
:10EF8000FF4C118E8F5F8430B0F380E094E090935B
:10EF90009D1A80939C1A80E09DE0989FF0011124B7
:10EFA000E956FF4C158214828F5F8A30B0F380934C
:10EFB0009B1A0895CF9320919C1A30919D1A2F5F30
:10EFC0003F4F21154DE7340710F020E030E1522F7C
:10EFD000432FE1E0F0E3C0E0C43059F0A18DAA2353
:10EFE00029F0A481B581A417B50749F3CF5FB09686
:10EFF000F3CF30939D1A20939C1A10929B1A20E015
:10F00000E0E0F0E02430E8F430E2239FD001112466
:10F01000AF5FBF4C59963C915997311104C0209372
:10F020009B1AFD0110C0373041F4309739F05A96E1
:10F030004C915A97328D341708F0DF012F5FFD0194
:10F04000E1CF20939B1A3097A1F122E0218F2091EC
:10F050009E1A248720919F1A25872091A01A26871F
:10F060002091A11A278728ED34E0338B228B358B32
:10F07000248B21E030E0318B208B138E21E0228F16
:10F0800023E0208F168A20E1278B20919C1A309153
:10F090009D1A32272327322735832483778366837B
:10F0A000DC014D915D916D917C9140835183628330
:10F0B0007383CF01CF910895CF93DF9320919C1A52
:10F0C00030919D1A2F5F3F4F21154DE7340710F007
:10F0D00020E030E1522F432FEBE9F0E3C0E0CA30EB
:10F0E00041F0A081B181CF5F3D96A417B507B9F774
:10F0F000E9CF30939D1A20939C1A40E05DE04A309E
:10F10000A0F4A1E0A40F549FF0011124E956FF4C94
:10F1100024813581232B39F440939B1A309741F495
:10F1200080E090E023C04A2FEACF40939B1AF8CFAB
:10F1300020919C1A30919D1A32272327322735833C
:10F14000248377836683009729F4108211821282C8
:10F15000138209C0EC0188819981AA81BB818083D7
:10F160009183A283B38380E48087CF01DF91CF9125
:10F17000089540E04430A0F4E42FF0E051E0540F53
:10F18000EE0FFF1FEF57FF4C208131812817390701
:10F1900029F440939B1A118210820895452FEACFDB
:10F1A00040939B1A089540E0443098F4E42FF0E037
:10F1B00051E0540FEE0FFF1FEF57FF4C20813181BC
:10F1C000232B29F440939B1A918380830895452F24
:10F1D000EBCF40939B1A0895AF92BF92CF92DF92EC
:10F1E000EF92FF920F931F93CF93DF93C091FF2F66
:10F1F000D0910030843009F4DCC122E23BE230934C
:10F20000FE2F2093FD2F3093F52A2093F42A83308C
:10F2100059F4898D8F70833009F06BC08889998982
:10F22000892B09F0DFC67FC0823009F080C0809151
:10F23000A11A8F5F8093A11A811113C08091A01A27
:10F240008F5F8093A01A81110CC080919F1A8F5FED
:10F2500080939F1A811105C080919E1A8F5F8093C1
:10F260009E1A1092F32A1092F22A1092963010925F
:10F270009530298D822F8D7F853041F48A8D8F5F67
:10F280008A8F843109F0AEC6198EACC6222309F4E8
:10F29000A9C688899989892B09F441C08A8D9FEF75
:10F2A000980F9A8F81119EC68B8D883031F09FEF19
:10F2B000920F923048F4853039F4198E80E88093AB
:10F2C000FA2F0E946B7347C5853038F493E0082EFF
:10F2D00001C0990F0A94EAF701C090E39A8F8F5FFB
:10F2E0008B8F822F8F708330A1F048F4813009F426
:10F2F0004FC3823009F076C610921B2B4CC3863068
:10F3000009F4C8C4883009F4C5C4843009F06AC659
:10F31000C1C484E08093FA2F0E946B734EC52F7096
:10F32000233009F05FC688E08093FA2F09C5853045
:10F3300019F5E091FB2FF091FC2F84819581892BA9
:10F3400009F450C6109200301092FF2F86E19BE224
:10F350009093FE2F8093FD2F9093F52A8093F42AAB
:10F3600010929630109295301092F32A1092F22A51
:10F3700088E08093FA2F1BC18091FA2A853409F026
:10F3800031C60091FC2A10E0102F00278091FD2A41
:10F39000080F111D8091F22A9091F32A801791078E
:10F3A00008F420C61093F32A0093F22A8091002BD0
:10F3B0008F7309F017C68091012B811113C68091BC
:10F3C000913090919230C0915703D09158038C178F
:10F3D0009D0759F4409193305091943020915903F6
:10F3E00030915A0342175307A1F020910A2B309114
:10F3F0000B2B2817390709F0F5C520910C2B3091FC
:10F400000D2B80919330909194302817390709F093
:10F41000E9C50E949777019609F0E4C58091032B16
:10F42000863009F429C18131E9F1813009F0DAC56A
:10F4300080910E2B883009F0D5C510920E2B80914B
:10F44000102B9091112B873F3FEF930710F00996F7
:10F4500001C008969093112B8093102B8091062B5E
:10F460009091072BA091082BB091092B80930A2B28
:10F4700090930B2BA0930C2BB0930D2B809191307C
:10F4800090919230A0919330B09194308093062B5C
:10F490009093072BA093082BB093092B80E48093C3
:10F4A000022B7DC50C5111091093F32A0093F22A07
:10F4B00086E19BE29093FE2F8093FD2F8091142B89
:10F4C0009091152B892B29F00E94AB77019609F0BA
:10F4D00089C52091102B3091112B2115310509F48C
:10F4E00081C587E990E39093FC2F8093FB2FA09038
:10F4F0000E2BB0900F2B4091590350915A036091FD
:10F500005B0370915C03A0915D03B0915E03009179
:10F51000062B1091072BE090082BF090092BE0911F
:10F52000FB2FF091FC2F81E3E931F80708F05AC571
:10F5300084819581009721F12817390709F5868183
:10F540009781009719F0A816B906D1F480819181AE
:10F550008C179D0729F4C280D380C416D506B1F05C
:10F560008617970729F4C280D380CA16DB0671F08C
:10F570000817190729F482819381E816F90631F0FA
:10F580003D96F093FC2FE093FB2FC9CF10920030F3
:10F590001092FF2F82E08093FA2F86E19BE29093F6
:10F5A000F52A8093F42A10929630109295300E949A
:10F5B0006B738091953090919630009709F412C545
:10F5C0009C01245E3F4F3093F32A2093F22A30931C
:10F5D000FC2A2093FD2AE091FB2FF091FC2F20853F
:10F5E0002093022B21E12093032B0896982789274B
:10F5F00098279093132B8093122B1092152B109217
:10F60000142B8481958190930F2B80930E2B8681F0
:10F6100097819093112B8093102B80919130909132
:10F620009230A0919330B09194308093062B9093B8
:10F63000072BA093082BB093092B80819181A28185
:10F64000B38180930A2B90930B2BA0930C2BB09338
:10F650000D2B82E29BE29093FE2F8093FD2F0E9460
:10F66000AB7780959095009711F48FEF9FEF909373
:10F67000152B8093142B93C40E94A877019609F050
:10F68000B1C48091102B9091112B009709F4AAC45A
:10F6900020910E2B30910F2B2115310509F4A2C4B6
:10F6A0004091062B5091072B6091082B7091092BEC
:10F6B000EAE1F0E3C1E0D0E3F080FF20A9F0AC8103
:10F6C000BD818A179B0781F4AE81BF812A173B0752
:10F6D00059F4A881B9814A175B0731F4AA81BB812B
:10F6E0006A177B0709F46FC1A096B096A0E3C138F2
:10F6F000DA0711F720911B2B2F732230D9F4909346
:10F70000991A8093981A40E0443090F4E42FF0E086
:10F71000EE0FFF1FEF57FF4C208131814F5F8217A3
:10F72000930791F710929B1A20E0C0E0D0E07EC0D2
:10F7300040939B1A80911B2B82FD54C484E18093DB
:10F740001B2B88E290E09093F32A8093F22A80E5C5
:10F7500080931A2B8091152B9091192B9093152B38
:10F760003091142B9091182B9093142B3093182BCD
:10F770002091132B9091172B9093132B2093172BE1
:10F780009091122B90939B1A4091162B4093122B21
:10F790009093162B8F5F8093192B81110FC081E0FE
:10F7A000830F8093182B811109C081E0820F809311
:10F7B000172B811103C09F5F9093162B80910E2B06
:10F7C00090910F2B9093991A8093981A2091102B57
:10F7D0003091112B30930F2B20930E2B9093112BE4
:10F7E0008093102B8091062B9091072BA091082BD2
:10F7F000B091092B80930A2B90930B2BA0930C2B89
:10F80000B0930D2B8091913090919230A0919330D4
:10F81000B09194308093062B9093072BA093082BE4
:10F82000B093092BA1C3373089F02F5F2430C0F487
:10F8300030E2239FC0011124FC01EF5FFF4C318DAA
:10F840003111F1CF20939B1AEF010CC0209721F0CA
:10F85000428D3A8D341748F7EC01CF5FDF4CE5CF8E
:10F8600020939B1A209709F4BDC3D0930030C09316
:10F87000FF2F83E08A8F888F1E8A84E08F8B1B8EF8
:10F880008091102B9091112B9D838C8380910E2B56
:10F8900090910F2B9F838E838091062B9091072B45
:10F8A000A091082BB091092B88839983AA83BB83ED
:10F8B00081E0898F80919E1A8C8780919F1A8D8715
:10F8C0008091A01A8E878091A11A8F8781E090E0A5
:10F8D000998B888B8091152B8B878091142B8A872D
:10F8E0008091132B89878091122B888781E090E08B
:10F8F0000E94568080911A2B282F207F30E02135DE
:10F9000031050CF445C082958F7090E00597880F03
:10F91000991F880F991F30919A1A20E0E22FF0E08A
:10F92000E817F9078CF5E650F54D30A5311105C003
:10F9300020939B1A10929A1A2BC0313011F42F5F2A
:10F94000EDCF3230E1F441A54430C9F420939B1A45
:10F9500030939A1A82A590E0982F882723A5822BAE
:10F960009093991A8093981A893DA4E09A0710F011
:10F9700088ED94E09B8B8A8B9D8B8C8B09C041A575
:10F98000442311F0240FCACF20939B1A30939A1A64
:10F9900080E180931B2B80911B2B826080931B2B1B
:10F9A00082E08093222B84E08093232B8093242B6E
:10F9B00088ED8093252B8CE290E09093F32A80933E
:10F9C000F22A80E67EC2D0930030C093FF2F1092BF
:10F9D000FA2F90911B2B92FF03C0198E80E21AC25E
:10F9E00080911A2B82958F70880F880F80939B1AB5
:10F9F000081B1109045111091093F32A0093F22AEC
:10FA00008F2D8F70823029F4892F8F73823139F4D2
:10FA10001FC0813021F4892F8F738230C9F0012BF0
:10FA200019F4892F8370A1F02091122B8885281357
:10FA30003EC22091132B8985281339C22091142BA3
:10FA40008A85281334C22091152B8B8528132FC249
:10FA500094FF4AC0688979896115710509F444C029
:10FA6000CE010C960E9456773091162B8091F62A83
:10FA700038133AC02091172B8091F72A281334C0ED
:10FA80009091182B8091F82A98132EC08091192BF1
:10FA90004091F92A841328C03C872D879E878F8741
:10FAA0008B8D81111AC02E89888D9A8D891B922F7A
:10FAB000969596959695891B280F2E8B87FD819597
:10FAC0009F89392F36953695931B980F9F8B822FE0
:10FAD000869586958695890F888F81E08093FA2F89
:10FAE000888D8A8F198A188A498D842F8F7090E0AB
:10FAF000FC013197E830F10508F074C2E057FF4F80
:10FB00000C94218A8091FA2F80FF14C083E0898FA2
:10FB100080E48093FA2F198A188A8091F22A9091B2
:10FB2000F32A009709F408C122E42093FA2F0E94D7
:10FB3000568002C180911B2B8F73823009F052C214
:10FB400027CF8091FA2F80FF70C080911B2B8F737D
:10FB5000823109F06AC080911A2B282F207F30E073
:10FB6000213531050CF445C082958F7090E00597E2
:10FB7000880F991F880F991F30919A1A20E0E22F61
:10FB8000F0E0E817F9078CF5E650F54D30A5311196
:10FB900005C020939B1A10929A1A2BC0313011F491
:10FBA0002F5FEDCF3230E1F441A54430C9F420930A
:10FBB0009B1A30939A1A82A590E0982F882723A544
:10FBC000822B9093991A8093981A893D24E092078A
:10FBD00010F088ED94E09B8B8A8B9D8B8C8B09C0F9
:10FBE00041A5442311F0240FCACF20939B1A3093D0
:10FBF0009A1A83E0898F8091122B88878091132B2A
:10FC000089878091142B8A878091152B8B8781E0BF
:10FC100090E00E94568082E48093FA2F198A188A15
:10FC20001092F32A1092F22A87C080E28093FA2F72
:10FC30000E946B73E091FF2FF0910030118E7ACD0E
:10FC400080911B2B80FF28C044FD26C0888999899C
:10FC5000892B09F0C7C18091F22A9091F32A01966D
:10FC60000E9456802091FA2F822F80618093FA2F74
:10FC70008091F22A9091F32A892B19F02261209326
:10FC8000FA2F0E946B7381E090E0998B888B88E05B
:10FC9000898F1B8E81E10CC185FF1CC08091202BB8
:10FCA00090E0982F88272091212B822B2091FD2FE7
:10FCB0003091FE2F280F391F3093FE2F2093FD2FF8
:10FCC0002091F22A3091F32A281B390B3093F32A22
:10FCD0002093F22A8091F22A9091F32A009749F01A
:10FCE00044FD07C02091FA2F22602093FA2F0E9432
:10FCF000568080911C2B90E0982F882720911D2BF7
:10FD0000820F911D9093991A8093981A2C893D899E
:10FD10002817390710F0892B21F43093991A209372
:10FD2000981A8091981A9091991A9B8B8A8B80913E
:10FD3000FA2F837009F456C11092963010929530C4
:10FD40000E946B738091FA2F85FF07C01092963046
:10FD500010929530198E84E1ABC084FF0AC01092D6
:10FD600096301092953081E090E0998B888B84E0FA
:10FD70008FCF209195303091963021153105E1F0EB
:10FD800080FF02C0198A188A88899989009781F4AE
:10FD90008A899B898217930720F4909396308093E9
:10FDA00095308091953090919630998B888B04C0D6
:10FDB00090939630809395301B8E8091F42A909189
:10FDC000F52A9093FE2F8093FD2F8091953090918E
:10FDD0009630892B59F088899989009739F088964F
:10FDE0009093F32A8093F22A88E10BC08091FA2F36
:10FDF00081FFF8C088E290E09093F32A8093F22A82
:10FE000080E180931B2B5CC08091FA2F80FFEAC0B9
:10FE1000198E80E18093FA2F0E946B73E3C080916A
:10FE2000F22A9091F32A009711F00E945680909147
:10FE30001B2B8091FA2F90FF0BC080FF06C087E03C
:10FE4000898F1A8E198A188A19C086E0898F16C080
:10FE500080FF1EC085E0898F198A188AC3C08091EF
:10FE6000F22A9091F32A009711F00E945680809117
:10FE70001B2B80FF0DC087E0898F1A8E81E090E0F8
:10FE80000E94568080E18093FA2F0E946B730FC00E
:10FE90008091F22A9091F32A892B49F4A3C0809192
:10FEA000FA2F80FF9FC087E0898F1A8E9BC080E168
:10FEB00080931B2B88E290E09093F32A8093F22AA0
:10FEC00080E580931A2B88858093162B89858093F3
:10FED000172B8A858093182B8B858093192B8C8503
:10FEE0008093122B8D858093132B8E858093142BFA
:10FEF0008F858093152B86E08093032B8C819D81C9
:10FF000090930F2B80930E2B8E819F819093112BBA
:10FF10008093102B8091913090919230A0919330EA
:10FF2000B09194308093062B9093072BA093082BCD
:10FF3000B093092B88819981AA81BB8180930A2B78
:10FF400090930B2BA0930C2BB0930D2B898D84FFDA
:10FF500005C010921D2B10921C2B06C084E08093CC
:10FF60001C2B88ED80931D2B80E48093022B8091C5
:10FF7000F22A9091F32A9093FC2A8093FD2A109202
:10FF8000212B1092202B10921F2B10921E2B0E94BF
:10FF9000A8778095909590931F2B80931E2B85E4D6
:10FFA0008093FA2A1092FB2A1092012B1092002BB8
:10FFB0008091A21A9091A31A01969093A31A80930C
:10FFC000A21A9093FE2A8093FF2A1092052B10927A
:10FFD000042B0E949777809590959093052B8093A2
:10FFE000042B04C01092F32A1092F22A1092FA2FD6
:10FFF000DF91CF911F910F91FF90EF90DF90CF9005
:020000021000EC
:10000000BF90AF90089598278927982708950E9458
:10001000278A0895FC018091F42A9091F52A2AEF0D
:100020003FE2281B390BAB01261737070CF4A90157
:100030001416150654F45093963040939530E817F3
:10004000F90719F0BF010C94568E089580E880934B
:100050006100109261000E94DC5E0E944B500E9481
:10006000B8628091A1289091A228009729F0019769
:100070009093A2288093A128C090A328D090A42870
:10008000E090A528F090A6280E947661C616D706B3
:10009000E806F90611F30E9476616093A328709335
:1000A000A4288093A5289093A628D7CF2091FF2F2E
:1000B00030910030BC01C90108960E945677E0914A
:1000C000FF2FF09100308091F62A80878091F72AE7
:1000D00081878091F82A82878091F92A8387089501
:1000E0002F923F924F925F926F927F928F929F9248
:1000F000AF92BF92CF92DF92EF92FF920F931F9336
:10010000CF93DF93CDB7DEB763970FB6F894DEBF1A
:100110000FBECDBF7C011B016A01FC011782168254
:10012000838181FF66C3BE016F5F7F4F4B01F70183
:100130009381F10193FD859193FF81911F018823A4
:1001400009F453C3853239F493FD859193FF81916E
:100150001F01853239F4B70190E00E94D98E560113
:100160006501E5CF10E0512C20E02032A0F48B3265
:1001700069F030F4803259F0833269F420612CC088
:100180008D3239F0803339F4216026C0226024603A
:1001900023C0286021C027FD27C030ED380F3A303A
:1001A00078F426FF06C0FAE01F9F300D1124132FAC
:1001B00013C06AE0569E300D1124532E20620CC0ED
:1001C0008E3221F426FD11C3206406C08C3611F452
:1001D000206802C0883641F4F10193FD859193FFB8
:1001E00081911F018111C1CF9BEB980F933018F4BF
:1001F0002061805E06C09BE9980F933008F0AAC189
:100200002F7E26FF16E02F73722E853621F4F22FF3
:10021000F0647F2E08C0863621F4622F6068762E47
:1002200002C01111115077FE07C01C3348F444245A
:100230004394410E27E00BC0183030F4212F06C044
:1002400027E04CE3442E03C027E017E0412C560181
:1002500074E0A70EB11CF6016081718182819381E7
:10026000042DA4010E945E8D6C01098100FF02C073
:1002700003FF06C071FC07C072FC08C0612C08C0F7
:100280003DE2632E05C02BE2622E02C090E2692E91
:10029000802F8C7099F1662011F084E001C083E01A
:1002A000851510F0512C0BC0581A73FC08C0B7010B
:1002B00080E290E00E94D98E5A94C9F7F3CF66206D
:1002C00029F0B701862D90E00E94D98E03FD03C06E
:1002D00004E910E102C000E910E1F72DF0717F2E72
:1002E000F8018491882309F476C271108052B70115
:1002F00090E00E94D98E0F5F1F4FF2CF77FE0FC0A4
:100300004C0C04FF04C08A81813309F44A9414140C
:1003100074F5F8E0F41578F588E0482E2CC076FCEA
:100320002AC0812F90E08C159D059CF06CEFC616BD
:100330006FEFD60674F0772D7068772E0AC0E2E072
:10034000F0E0EC0FFD1FE10FF11D8081803319F407
:1003500011501111F4CF77FE0EC044244394410E86
:10036000812F90E0C816D9062CF41C1904C044242F
:10037000439401C010E077FE07C01C141D043CF438
:1003800096012F5F3F4F05C025E030E002C021E01D
:1003900030E0662011F02F5F3F4F112331F0412FE5
:1003A00050E04F5F5F4F240F351F452D50E024175D
:1003B000350714F4521A01C0512C872D897049F465
:1003C000552039F0B70180E290E00E94D98E5A940E
:1003D000F7CF662029F0B701862D90E00E94D98ED4
:1003E00073FC09C0552039F0B70180E390E00E940A
:1003F000D98E5A94F7CF77FE5FC09C2D8D2DD7FEF6
:1004000002C090E080E0692E782E40E050E0C60106
:10041000841991099D878C87960126193709280D23
:10042000391D812F90E0EE27FF27E81BF90BFF878E
:10043000EE87FFEF6F167F0669F4B7018EE290E05A
:100440002B8B3A8B488B598B0E94D98E59894889BE
:100450003A892B89C614D70454F06C857D856615BE
:1004600077052CF4F901E40FF51F818101C080E3C9
:1004700071E0671A71084F5F5F4FEE85FF856E165A
:100480007F066CF0B70190E02B8B3A8B488B598B31
:100490000E94D98E2B893A8948895989CACF6C1410
:1004A0007D0439F49A81963318F4953311F404FFDE
:1004B00081E3B70190E04BC08A81813309F00F7E60
:1004C000B70190E00E94D98E111105C074FE18C0CA
:1004D00085E490E017C0B7018EE290E00E94D98ECB
:1004E00082E066246394680EF401E80FF11D8081B8
:1004F000B70190E00E94D98E115041F3862DF1CFC3
:1005000085E690E0B7010E94D98ED7FC05C0C114E2
:10051000D10439F404FF05C0D194C194D1088DE20F
:1005200001C08BE2B70190E00E94D98E80E36AE0BF
:10053000C616D1042CF08F5FFAE0CF1AD108F7CF9E
:10054000B70190E00E94D98EB701C601C0960E9403
:10055000D98E41C1833631F0833779F0833509F084
:1005600058C021C0560172E0A70EB11CF60180816F
:10057000898301E010E0640114C05601F2E0AF0E7F
:10058000B11CF601C080D18026FF03C0612F70E04E
:1005900002C06FEF7FEFC6012B8B0E94858E8C010E
:1005A0002B892F7715C05601F2E0AF0EB11CF60172
:1005B000C080D18026FF03C0612F70E002C06FEFC2
:1005C0007FEFC6012B8B0E94478E8C012B89206800
:1005D000722E23FD1AC0852D90E008171907A8F484
:1005E000B70180E290E00E94D98E5A94F4CFF601D0
:1005F00077FC859177FE81916F01B70190E00E94B1
:10060000D98E51105A94015011090115110579F72D
:10061000E2C0843611F0893651F5560127FF09C032
:10062000F4E0AF0EB11CF60160817181828193818B
:100630000AC0F2E0AF0EB11CF6016081718188271B
:1006400077FD8095982F022F0F7697FF08C0909521
:100650008095709561957F4F8F4F9F4F00682AE07E
:1006600030E0A4010E941390C82EC8183EC0022F8B
:10067000853721F40F7E2AE030E01DC0097F8F36D8
:1006800091F018F4883559F0B0C0803719F08837E8
:1006900011F0ABC0006104FF09C0046007C024FF73
:1006A00008C0066006C028E030E005C020E130E068
:1006B00002C020E132E0560107FF09C0F4E0AF0EAE
:1006C000B11CF601608171818281938108C0F2E0E2
:1006D000AF0EB11CF6016081718180E090E0A40151
:1006E0000E941390C82EC8180F7706FF0BC0202F4A
:1006F0002E7FC11650F404FF0AC002FD08C0202F4F
:100700002E7E05C0DC2C202F03C0DC2C01C0D12E96
:1007100024FF0DC0FE01EC0DF11D8081803311F42A
:10072000297E09C022FF06C0D394D39404C0822F2F
:10073000867809F0D39423FD13C020FF06C01C2D3A
:10074000D51418F4150D1D19D52CD51468F4B7015E
:1007500080E290E02B8B0E94D98ED3942B89F5CF29
:10076000D51410F45D1801C0512C24FF12C0B7013C
:1007700080E390E02B8B0E94D98E2B8922FF17C03B
:1007800021FF03C088E590E002C088E790E0B70150
:100790000CC0822F867859F021FD02C080E201C092
:1007A0008BE227FD8DE2B70190E00E94D98EC11641
:1007B00038F4B70180E390E00E94D98E1150F7CF52
:1007C000CA94F401EC0DF11D8081B70190E00E9404
:1007D000D98EC110F5CF552009F4C2CCB70180E203
:1007E00090E00E94D98E5A94F6CFF70186819781C6
:1007F00002C08FEF9FEF63960FB6F894DEBF0FBE77
:10080000CDBFDF91CF911F910F91FF90EF90DF90BF
:10081000CF90BF90AF909F908F907F906F905F90A0
:100820004F903F902F9008955058BB27AA270ED085
:100830004EC23FD230F044D220F031F49F3F11F449
:100840001EF4FFC10EF4E095E7FBF5C1E92F50D28D
:1008500080F3BA17620773078407950718F071F4DD
:100860009EF568C20EF4E0950B2EBA2FA02D0B0159
:10087000B90190010C01CA01A0011124FF27591BE5
:1008800099F0593F50F4503E68F11A16F040A22FEB
:10089000232F342F4427585FF3CF4695379527955C
:1008A000A795F0405395C9F77EF41F16BA0B620B5B
:1008B000730B840BBAF09150A1F0FF0FBB1F661FA2
:1008C000771F881FC2F70EC0BA0F621F731F841FE5
:1008D00048F4879577956795B795F7959E3F08F00B
:1008E000B3CF9395880F08F09927EE0F97958795CA
:1008F0000895DFD158F080E891E009F49EEFE0D14F
:1009000028F040E851E059F45EEF09C09AC112C2E4
:10091000E92FE078EDD168F3092E052AC1F32617F7
:1009200037074807590738F00E2E07F8E02569F019
:10093000E025E0640AC0EF6307F8009407FADB01E2
:10094000B9019D01DC01CA01AD01EF9347D0BFD1D0
:100950000AD05F91552331F02BED3FE049E450FD83
:1009600049EC63CF0895DF93DD27B92FBF7740E8C7
:100970005FE31616170648075B0710F4D92FE1D17D
:100980009F938F937F936F9346D3E0E3F1E06CD115
:100990009ED12F913F914F915F919AD2DD2349F0E3
:1009A0009058A2EA2AED3FE049EC5FE3D0785D275A
:1009B0004DDFDF918CC11BD108F481E008950CD08C
:1009C00086C17ED140F075D130F021F45F3F19F03F
:1009D00032C15111B0C135C18BD198F39923C9F3FC
:1009E0005523B1F3951B550BBB27AA276217730735
:1009F000840738F09F5F5F4F220F331F441FAA1FE9
:100A0000A9F333D00E2E3AF0E0E830D091505040A8
:100A1000E695001CCAF729D0FE2F27D0660F771F56
:100A2000881FBB1F261737074807AB07B0E809F038
:100A3000BB0B802DBF01FF2793585F4F2AF09E3FCD
:100A4000510568F0F8C077C15F3FECF3983EDCF3E6
:100A5000869577956795B795F7959F5FC9F7880F46
:100A6000911D9695879597F90895E1E0660F771F98
:100A7000881FBB1F621773078407BA0720F0621B29
:100A8000730B840BBA0BEE1F88F7E095089519F4E9
:100A90000EF0D1C04FC1D5C033D1C8F39638C0F7DE
:100AA00007F80F92E8942BE33AEA48EB5FE712D29B
:100AB0000F920F920F924DB75EB70F92CAD1EDE52C
:100AC000F1E0D2D04F915F91EF91FF91E595EE1F4C
:100AD000FF1F49F0FE57E0684427EE0F441FFA95C8
:100AE000E1F74195550B36D10F9007FE2AC10895C5
:100AF00097FB0EF4A9D03EC0E89409C097FB3EF4E2
:100B000090958095709561957F4F8F4F9F4F99235A
:100B1000A9F0F92F96E9BB279395F69587957795D8
:100B20006795B795F111F8CFFAF4BB0F11F460FF98
:100B30001BC06F5F7F4F8F4F9F4F16C0882311F0F0
:100B400096E911C0772321F09EE8872F762F05C004
:100B5000662371F096E8862F70E060E02AF09A959F
:100B6000660F771F881FDAF7880F9695879597F994
:100B70000895E894F92F96EBFF2381F012161306DF
:100B80001406440B9395F695879577956795579539
:100B90004040FF23B9F71BC099270895882351F4DB
:100BA0009850D2F7872B762F652F542F432F322F53
:100BB00020E0B1F3121613061406440B88233AF012
:100BC0009A95440F551F661F771F881FCAF7552334
:100BD0004AF4440F551F11F460FF04C06F5F7F4F4C
:100BE0008F4F9F4F880F9695879597F90895990F86
:100BF0000008550FAA0BE0E8FEEF16161706E807E7
:100C0000F907C0F012161306E407F50798F0621B07
:100C1000730B840B950B39F40A2661F0232B242BDC
:100C2000252B21F408950A2609F4A140A6958FEFFB
:100C3000811D811D089597F99F6780E870E060E04D
:100C400008959FEF80EC089590958095709560953C
:100C500050954095309521953F4F4F4F5F4F6F4FC7
:100C60007F4F8F4F9F4F0895DF93CF931F930F9325
:100C7000FF92EF92DF927B018C01689405C0DA2E1F
:100C8000EF0126D1FE01E894A5912591359145917A
:100C90005591AEF3EF01DADDFE019701A801DA9478
:100CA00079F7DF90EF90FF900F911F91CF91DF9137
:100CB000089500240A9416161706180609060895C2
:100CC00000240A9412161306140605060895092E28
:100CD0000394000C11F4882352F0BB0F40F4BF2B97
:100CE00011F460FF04C06F5F7F4F8F4F9F4F0895D7
:100CF00057FD9058440F551F59F05F3F71F04795CD
:100D0000880F97FB991F61F09F3F79F087950895B1
:100D1000121613061406551FF2CF4695F1DF08C0D0
:100D2000161617061806991FF1CF869571056105ED
:100D300008940895E894BB2766277727CB0197F995
:100D400008959B01AC0160E070E080E89FE337CE3E
:100D500072CF64C1D5DFE8F39923D9F3940F511D05
:100D6000BBF39150504094F059F0882332F0660F55
:100D7000771F881F91505040C1F79E3F510544F79F
:100D8000880F911D9695879597F908955F3FACF070
:100D9000983E9CF0BB27869577956795B79508F4A4
:100DA000B1609395C1F7BB0F58F711F460FFE8CF1E
:100DB0006F5F7F4F8F4F9F4FE3CFBDCF0AD029ED9D
:100DC0003BE54EED5EE378C00EF028C13ACF689463
:100DD00032CF96DFC8F39923D1F3C6F3DF93CF93D5
:100DE0001F930F93FF92C92FDD2788232AF02197A5
:100DF000660F771F881FDAF720E030E040E85FEBEE
:100E00009FE3883920F0803E30F021968F770DDD0A
:100E1000E5E8F1E003C009DDE2EBF1E025DF8B015D
:100E2000BE01EC01FB2E6F5771097595771F880B7A
:100E3000990B64DE28E132E741E35FE349D0AF2D4F
:100E40009801AE01FF900F911F91CF91DF91FEDCD1
:100E50003ECFFA01DC01AA0FBB1F9B01AC01BF57BB
:100E600028F422273327442750781FC0B75188F42D
:100E7000AB2F0024469537952795011CA395D2F3F7
:100E8000002069F0220F331F441FB395DAF30DD011
:100E9000CBCC61307105A0E88A07B94630F49B01DC
:100EA000AC016627772788279078309621F0208339
:100EB00031834283538308950BD009CFFADE28F0A3
:100EC000FFDE18F0952309F0B6CEBBCE112433CF48
:100ED0000FDFA0F3959FD1F3950F50E0551F629F50
:100EE000F001729FBB27F00DB11D639FAA27F00D83
:100EF000B11DAA1F649F6627B00DA11D661F829FAA
:100F00002227B00DA11D621F739FB00DA11D621F8E
:100F1000839FA00D611D221F749F3327A00D611DAB
:100F2000231F849F600D211D822F762F6A2F11248D
:100F30009F5750408AF0E1F088234AF0EE0FFF1FE0
:100F4000BB1F661F771F881F91505040A9F79E3F17
:100F5000510570F070CEEFCE5F3FECF3983EDCF3BE
:100F6000869577956795B795F795E7959F5FC1F754
:100F7000FE2B880F911D9695879597F90895FA0194
:100F8000EE0FFF1F30962105310599F161157105AE
:100F900061F48038BFE39B0749F16894903881057C
:100FA00061F08038BFEF9B0741F0992342F5FF3F86
:100FB000E1053105210511F1E8940894E795D9017F
:100FC000AA2329F4AB2FBE2FF85FD0F310C0FF5F28
:100FD00070F4A695E0F7F73950F019F0FF3A38F4BD
:100FE0009F779F930CD00F9007FC905808953EF088
:100FF00028CE60E070E080E89FE308954FE79F7798
:101000005F934F933F932F93E4DE2F913F914F9146
:101010005F9152DF41CD9B01AC014ECF9F3F31F03C
:10102000915020F4879577956795B795880F911D16
:101030009695879597F908950E942488332312F492
:101040008A1B9B0B0C943588A29FB001B39FC001F3
:10105000A39F700D811D1124911DB29F700D811DE4
:101060001124911D08950E942488B7FF0895821BC2
:10107000930B08950E942488A59F900DB49F900D16
:10108000A49F800D911D11240895B7FF0C943A88F8
:101090000E943A88821B930B0895DB018F939F93E4
:1010A0000E943A88BF91AF91A29F800D911DA39F8E
:1010B000900DB29F900D11240895AA1BBB1B51E106
:1010C00007C0AA1FBB1FA617B70710F0A61BB70BB8
:1010D000881F991F5A95A9F780959095BC01CD015D
:1010E000089597FB072E16F4009407D077FD09D0DA
:1010F0000E945D8807FC05D03EF4909581959F4F36
:101100000895709561957F4F0895A1E21A2EAA1B4C
:10111000BB1BFD010DC0AA1FBB1FEE1FFF1FA217A7
:10112000B307E407F50720F0A21BB30BE40BF50BA4
:10113000661F771F881F991F1A9469F7609570952D
:10114000809590959B01AC01BD01CF010895052EBE
:1011500097FB1EF400940E94D28957FD07D00E948D
:10116000858807FC03D04EF40C94D28950954095A5
:10117000309521953F4F4F4F5F4F0895689401C0C0
:10118000E894F92FF12B12F00C94F288A0E0B0E073
:10119000ECECF8E80C94F089092E059422F40E94F6
:1011A000DA89112392F4F0E80F26FFEFE094F0942F
:1011B00000951095B094C094D094A194BF0ACF0A22
:1011C000DF0AEF0AFF0A0F0B1F0B0E94818907FC41
:1011D0000E94DA89CDB7DEB7ECE00C940C8A6894F3
:1011E00001C0E8948F929F92CF93DF930E948189F0
:1011F000DF91CF919F908F900895DF93CF931F93AE
:101200000F939A9DF02D219FF00D8B9DF00D8A9DDF
:10121000E02DF10D039FF00D029FE00DF11D4E9D9D
:10122000E00DF11D5E9DF00D4F9DF00D7F936F93CE
:10123000BF92AF925F934F93D5010E9424888B0198
:10124000AC01D7010E942488EB01E80FF91FD601F9
:101250000E944D892F913F91D6010E942488C60F8C
:10126000D71FE81FF91FAF91BF910E944D892F91A1
:101270003F910E942488C60FD71FE81FF91FD6018F
:101280000E942488E60FF71F9801BE01CF011124A8
:101290000F911F91CF91DF9108950E942488460FEE
:1012A000571FC81FD91F08F431960895E894DF939B
:1012B000CF93FC01DB010E9424887F936F93E901A7
:1012C0009A01AC01BF93AF933F932F93DF010E942C
:1012D000248826F46C1B7D0B820B930B9E01EB0183
:1012E000FC010E944D89AF91BF912F913F910E94C7
:1012F0004D89BE01CF01F9012F913F91CF91DF912F
:10130000089588249924F401E401B0E49F93AA2766
:101310009A158B049C04ED05FE05CF05D007A107A7
:1013200098F4AD2FDC2FCF2FFE2FE92D982C892E8E
:10133000982F872F762F652F542F432F322F222758
:10134000B85031F7BF9127C01B2EBF91BB27220F8A
:10135000331F441F551F661F771F881F991F881C46
:10136000991CEE1FFF1FCC1FDD1FAA1FBB1F8A1475
:101370009B04EC05FD05CE05DF05A007B10748F08D
:101380008A189B08EC09FD09CE09DF09A00BB10BF7
:1013900021601A94E1F62EF49401AF01BE01CD0153
:1013A000000C089590958095709561957F4F8F4FB3
:1013B0009F4F0895609570958095909530954095D4
:1013C000509521953F4F4F4F5F4F6F4F7F4F8F4F3E
:1013D0009F4F08952F923F924F925F926F927F920C
:1013E0008F929F92AF92BF92CF92DF92EF92FF9235
:1013F0000F931F93CF93DF93CDB7DEB7CA1BDB0BE1
:101400000FB6F894DEBF0FBECDBF09942A88398885
:1014100048885F846E847D848C849B84AA84B9848C
:10142000C884DF80EE80FD800C811B81AA81B98198
:10143000CE0FD11D0FB6F894DEBF0FBECDBFED01AC
:101440000895EE0FFF1F0590F491E02D0994692790
:101450009627692778278727782708950F930830DC
:1014600090F0982F872F762F652F542F432F322FF0
:1014700022270850F4CF220F331F441F551F661F29
:10148000771F881F991F0A95B2F70F91089597FB50
:1014900010F8169400080F93083098F00850232F86
:1014A000342F452F562F672F782F892F902DF4CF6B
:1014B00005949795879577956795579547953795AF
:1014C00027950A95AAF70F9108952A0D3B1D4C1DEB
:1014D0005D1D6E1D7F1D801F911F08950024A7FDB7
:1014E00000942A0F301D401D501D601D701D801D71
:1014F000901D08952A193B094C095D096E097F0961
:10150000800B910B08952A153B054C055D056E0572
:101510007F058007910708950024A7FD00942A17EE
:10152000300540055005600570058005900508955B
:101530008F929F92AF92BF92CF92DF92EF92FF92E3
:10154000CF93DF93EC01688179818A819B8161155A
:1015500071058105910521F464E279ED8BE597E051
:101560002DE133EF41E050E00E94A78849015A0184
:101570009B01AC01A7EAB1E40E943A886B017C01AF
:10158000ACEEB4EFA50194010E944888C60ED71EA8
:10159000E81EF91EF7FE06C081E0C81AD108E1086E
:1015A00080E8F80AC882D982EA82FB82C6019F7766
:1015B000DF91CF91FF90EF90DF90CF90BF90AF90F1
:1015C0009F908F9008950C94988A80EE92E00C94EE
:1015D000988AA0E0B0E08093E0029093E102A093AB
:1015E000E202B093E30208952F923F925F926F92CE
:1015F0007F928F929F92AF92BF92CF92DF92EF92A3
:10160000FF920F931F93CF93DF938B01EA01611534
:10161000710521F0DB018C9311969C93209739F092
:101620009E01225031092332310508F0FBC07C01B4
:101630006701BFEFCB1ADB0A5601F7016080862DE8
:1016400090E00E94368E892B11F07601F1CFFDE2F9
:101650006F120AC0570182E0A80EB11CD701119683
:101660006C90772473940BC0BBE26B1207C05701D8
:10167000E2E0AE0EB11CD70111966C90712CCE0138
:101680008F7E892B89F4B0E36B1222C0F501808133
:101690008F7D883541F56180F2E0AF0EB11C872D5A
:1016A0008260782EC0E1D0E0C830D105F1F04CF472
:1016B000C230D10511F5C12CD12CE12CB0E4FB2EA8
:1016C0002FC0CA30D10531F0C031D10521F115C08C
:1016D000209751F7CAE0D0E0ACECCA2EDC2CEC2C01
:1016E000ACE0FA2E1DC02097F9F6C8E0D0E0C12C7E
:1016F000D12CE12CF0E1FF2E13C060E070E080E01F
:1017000090E89E01442737FD4095542F0E9485881C
:1017100069017A0105C0C12CD12CE12CE8E0FE2E34
:10172000F50160E020E030E0A9014E01AA2497FC19
:10173000A094BA2C1F0170ED572E560CA9E0A515E8
:1017400070F48FEB860D8A3118F499EC592E06C08F
:101750008FE9860D8A3130F589EA582E560C852D91
:1017600090E08C179D07F4F467FD18C0C216D306ED
:10177000E406F50680F0C501B4010E944D889B0186
:10178000AC01250D311D411D511D21303105410593
:10179000B0E85B0710F06FEF01C061E03196D10156
:1017A0006C90C8CF872D81700115110571F06623EB
:1017B00029F03197D801ED93FC9307C071FE19C051
:1017C0003297D801ED93FC9314C067FF12C08823B1
:1017D00029F020E030E040E050E804C02FEF3FEF78
:1017E0004FEF5FE782E290E09093203180931F31CA
:1017F00016C0882341F050954095309521953F4F74
:101800004F4F5F4F0CC057FF0AC082E290E09093A9
:10181000203180931F312FEF3FEF4FEF5FE7B9018A
:10182000CA0104C060E070E080E090E0DF91CF91F9
:101830001F910F91FF90EF90DF90CF90BF90AF90EE
:101840009F908F907F906F905F903F902F90089522
:101850002F923F925F926F927F928F929F92AF9260
:10186000BF92CF92DF92EF92FF920F931F93CF938D
:10187000DF938B01EA016115710521F0DB018C9387
:1018800011969C93209739F09E0122503109233202
:10189000310508F0D8C07C016701BFEFCB1ADB0A25
:1018A0005601F7016080862D90E00E94368E892BCC
:1018B00011F07601F1CFFDE26F120AC0570182E00C
:1018C000A80EB11CD70111966C90772473940BC0AD
:1018D000BBE26B1207C05701E2E0AE0EB11CD701AC
:1018E00011966C90712CCE018F7E892B89F4B0E318
:1018F0006B1237C0F50180818F7D8835D1F461800E
:10190000F2E0AF0EB11C872D8260782EC0E1D0E0EE
:10191000CA30D10551F1C031D10521F0C830D1050F
:1019200099F409C0CC24CA94DC2CEC2CAFE0FA2E3C
:1019300022C0209769F7C8E0D0E0CC24CA94DC2C00
:10194000EC2CFFE1FF2E17C06FEF7FEFCB019E0164
:10195000442737FD4095542F0E94858869017A01FC
:101960000AC02097A9F6CAE0D0E0E9E9CE2EDC2C27
:10197000EC2CE9E1FE2EF50160E020E030E0A90169
:101980004E01AA2497FCA094BA2C1F0170ED572E8B
:10199000560CA9E0A51570F48FEB860D8A3118F46A
:1019A00099EC592E06C08FE9860D8A3148F589EAEF
:1019B000582E560C852D90E08C179D070CF56F3F27
:1019C000D9F0C216D306E406F50698F0C501B401B5
:1019D0000E944D889B01AC01852D90E0A0E0B0E015
:1019E000280F391F4A1F5B1F281739074A075B0753
:1019F00010F46FEF01C061E03196D1016C90C5CF5A
:101A00000115110551F0662311F0319703C071FEE5
:101A100004C03297D801ED93FC9370FE07C0509537
:101A20004095309521953F4F4F4F5F4F67FF10C056
:101A300082E290E09093203180931F316FEF7FEF2F
:101A40008FEF9FEF07C060E070E080E090E002C0A1
:101A5000B901CA01DF91CF911F910F91FF90EF90D3
:101A6000DF90CF90BF90AF909F908F907F906F90BE
:101A70005F903F902F900895662777270C94AC9045
:101A8000FC0188279927E89421912032E9F3293035
:101A900010F02E30C8F32B3241F02D3239F4689417
:101AA00004C00E94D18E820F911D219120532A30B3
:101AB000C0F31EF4909581959F4F0895283008F04B
:101AC00027E03327DA01990F311D87FD91600096D9
:101AD0006105710539F432602E5F3D9330E32A953C
:101AE000E1F708959F3F30F080387105610509F0F6
:101AF0003C5F3C5F3D93913008F08068911DDF931F
:101B0000CF931F930F93FF92EF92192F987F969583
:101B1000E92F96959695E90FFF27EE50FF4E9927EE
:101B20003327EE24FF24A701E701059008940794CA
:101B300028F4360FE71EF81E491F511D660F771F48
:101B4000881F991F0694A1F70590079428F4E70EC3
:101B5000F81E491F561FC11D770F881F991F661F4A
:101B60000694A1F70590079428F4F80E491F561F14
:101B7000C71FD11D880F991F661F771F0694A1F7F5
:101B80000590079420F4490F561FC71FD81F990FBF
:101B9000661F771F881F0694A9F784911095177008
:101BA00041F0D695C79557954795F794E7941A95C0
:101BB000C1F7E8E9F0E168941590159135916591C8
:101BC000959105907FE27395E118F10A430B560B4E
:101BD000C90BD009C0F7E10CF11E431F561FC91FE6
:101BE000D01D7EF4703311F48A95E6CFE89401504D
:101BF00030F0080F0AF40027021708F4202F23956D
:101C0000022F7A3328F079E37D932A95E9F710C003
